:100000000C94A8530C94D9530C94D9530C94D953F1
:100010000C94D9530C948A8C0C94D9530C94D953C6
:100020000C940B8C0C94D9530C94D9530C94A4ECD1
:100030000C94D9530D942BD60C94D9530C94D953BA
:100040000C94D9530D9438410C94D9530C94D95332
:100050000C94D9530C94D9530D9431570D945CCE14
:100060000C94D9530C9412650C94D9530C94D95315
:100070000C94D9530C94D9530C94D9530C94D95350
:100080000C94D9530C94D9530C94D9530C94D95340
:100090000C94D9530C94D9530C94D9530C94D95330
:1000A0000C94D9530C94D9530C94D9530C94D95320
:1000B0000C94D9530C94D9530C94D9530C94D95310
:1000C0000C94D9530C94D9530C94D9530C94526575
:1000D0000C94D9530C94D9530C94D9530C94D953F0
:1000E0000C94D953FF01D501EF01C901C101A3014E
:1000F000DB0181010902A101AD017501D701BF0139
:100100003D01CF0139018B014101DD017F013F013B
:10011000950177017301D9010B02FB019301E701FE
:100120005D010702BD01F101A701B7016F01670180
:100130006B016B016B01A901A901A901B9019B0127
:10014000A9015501BB01F701B101C701F5019701F3
:100150005701430135013B014B01F9019901E301CD
:10016000970147012F01D301F3018D015B01CD01FF
:10017000B50165014F01D101E101E90169018F017B
:1001800061019D016501370187014901084AD73B9B
:100190003BCE016E84BCBFFDC12F3D6C74319ABD56
:1001A00056833DDA3D00C77F11BED9E4BB4C3E917A
:1001B0006BAAAABE000000803F05A84CCDB2D44E69
:1001C000B93836A9020C50B9918688083CA6AAAA6B
:1001D0002ABE000000803F07634236B79BD8A71AAB
:1001E00039685618AEBAAB558C1D3CB7CC5763BDB9
:1001F0006DEDFD753EF6177231BF000000803F08BF
:10020000000000BE922449123EABAAAA2ABECDCC61
:10021000CC4C3E00000080BEABAAAAAA3E00000063
:1002200000BF000000803F0000000000084178D3BC
:10023000BB4387D1133D190E3CC3BD4282AD2B3E5B
:1002400068EC8276BED98FE1A93E4C80EFFFBE01FB
:10025000C4FF7F3F0000000000000D949EB70D9486
:1002600020D00D941A440D94BD870D94D5CF0D94D4
:1002700083D00D9495930D94DFCF0D9492580D94E7
:100280001A940D94D5930D94CDCF0D94C6670D940B
:1002900016D00D948BD00D94E9CF0D94D5670D94A5
:1002A0005DD00D94DDC30D94128B0D948B9F0D9436
:1002B000C5CF0D948A850D9448D00D94629B0D9402
:1002C000F1B30D9479D00D94CE840D9490D00D940B
:1002D000719F0D946FD00D94799F0D941A7D0D949C
:1002E000699F0D94B6860D949B9A0D944A580D946F
:1002F00050940D948D790D947F640D94D47E0D945B
:1003000010940D9434580D94D9B20D943B6D0D9406
:1003100087D00D945BBF0D94B4930D9459D00D9478
:1003200075D00D94256A0D942F9B0D9435940D94E2
:1003300034D00D9402D00D94AF9F0D947DD00D94C8
:1003400094730D943A580D9416580D94EC870D94AF
:10035000819C0D949F9F0D94167A0D943C580D949A
:100360004D1E0D94A7CF0D9427D10D9452D00D940E
:10037000A69C0D94819F0D949DCF0D944F9C0D9440
:1003800072580D9408580D94B0680D94C5840D945E
:10039000B1CF0D94EE570D9403AC0D944CD00D9449
:1003A0007A930D9461D00D942AD00D94C4570D9476
:1003B00064580D94B39A0D9430580D9406940D948E
:1003C000F4650D9467D00D940CD00D943FBC0D9442
:1003D000439B0D946BD00D94D7840D94DB670D94E3
:1003E000E0570D94649C0D9456D00D94BBCF0D94A2
:1003F000A2CF0D94F3CF0D941B9B0D9459830D94B4
:10040000B6570D94E0840D9431760D94A7900D9419
:100410002E9C0D9436580D94CC9A0D949967486192
:100420007264636F6465642044656661756C7420F2
:1004300053657474696E6773204C6F616465640002
:1004400053746F7265642073657474696E6773208A
:1004500072657472696576656400202020452F44BA
:10046000203D20002020204D393030204B004C69A9
:100470006E65617220616476616E63652073657478
:1004800074696E67733A0046696C616D656E7420BD
:1004900073657474696E67733A2044697361626C42
:1004A0006564002020204D32303020440046696CC5
:1004B000616D656E742073657474696E67733A005C
:1004C0002020204D3230392053004175746F2D5259
:1004D0006574726163743A20533D3020746F2064F8
:1004E000697361626C652C203120746F20696E74B1
:1004F00065727072657420657874727564652D6FAD
:100500006E6C79206D6F76657320617320726574EF
:100510007261637473206F72207265636F766572A7
:10052000696573002046002020204D32303820536A
:10053000005265636F7665723A20533D4578747258
:1005400061206C656E67746820286D6D2920463ABD
:10055000537065656420286D6D2F6D2900205A0049
:100560002046002020204D32303720530052657441
:10057000726163743A20533D4C656E67746820283D
:100580006D6D2920463A537065656420286D6D2F86
:100590006D29205A3A205A4C69667420286D6D29BD
:1005A000002044002049002020204D3330342050CA
:1005B0000050494420686561746265642073657405
:1005C00074696E67733A002044002049002020209F
:1005D0004D333031205000504944207365747469A4
:1005E0006E67733A00205A0020590020204D3230A7
:1005F00036205800486F6D65206F666673657420FD
:10060000286D6D293A00204500205A00205900200D
:10061000580020420020540020204D323035205315
:1006200000416476616E636564207661726961621F
:100630006C65733A20533D4D696E20666565647242
:1006400061746520286D6D2F73292C20543D4D69F0
:100650006E2074726176656C206665656472617483
:100660006520286D6D2F73292C20423D6D696E69C0
:100670006D756D207365676D656E742074696D6549
:1006800020286D73292C20583D6D6178696D756D3A
:10069000205859206A65726B20286D6D2F73292CA4
:1006A00020205A3D6D6178696D756D205A206A650C
:1006B000726B20286D6D2F73292C2020453D6D61B4
:1006C00078696D756D2045206A65726B20286D6DA7
:1006D0002F73290020540020204D32303420530045
:1006E000416363656C65726174696F6E3A20533D56
:1006F000616363656C65726174696F6E2C20543D33
:100700007265747261637420616363656C657261A4
:1007100074696F6E00204500205A00205900202087
:100720004D3230312058004D6178696D756D204132
:100730006363656C65726174696F6E20286D6D2FDF
:100740007332293A00204500205A00205900202009
:100750004D3230332058004D6178696D756D2066DB
:10076000656564726174657320286D6D2F73293A15
:1007700000204500205A0020590020204D39322009
:10078000580053746570732070657220756E6974BB
:100790003A0053657474696E67732053746F7265A1
:1007A0006400454550524F4D204572726F720000F3
:1007B00020006D65736820626564206C6576656CE9
:1007C000696E673A200029002C20002C20007068F8
:1007D00079736963616C20636F6F7264696E6174B1
:1007E00065733A20280029002C20002C2000776F08
:1007F000726C6420636F6F7264696E617465733AC2
:100800002028002046002045004731205A004D3264
:1008100034004D32362053256C75004D3130362072
:10082000530047312046256400473120453120469A
:10083000343830004731205A002046323030300002
:1008400020590047312058004D383300506F7369EC
:1008500074696F6E20726561642066726F6D2065C9
:100860006570726F6D3A004D3233202573002E672C
:10087000636F0046656564726174653A0072656312
:100880006F7665725F6D616368696E655F737461D1
:1008900074655F61667465725F706F7765725F70B3
:1008A000616E69632C20696E697469616C200072E5
:1008B00065636F7665725F6D616368696E655F73AE
:1008C000746174655F61667465725F706F7765727D
:1008D0005F70616E69632C20696E697469616C2058
:1008E000007265636F7665725F6D616368696E65DE
:1008F0005F73746174655F61667465725F706F7752
:1009000065725F70616E69632C20696E69746961DC
:100910006C200063757272656E745F706F736974BA
:10092000696F6E5B5A5F415849535D3A0043757277
:1009300072656E7420706F736974696F6E20595F91
:10094000415849533A0043757272656E7420706F56
:10095000736974696F6E20585F415849533A00417A
:10096000667465722077616974696E6720666F725C
:100970002074656D703A00473120452D3120463492
:1009800038300047312045352046313230004D386F
:1009900033004D31393020532564004D313039203A
:1009A0005325640047323820582059004731205AD7
:1009B00032352046383030004D31343020532564F4
:1009C000004D3130342053256400494E54340055D5
:1009D000564C4F202D20656E640073747073005563
:1009E000564C4F0020423A0020453A00543A005AF3
:1009F000206C6976652061646A757374206F757404
:100A0000206F662072616E67652E2053657474696D
:100A10006E6720746F20302E20436C69636B2074E6
:100A20006F20636F6E74696E75652E005A206C6955
:100A300076652061646A757374206F7574206F66C3
:100A40002072616E67652E2053657474696E67202D
:100A5000746F20300020573A0020453A00543A0085
:100A60004B494C4C3A20004175746F0020452F448F
:100A70003D00416476616E6365204B3D0022283263
:100A80002900443130303000473238205900473295
:100A9000382058005400496E76616C6964205420F7
:100AA000636F64652E00496E76616C6964204D2029
:100AB000636F64652E004D3232302053256900206B
:100AC0003A2000004C414E472053454C20464F529F
:100AD00043454400222831290020453A00205A3A53
:100AE0000020593A0020453A00205A3A0020593A4D
:100AF00000583A0020002E0020423A0020453A00DB
:100B0000543A0020413A0020503A002042403A0036
:100B100020403A00202F003A00205400202F0020CF
:100B2000423A00202F006F6B20543A002569206D57
:100B3000696E2C2025692073656300496E76616CAF
:100B40006964204D20636F6465004D6573682062A1
:100B50006564206C6576656C696E67206E6F7420C5
:100B60006163746976652E000A002020000A4D65D5
:100B700061737572656420706F696E74733A000AF0
:100B80005A20736561726368206865696768743AA2
:100B900020002C004E756D20582C593A2000476FCC
:100BA00020686F6D652066696E6973686564004DC5
:100BB00065736820626564206C6576656C696E6734
:100BC0002061637469766174656400557073616D4A
:100BD000706C652066696E6973686564004265645F
:100BE000206C6576656C696E6720636F72726563F1
:100BF00074696F6E2066696E697368656400206D44
:100C00006963726F6E7300457863657373697665A7
:100C100020626564206C6576656C696E6720636F21
:100C20007272656374696F6E3A20006261627973F3
:100C3000746570206170706C69656400636C6561D7
:100C40006E2075702066696E697368656420004760
:100C50003238205730003A200054656D706572615B
:100C6000747572652063616C6962726174696F6E1C
:100C700020646F6E652E20436F6E74696E756520FB
:100C800077697468207072657373696E6720746821
:100C900065206B6E6F622E0000205A2073686966B3
:100CA0007420286D6D293A0050494E4441207465E6
:100CB0006D70657261747572653A2000002F3600A0
:100CC000537465703A200000205A20736869667476
:100CD00020286D6D293A0050494E44412074656DBD
:100CE00070657261747572653A20002F3620287322
:100CF0006B69707065642900537465703A20000058
:100D00005A45524F3A200000737461727420746522
:100D10006D70657261747572653A200050494E4479
:100D2000412070726F62652063616C6962726174E8
:100D3000696F6E20737461727400473238205730C7
:100D4000000A00205A3A200020593A200020583A40
:100D500020004732382C2066696E616C20004732D3
:100D6000382C2066696E616C20004732382C206672
:100D7000696E616C20004732382C20696E69746995
:100D8000616C20004732382C20696E697469616C8F
:100D9000200044393939004D3239002055706C6FCC
:100DA000616420696E2070726F6772657373006989
:100DB0006E697469616C207A737465707320616602
:100DC0007465722072657365743A2000696E697487
:100DD00069616C207A7374657073206F6E20706F18
:100DE0007765722075703A2000466163746F72797E
:100DF00020524553455400202020203344202050C9
:100E000072696E7465727320202020002020204FAC
:100E1000726967696E616C20507275736120202061
:100E2000004E6F76203133203230313700436F6D02
:100E300070696C65643A2000286E6F6E652C2064C2
:100E4000656661756C7420636F6E66696729004E14
:100E50006F7620313320323031372032313A323020
:100E60003A343000737461727400202020203344BF
:100E700020205072696E746572732020202000203B
:100E800020204F726967696E616C205072757361C2
:100E900020202000250020202020202000202020AD
:100EA0002020200045524153494E4720616C6C2060
:100EB0006461746100466163746F727920524553B6
:100EC000455400FFFFFF0000A0400000A0400000CC
:100ED000004000007A4300005E439AD9514300006D
:100EE0000000000040C19A99193E00007A430000BA
:100EF00052430000524300000000000040C19A9994
:100F0000193E6563686F3A004572726F723A00006D
:100F1000002110422063308440A550C660E770086D
:100F20008129914AA16BB18CC1ADD1CEE1EFF131F4
:100F300012100273325222B5529442F772D66239BD
:100F40009318837BB35AA3BDD39CC3FFF3DEE36244
:100F500024433420040114E664C774A44485546A0D
:100F6000A54BB528850995EEE5CFF5ACC58DD553D4
:100F700036722611163006D776F6669556B4465B5D
:100F8000B77AA719973887DFF7FEE79DD7BCC7C4A4
:100F900048E5588668A7784008611802282338CCAD
:100FA000C9EDD98EE9AFF9488969990AA92BB9F534
:100FB0005AD44AB77A966A711A500A333A122AFDFD
:100FC000DBDCCBBFFB9EEB799B588B3BBB1AABA604
:100FD0006C877CE44CC55C222C033C600C411CAE4D
:100FE000ED8FFDECCDCDDD2AAD0BBD688D499D9714
:100FF0007EB66ED55EF44E133E322E511E700E9F9D
:10100000FFBEEFDDDFFCCF1BBF3AAF599F788F8863
:1010100091A981CAB1EBA10CD12DC14EF16FE18034
:1010200010A100C230E3200450254046706760B92B
:10103000839893FBA3DAB33DC31CD37FE35EF3B184
:10104000029012F322D2323542145277625672EA7B
:10105000B5CBA5A89589856EF54FE52CD50DC5E2D4
:1010600034C324A01481046674476424540544DB0B
:10107000A7FAB79987B8975FE77EF71DC73CD7D324
:1010800026F2369106B01657667676154634564CDB
:10109000D96DC90EF92FE9C899E9898AB9ABA94474
:1010A00058654806782768C018E1088238A3287D6B
:1010B000CB5CDB3FEB1EFBF98BD89BBBAB9ABB75C4
:1010C0004A545A376A167AF10AD01AB32A923A2E3B
:1010D000FD0FED6CDD4DCDAABD8BADE89DC98D2614
:1010E0007C076C645C454CA23C832CE01CC10C1F4B
:1010F000EF3EFF5DCF7CDF9BAFBABFD98FF89F1764
:101100006E367E554E745E932EB23ED10EF01E7C2E
:101110003C3E5E2B3D3F2F5B5D3B2C2A225C004D0D
:10112000383420582059205A2045004D3234004D83
:101130003233202573006175746F25692E67000AAC
:10114000002F000A002E0044656C6574696F6E20E4
:101150006661696C65642C2046696C653A200046BE
:10116000696C652064656C657465643A002E002EB8
:10117000002E002E004E6F77206672657368206621
:10118000696C653A20004E6F7720646F696E672046
:1011900066696C653A20002220706F73002220700F
:1011A0006172656E743A2200535542524F5554494C
:1011B0004E452043414C4C207461726765743A225D
:1011C00000747279696E6720746F2063616C6C20A3
:1011D0007375622D67636F64652066696C65732043
:1011E0007769746820746F6F206D616E79206C650B
:1011F00076656C732E204D4158206C6576656C20A9
:1012000069733A00256920686F757273202569201B
:101210006D696E757465730054494D454F55543A68
:10122000004D3131300046756C6C205258204275AB
:10123000666665720022206661696C65643A2042C8
:1012400075666665722066756C6C2100456E7175F9
:1012500065696E6720746F207468652066726F6EB2
:10126000743A2022002200456E717565696E672010
:10127000746F207468652066726F6E743A20220065
:1012800022206661696C65643A2042756666657203
:101290002066756C6C210022004D36303000507293
:1012A000757361206933204D4B3320626572656927
:1012B000742E005072757361206933204D4B3320BA
:1012C000676F746F776100507275736120693320A6
:1012D0004D4B3320707265702E0050727573612013
:1012E0006933204D4B332070726F6E74612E005045
:1012F00072757361206933204D4B33206F6B005042
:1013000072757361206933204D4B332072656164BF
:10131000792E007A5F6D696E3A20007A5F6D617890
:101320003A20005A204F666673657400795F6D69D4
:101330006E3A2000795F6D61783A20004A6100546E
:10134000616B00536900536900416E6F005965730A
:1013500000785F6D696E3A2000785F6D61783A20A1
:1013600000496368207765726465206A65747A74E1
:1013700020646965205A204B616C696272696572EC
:10138000756E672064757263686675656872656EF0
:101390002E00576C61637A616D206B616C696272BB
:1013A00061636A65207A2E00566F7920612068613A
:1013B0006365722043616C6962726163696F6E205C
:1013C0005A2061686F72612E0041646573736F20EB
:1013D0006176766965726F20756E612043616C6914
:1013E0006272617A696F6E65205A2E004E796E695D
:1013F0002070726F76656475207A206B616C69620B
:10140000726163692E00492077696C6C2072756E79
:10141000207A2063616C6962726174696F6E206EFC
:101420006F772E00496368207765726465206A656E
:10143000747A74206469652058595A2D4B616C691F
:101440006272696572756E6720647572636866752D
:10145000656872656E2E204573207769726420631B
:10146000612E203132204D696E7574656E20646185
:101470007565726E00576C61637A616D206B616C8B
:1014800069627261636A652078797A2E205A616A8E
:101490006D696520746F206F6B2E203132206D696D
:1014A0006E2E0048617265206C612063616C696218
:1014B000726163696F6E2058595A2E2054617264AC
:1014C000617261203132206D696E2E206170726F01
:1014D00078696D6164616D656E74652E0041646547
:1014E00073736F206176766965726F20756E612007
:1014F00043616C696272617A696F6E652058595AEE
:101500002E2050756F206475726172652063697258
:101510006361203132206D696E2E004E796E692034
:1015200070726F766564752078797A206B616C696A
:1015300062726163692E205A616265726520746F00
:1015400020707269626C697A6E65203132206D6933
:101550006E2E00492077696C6C2072756E20787948
:101560007A2063616C6962726174696F6E206E6F5C
:10157000772E2049742077696C6C2074616B65202C
:10158000617070726F782E203132206D696E732E0B
:10159000004A65747A7420776572646520696368AF
:1015A00020646965204475657365206675657220E1
:1015B000504C4120766F726865697A656E2E200006
:1015C0004E6167727A6577616D206479737A652000
:1015D000646C6120504C412E00566F792061207060
:1015E000726563616C656E74617220656C206E6FEC
:1015F0007A7A6C65207061726120504C412061687C
:101600006F72612E0041646573736F207072657232
:10161000697363616C6465726F206C277567656CB4
:101620006C6F2070657220504C412E004E796E69AF
:101630002070726564656872656A69207472797376
:101640006B752070726F20504C412E004E6F7720CA
:10165000492077696C6C2070726568656174206ED2
:101660006F7A7A6C6520666F7220504C412E00486C
:10167000616C6C6F2C206963682062696E20646500
:10168000696E204F726967696E616C205072757364
:101690006120693320447275636B65722E204D6F33
:1016A00065636874656E20536965206D65696E6554
:1016B0002048696C66652064757263682064656E95
:1016C0002053657475702D50726F7A6573733F0087
:1016D000437A6573632C206A657374656D20547753
:1016E0006F6A61206472756B61726B61204F726901
:1016F00067696E616C2050727573612069332E20AA
:10170000437A7920706F74727A6562756A65737A4C
:1017100020706F6D6F6379207A20696E7374616CCD
:1017200061636A613F00486F6C612C20736F7920A0
:10173000747520696D707265736F7261204F726984
:1017400067696E616C2050727573612069332E2059
:1017500051756965726573207175652074652067C0
:1017600075696520612074726176657320646520F7
:101770006C6120636F6E66696775726163696F6E15
:101780003F004369616F2C20736F6E6F206C612086
:10179000747561207374616D70616E7465204F7231
:1017A0006967696E616C2050727573612069332EB0
:1017B0002047726164697265737469206169757428
:1017C0006F206174747261766572736F20696C202A
:1017D00070726F636573736F20646920636F6E66E8
:1017E00069677572617A696F6E653F00446F6272F6
:1017F000792064656E2C206A73656D20766173654F
:10180000207469736B61726E61204F726967696ED3
:10181000616C2050727573612069332E20436863B8
:101820006574652061627963682056617320707207
:101830006F7665646C61206B616C69627261636E66
:10184000696D2070726F636573656D3F0048692C28
:10185000204920616D20796F7572204F7269676928
:101860006E616C20507275736120693320707269EB
:101870006E7465722E20576F756C6420796F7520B9
:101880006C696B65206D6520746F20677569646590
:1018900020796F75207468726F7567682074686549
:1018A0002073657475702070726F636573733F0089
:1018B000496368207765726465206A65747A74206C
:1018C0006572737465204C696E6965206472756316
:1018D0006B656E2E205761656872656E6420646565
:1018E0007320447275636B6573206B6F656E6E65F4
:1018F0006E205369652064696520447565736520B1
:10190000616C6C6D6165686C6963682073656E6B92
:10191000656E20696E64656D205369652064656E2F
:10192000204B6E6F70662064726568656E2C206255
:1019300069732053696520646965206F7074696DEF
:10194000616C6520486F65686520657272656963C2
:1019500068656E2E20556562657270727565666584
:101960006E20536965206469652042696C64657204
:1019700020696E20756E736572656D2048616E64B6
:101980006275636820696D204B61706974656C20B5
:101990004B616C696272696572756E67005A61634A
:1019A0007A6E65206472756B6F776163206C696E07
:1019B00069652E2053746F706E696F776F206F703A
:1019C00075737A637A616A206479737A65207072BC
:1019D0007A656B726563616A61632067757A696BAA
:1019E0002C20706F6B69206E696520757A79736B36
:1019F00061737A206F7074796D616C6E656A20779F
:101A000079736F6B6F7363692E20537072617764A3
:101A10007A206F6272617A6B692077206E61737AC7
:101A2000796D20706F7261646E696B7520772072BA
:101A30006F7A647A2E204B616C69627261636A61AD
:101A400000566F79206120636F6D656E7A61722038
:101A50006120696D7072696D6972206C61206C69BA
:101A60006E656120792074752062616A61726173AC
:101A700020656C206E6F7A7A6C6520677261647580
:101A8000616C6D656E746520616C20726F7461723B
:101A900020656C206D616E646F2C206861737461C9
:101AA00020717565206C6C65677565732061206CAD
:101AB0006120616C74757261206F7074696D612E44
:101AC000204D697261206C617320696D6167656E7C
:101AD00065732064656C206361706974756C6F2038
:101AE00043616C6962726163696F6E20656E206527
:101AF0006C206D616E75616C2E0041646573736F4F
:101B000020696E697A6965726F2061207374616DF6
:101B10007061726520756E61206C696E656120650B
:101B200020747520646F76726169206162626173EE
:101B300073617265206C277567656C6C6F20706FC0
:101B4000636F2070657220766F6C74612072756FA0
:101B500074616E646F206C61206D616E6F706F6C6C
:101B6000612073696E6F2061207261676769756EAD
:101B70006765726520756E6120616C74657A7A6143
:101B8000206F7474696D616C652E205065722066DB
:101B900061766F72652064616920756E6F2073676E
:101BA000756172646F20616C6C27696D6D61676926
:101BB0006E652064656C206E6F7374726F206D614A
:101BC0006E75616C652C206361702E43616C696277
:101BD00072617A696F6E652E005A61636E7520744A
:101BE00069736B6E6F7574206C696E6B7520612004
:101BF00056792062756465746520706F73747570B2
:101C00006E6520736E697A6F766174207472797371
:101C10006B75206F746163656E696D20746C6163B0
:101C200069746B6120646F6B7564206E65646F739B
:101C300061686E657465206F7074696D616C6E6942
:101C4000207679736B792E2050726F686C65646EA4
:101C5000657465207369206F6272617A6B79207692
:101C6000206E617369207072697275636365207696
:101C7000206B617069746F6C65204B616C69627276
:101C800061636500492077696C6C207374617274BC
:101C900020746F207072696E74206C696E652061AB
:101CA0006E6420796F752077696C6C20677261644F
:101CB00075616C6C79206C6F776572207468652033
:101CC0006E6F7A7A6C6520627920726F74617469C4
:101CD0006E6720746865206B6E6F622C20756E7461
:101CE000696C20796F75207265616368206F70740C
:101CF000696D616C206865696768742E204368654A
:101D0000636B2074686520706963747572657320F5
:101D1000696E206F75722068616E64626F6F6B20F0
:101D2000696E20636861707465722043616C6962DA
:101D3000726174696F6E2E004A65747A74207765DB
:101D4000726465206963682064656E204162737403
:101D5000616E64207A7769736368656E2044756587
:101D600073656E737069747A6520756E6420447251
:101D700075636B62657474206B616C69627269650E
:101D800072656E2E004B616C696272756A65206FB8
:101D9000646C65676C6F7363206D6965647A792024
:101DA0006B6F6E636F776B61206479737A792061F2
:101DB0002073746F6C696B69656D2E00566F7920A6
:101DC000612063616C6962726172206C6120646978
:101DD0007374616E63696120656E747265206C61F5
:101DE0002070756E74612064656C206E6F7A7A6CF9
:101DF000652079206C61207375706572666963690E
:101E000065206465206C6120686561746265642E7C
:101E10000041646573736F2074617265726F206C2A
:101E20006F2073746163636F2066726120756765EC
:101E30006C6C6F20652073757065726669636520D0
:101E400064656C2070696174746F2E004E796E69E0
:101E5000207A6B616C696272756A6920767A646156
:101E60006C656E6F7374206D657A69206B6F6E633D
:101E7000656D20747279736B79206120706F767252
:101E80006368656D2068656174626564752E004ED7
:101E90006F7720492077696C6C2063616C6962728E
:101EA0006174652064697374616E63652062657432
:101EB0007765656E20746970206F66207468652090
:101EC0006E6F7A7A6C6520616E64206865617462F9
:101ED000656420737572666163652E005A756E6164
:101EE00065636873742066756568726520696368E8
:101EF0002064656E2053656C62737474657374201E
:101F0000647572636820756D206469652068616519
:101F1000756669677374656E2050726F626C656D6B
:101F2000652062656920646572204175666261752D
:101F3000207A752075656265727072756566656E6A
:101F40002E004E616A706965727720776C61637AE2
:101F500065206175746F7465737420772063656C98
:101F600075206B6F6E74726F6C6C69206E616A6342
:101F70007A657374737A7963682070726F626C65C6
:101F80006D6F77207A206D6F6E74617A656D2E00AB
:101F90005072696D65726F2C206861726520656C86
:101FA0002053656C66746573742070617261206380
:101FB0006F6D70726F626172206C6F732070726FE0
:101FC000626C656D6173206465206D6F6E74616A0B
:101FD00065206D617320636F6D756E65732E0041B2
:101FE0006E7A69747574746F206176766965726F44
:101FF00020696C2053656C6620546573742070658D
:102000007220636F6E74726F6C6C61726520676CA6
:1020100069206572726F72692064692061737365EB
:102020006D626C616767696F2070697520636F6DA1
:10203000756E692E004E656A6472697620706F6DE8
:102040006F63692073656C667465737475207A6B51
:102050006F6E746F6C756A69206E656A6361737404
:10206000656A736920636879627920767A6E696B34
:10207000616A69636920707269207365737461763F
:10208000656E69207469736B61726E792E004669A2
:102090007273742C20492077696C6C2072756E20E5
:1020A0007468652073656C667465737420746F2042
:1020B000636865636B206D6F737420636F6D6D6F04
:1020C0006E20617373656D626C792070726F626CE3
:1020D000656D732E00446572206C617566656E6473
:1020E0006520417373697374656E74206C6F6573DA
:1020F0006368742064696520616B7475656C6C65D8
:10210000204B616C69627269657265726765626EA7
:102110006973736520756E64207769726420766FC9
:102120006E20416E66616E6720616E206265676930
:102130006E6E656E2E20466F72747365747A656E6E
:102140003F00576C61637A656E69652057697A61F3
:102150007264207573756E6965206F6265636E6564
:102160002064616E65206B616C6962726163796A7B
:102170006E652069207A61637A6E6965206F6420DC
:102180006E6F77612E204B6F6E74796E756F77610D
:10219000633F00456A65637574617220656C205702
:1021A000697A61726420626F7272617261206C6F11
:1021B000732076616C6F7265732064652063616C57
:1021C0006962726163696F6E2061637475616C65C9
:1021D00073207920636F6D656E7A6172612064652A
:1021E000206E7565766F2E20436F6E74696E756113
:1021F000723F005365206176766920696C205769CB
:102200007A617264207065726465726169206C61C4
:102210002063616C696272617A696F6E65207072A9
:10222000656573697374656E7465206520646F7687
:10223000726169207269636F6D696E63696172654D
:102240002064616C6C27696E697A696F2E20436F18
:102250006E74696E756172653F0053707573746555
:102260006E692057697A617264612076796D617A4E
:102270006520756C6F7A656E65207679736C656420
:102280006B79207673656368206B616C696272613B
:102290006369206120737075737469206B616C6968
:1022A000627261636E692070726F636573206F6420
:1022B000207A616361746B752E20506F6B7261635D
:1022C0006F7661743F0052756E6E696E6720576954
:1022D0007A6172642077696C6C2064656C657465E2
:1022E0002063757272656E742063616C69627261DD
:1022F00074696F6E20726573756C747320616E649F
:102300002073746172742066726F6D20746865202A
:10231000626567696E6E696E672E20436F6E7469C1
:102320006E75653F004D6F65636874656E20536917
:10233000652064656E206C65747A74656E205363E5
:10234000687269747420776965646572686F6C651A
:102350006E20756D2064656E2041627374616E64D9
:10236000207A7769736368656E20447565736520AC
:10237000756E6420447275636B62657474206E655B
:10238000752065696E7A757374656C6C656E3F0057
:1023900043686365737A20706F77746F727A7963BC
:1023A000206F737461746E69206B726F6B2069208B
:1023B00070727A65737461776963206F646C6567A6
:1023C0006C6F7363206D6965647A79206479737AC0
:1023D0006120612073746F6C696B69656D3F00519A
:1023E00075696572657320726570657469722065C0
:1023F0006C20756C74696D6F207061736F207061F3
:102400007261207265616A7573746172206C6120FB
:1024100064697374616E636961206E6F7A7A6C654A
:102420002D686561746265643F0044657369646525
:102430007269207269706574657265206C27756CAD
:1024400074696D6F2070617373616767696F207065
:102450006572206D69676C696F72617265206C616D
:102460002064697374616E7A612066726120756799
:10247000656C6C6F20652070696174746F3F0043F8
:102480006863657465206F70616B6F76617420702E
:102490006F736C65646E69206B726F6B2061207066
:1024A0006F7A6D656E697420767A64616C656E6FA3
:1024B0007374206D657A6920747279736B6F7520FF
:1024C0006120686561746265643F00446F20796FC4
:1024D000752077616E7420746F2072657065617409
:1024E000206C617374207374657020746F20726542
:1024F00061646A7573742064697374616E636520C6
:102500006265747765656E206E6F7A7A6C6520619E
:102510006E6420686561746265643F00536965207C
:102520006B6F656E6E656E20696D6D65722064659A
:102530006E204173697374656E74656E20696D20D9
:102540004D656E75206E6575206175667275666580
:102550006E3A204B616C696272696572756E6720B4
:102560002D3E20417373697374616E74005A6177F4
:10257000737A65206D6F7A65737A2070727A7977D5
:10258000726F6369632057697A6172642070727A2E
:10259000657A204B616C69627261636A61202D3ECD
:1025A0002057697A6172642E005369656D70726597
:1025B000207075656465732061636365646572206E
:1025C000616C206173697374656E746520646573F2
:1025D00064652043616C6962726163696F6E202D6E
:1025E0003E2057697A617264004520706F73736989
:1025F00062696C652070726F7365677569726520BA
:102600006C612067756964652057697A617264201E
:10261000696E207175616C7369617369206D6F6D8E
:10262000656E746F206174747261766572736F2069
:1026300043616C696272617A696F6E65202D3E201C
:1026400057697A6172642E0057697A6172646120F9
:102650006D757A657465206B64796B6F6C69762033
:102660007A6E6F76752073707573746974207A2032
:102670006D656E752043616C6962726174696F6E1D
:10268000202D3E2057697A61726400596F7520636E
:10269000616E20616C7761797320726573756D6509
:1026A000207468652057697A6172642066726F6D64
:1026B0002043616C6962726174696F6E202D3E20E7
:1026C00057697A6172642E004973742065732077AC
:1026D00069726B6C69636820504C412046696C617B
:1026E0006D656E743F00437A7920746F2066696C63
:1026F000616D656E7420504C413F00457320656CE0
:102700002066696C616D656E746F20504C413F00AE
:10271000452071756573746F20756E2066696C61F4
:102720006D656E746F20646920504C413F004A65AE
:1027300020746F20504C412066696C616D656E7429
:102740003F00497320697420504C412066696C61D8
:102750006D656E743F004675656872656E205369DD
:102760006520626974746520504C412046696C6133
:102770006D656E7420696E2064656E204578747294
:102780007564657220756E6420626573746165742A
:102790006967656E205369652064656E204B6E6FB6
:1027A000706620756D206573207A75206C61646594
:1027B0006E2E0050726F737A6520756D6965736354
:1027C0002066696C616D656E7420504C41207720E5
:1027D000656B737472756465727A652069206E61C9
:1027E0006369736E696A2070727A796369736B20AA
:1027F0006279207A616C61646F7761632E00496E43
:1028000073657274612C20706F72206661766F72CE
:102810002C2066696C616D656E746F20504C412090
:10282000656E20656C206578747275736F722E20EA
:10283000446573707565732068617A20636C6963A1
:102840002070617261206361726761726C6F2E002B
:10285000506572206661766F726520696E7365726D
:102860006973636920696C2066696C616D656E745B
:102870006F20646920504C41206E656C6C27657335
:10288000747275736F72652C20706F692070726539
:102890006D69206C61206D616E6F706F6C6120706E
:1028A00065722063617269636172652E0050726F98
:1028B00073696D20766C6F7A746520504C41206688
:1028C000696C616D656E7420646F206578747275D3
:1028D000646572752C20706F207465207374697341
:1028E0006B6E65746520746C616369746B6F2070C6
:1028F000726F207A61766564656E692066696C61C5
:102900006D656E74752E00506C6561736520696E1F
:102910007365727420504C412066696C616D656E00
:102920007420746F207468652065787472756465AE
:10293000722C207468656E207072657373206B6EE4
:102940006F6220746F206C6F61642069742E004286
:1029500069747465206C6164656E205369652050EC
:102960004C412D46696C616D656E7420756E6420F6
:1029700066616872656E20536965206D69742064B4
:10298000656D20417373697374656E74656E20663E
:102990006F72742C20696E64656D205369652064C4
:1029A000656E20447275636B6572206E6575207369
:1029B00074617274656E2E0050726F737A65207A3E
:1029C000616C6164756A2066696C616D656E742006
:1029D000504C4120692070727A7977726F6320576A
:1029E000697A6172642070727A657A207265737494
:1029F000617274206472756B61726B692E00436141
:102A00007267612066696C616D656E746F20504CF1
:102A1000412C20706F72206661766F722C207920B5
:102A20007265696E69636961206C6120696D70729D
:102A300065736F7261207061726120636F6E74697B
:102A40006E75617220636F6E20656C2057697A61C4
:102A5000726400506572206661766F7265206361F2
:102A6000726963612066696C616D656E746F206464
:102A70006920504C4120652072697072656E6469EE
:102A800020696C2057697A61726420646F706F20CE
:102A9000617665722072696176766961746F206C07
:102AA00061207374616D70616E74652E0050726F79
:102AB00073696D207A61766564746520504C41209D
:102AC00066696C616D656E74206120706F2074653D
:102AD000206F626E6F7674652057697A61726461E7
:102AE00020737469736B6E7574696D20726573659C
:102AF0007420746C616369746B612E00506C656145
:102B00007365206C6F616420504C412066696C6174
:102B10006D656E7420616E64207468656E207265E8
:102B200073756D652057697A6172642062792072CD
:102B300065626F6F74696E67207468652070726972
:102B40006E7465722E00566F726865697A656E20C4
:102B50006465722044756573652E204269747465DE
:102B60002077617274656E2E004E6167727A6577A8
:102B7000616E6965206479737A792E2050726F7363
:102B80007A6520637A656B61632E005072656361BC
:102B90006C656E74616E646F206E6F7A7A6C652EF0
:102BA0002045737065726120706F72206661766F68
:102BB000722E0053746F2070726572697363616C5A
:102BC00064616E646F206C277567656C6C6F2E2076
:102BD000506572206661766F726520617474656EEF
:102BE00064692E00507265646568726976616D2053
:102BF000747279736B752E2050726F73696D2063D8
:102C0000656B656A74652E005072656865617469EC
:102C10006E67206E6F7A7A6C652E20506C656173DA
:102C20006520776169742E00497374206461732094
:102C300046696C616D656E742067656C6164656E74
:102C40003F0046696C616D656E74206A657374201F
:102C50007A616C61646F77616E793F00457374616E
:102C600020656C2066696C616D656E746F206361B0
:102C7000726761646F3F00496C2066696C616D65C5
:102C80006E746F206520737461746F206361726964
:102C90006361746F3F004A652066696C616D656EA3
:102CA00074207A61766564656E3F004973206669B9
:102CB0006C616D656E74206C6F616465643F00418A
:102CC0006C6C657320777572646520676574616EDE
:102CD0002E205669656C205370617373206265699C
:102CE0006D20447275636B656E2100476F746F775A
:102CF000652E205564616E65676F206472756B7513
:102D000021005465726D696E61646F212046656CA7
:102D1000697A20696D70726573696F6E2100426512
:102D20006E20666174746F2E2042756F6E61207321
:102D300074616D70612100567365206A6520686F4B
:102D4000746F766F2E00416C6C20697320646F6E17
:102D5000652E204861707079207072696E74696E9A
:102D60006721004269747465207265696E696765E0
:102D70006E2053696520646173204865697A6265D5
:102D8000747420756E642064727565636B656E2063
:102D90005369652064616E6E2064656E204B6E6FB2
:102DA00070662E0050726F737A65206F637A797344
:102DB000632073746F6C696B2069206E6163697343
:102DC0006E696A2067757A696B2E004C696D70694F
:102DD00061206C6120737570657266696369652036
:102DE0006465206C6120686561746265642C207084
:102DF0006F72206661766F722C20792068617A206C
:102E0000636C696300506572206661766F7265203D
:102E100070756C6973636920696C20706961747482
:102E20006F2C20706F69207072656D69206C612055
:102E30006D616E6F706F6C612E0050726F73696D93
:102E4000206F636973746574652068656174626579
:102E500064206120737469736B6E65746520746C93
:102E6000616369746B6F2E00506C656173652063DC
:102E70006C65616E206865617462656420616E6472
:102E8000207468656E2070726573732074686520A5
:102E90006B6E6F622E0042697474652075656265A1
:102EA000727072756566656E2053696520756E7304
:102EB00065722048616E646275636820756E642077
:102EC0006265686562656E20536965206461732080
:102ED00050726F626C656D2E2046616872656E205F
:102EE0005369652064616E6E206D69742064656D40
:102EF00020417373697374656E74656E20666F72BA
:102F0000742C20696E64656D205369652064656E5C
:102F100020447275636B6572206E657520737461F1
:102F20007274656E2E0050726F737A6520737072C2
:102F30006177647A206E61737A20706F7261646E5B
:102F4000696B2069206E61707261772070726F62A8
:102F50006C656D2E20506F74656D2070727A797774
:102F6000726F632057697A6172642072657374614D
:102F70007274756A6163206472756B61726B652E21
:102F8000004C656520656C206D616E75616C207903
:102F90002072657375656C766520656C2070726F44
:102FA000626C656D612E20446573707565732C20AD
:102FB0007265696E69636961206C6120696D707208
:102FC00065736F7261207920636F6E74696E7561CD
:102FD00020636F6E20656C2057697A6172640050BF
:102FE0006572206661766F726520636F6E73756CB3
:102FF000746120696C206E6F7374726F206D616EE6
:1030000075616C6520706572207269736F6C76658E
:10301000726520696C2070726F626C656D612E2024
:10302000506F692072697072656E646920696C20E6
:1030300057697A61726420646F706F20617665727F
:103040002072696176766961746F206C6120737497
:10305000616D70616E74652E0050726F73696D20C2
:103060006E61686C65646E65746520646F206D6167
:103070006E75616C752061206F7072617674652069
:1030800070726F626C656D2E20506F207465206FBA
:10309000626E6F7674652057697A6172646120721E
:1030A00065626F6F746F76616E696D207469736BA2
:1030B00061726E792E00506C65617365206368657E
:1030C000636B206F75722068616E64626F6F6B2036
:1030D000616E6420666978207468652070726F6222
:1030E0006C656D2E205468656E20726573756D6514
:1030F000207468652057697A617264206279207251
:1031000065626F6F74696E6720746865207072699C
:103110006E7465722E0057697A617264002057617F
:10312000746368646F6720526573657400496E66E6
:103130006F726D6174696F6E00496E666F726D615A
:10314000636A65004D6F6E69746F72697A617200AF
:1031500053636865726D61746120696E666F0049C2
:103160006E666F726D61636500496E666F20736392
:103170007265656E0045727374652D53636869638B
:103180006874204B616C004B616C2E20312E2077CF
:103190006172737477790043616C2E207072696D6F
:1031A000657261206361702E0043616C2E20707225
:1031B000696D6F206C617965722E004B616C2E20F9
:1031C0007072766E692076727374767900466972D1
:1031D0007374206C617965722063616C2E00576195
:1031E0007274652061756620757365722E2E2E00CF
:1031F0004573706572616E646F206F7264656E6591
:103200007300417474656E64656E646F20757465D7
:103210006E7465005761697420666F7220757365FE
:10322000722E2E2E004265696D20447275636B20EC
:1032300062656E75747A746500557A79746520706C
:10324000727A79206472756B7500557361646F20B2
:10325000656E20696D70726573696F6E005573617C
:103260007469206E656C6C61207374616D706100AF
:10327000506F757A69746520626568656D20746940
:10328000736B75005573656420647572696E672091
:103290007072696E740046696C616D656E7420654C
:1032A0006E746C6164656E0057796A61632066694B
:1032B0006C616D656E7400536F6C74617220666929
:1032C0006C616D656E746F00536361726963612038
:1032D00066696C616D656E746F0056796A6D6F75A5
:1032E000742066696C616D656E7400556E6C6F61FB
:1032F000642066696C616D656E740046696C616D11
:10330000656E742061757377657266656E005779B6
:10331000737577616D2066696C616D656E740053BD
:103320006F6C74616E646F2066696C616D656E743C
:103330006F0052696C6173632E2066696C616D6504
:103340006E746F005679736F7576616D2066696C67
:10335000616D656E7400556E6C6F6164696E672097
:1033600066696C616D656E7400556E6B6E6F776E1D
:1033700020636F6D6D616E643A2022004665696E50
:1033800065696E7374656C6C756E67004E617374FD
:10339000726F696300416A75737461720052656788
:1033A0006F6C61004C616469740054756E65005304
:1033B00044204B61727465205B466C61736841699F
:1033C000725D006B617274612053445B466C73687C
:1033D0004169725D0053442063617264205B466CF6
:1033E00073684169725D005344204B6172746520BB
:1033F0005B6E6F726D616C5D006B61727461205306
:1034000044205B6E6F726D616C5D0053442063619C
:103410007264205B6E6F726D616C5D0054656D70DF
:103420002E204B616C2E205B4F4E5D004369657012
:103430006C2E206B616C2E205B4F4E5D0043616CE7
:103440002E2074656D702E205B4F4E5D0043616CC5
:103450002E2074656D702E205B4F4E5D005465709C
:103460006C2E206B616C2E205B4F4E5D0054656DA1
:10347000702E2063616C2E205B4F4E5D0054656D95
:10348000702E204B616C2E205B4F46465D004369D9
:1034900065706C2E206B616C2E205B4F46465D0084
:1034A00043616C2E2074656D702E205B4F46465D27
:1034B0000043616C2E2074656D702E205B4F464674
:1034C0005D005465706C2E206B616C2E205B4F4646
:1034D000465D0054656D702E2063616C2E205B4F3D
:1034E00046465D0054656D702E204B616C696272BA
:1034F000696572756E67206665727469672E204B08
:103500006C69636B656E20756D2077656974657293
:10351000207A7520676568656E2E00436965706C5A
:103520006E61206B616C69627261636A61207A61AD
:103530006B6F6E637A6F6E612E204B6F6E74796E57
:1035400075756A2070727A796369736B69656D004D
:1035500043616C69627261636F6E2074656D706542
:10356000726174757261207465726D696E616461F7
:103570002E2050726573696F6E6172207061726186
:1035800020636F6E74696E7561722E005461726192
:10359000747572612074656D7065726174757261A5
:1035A000207465726D696E6174612E20466172656A
:1035B00020636C69636B2070657220636F6E746941
:1035C0006E756172652E005465706C6F746E692043
:1035D0006B616C69627261636520646F6B6F6E63AF
:1035E000656E612E20506F6B726163756A74652021
:1035F000737469736B656D20746C616369746B615E
:103600002E0054656D70657261747572652063611A
:103610006C6962726174696F6E2069732066696E8D
:1036200069736865642E20436C69636B20746F2036
:10363000636F6E74696E75652E0054656D70204BF6
:10364000616C69622E202020202020202020004351
:103650006965706C2E206B616C2E2020202020204C
:103660002020200043616C2E2074656D702E202078
:1036700020202020202020200043616C2E20746513
:103680006D702E2020202020202020202000546536
:10369000706C2E206B616C2E20202020202020209A
:1036A00020200054656D702E2063616C2E20202038
:1036B000202020202020200054656D7065726174E8
:1036C00075720054656D7065726174757261005435
:1036D000656D70657261747572610054656D7065B9
:1036E000726174757261005465706C6F746100541E
:1036F000656D706572617475726500506F6D6F6392
:1037000000536F706F72746500506F64706F7261F8
:1037100000537570706F727400447275636B206132
:10372000626272656368656E005A6174727A796D5F
:103730006163206472756B00446574656E65722008
:10374000696D70726573696F6E0041727265737432
:1037500061207374616D7061005A61737461766980
:1037600074207469736B0053746F70207072696E8B
:103770007400474553544F5050542E20005041522E
:103780004144410041525245535441544F2E00533D
:10379000544F505045442E2000537465707261742C
:1037A0006520746F6F20686967683A20004973204C
:1037B000737465656C207368656574206F6E20682E
:1037C0006561746265643F00546F74616C65204488
:1037D0007275636B7A6569743A00437A617320632A
:1037E000616C6B6F77697479203A005469656D700C
:1037F0006F20746F74616C203A0054656D706F2097
:103800007374616D706120746F743A0043656C6B02
:103810006F767920636173203A00546F74616C2075
:103820007072696E742074696D65203A0047657323
:10383000616D7466696C616D656E743A0046696CA1
:10384000616D656E74206C61637A6E6965203A0003
:1038500046696C616D656E746F20746F74616C3A4B
:103860000046696C616D656E746F20746F743A0008
:1038700046696C616D656E742063656C6B656D2067
:103880003A00546F74616C2066696C616D656E748A
:10389000203A00447275636B7A6569743A2020009F
:1038A000437A6173206472756B75203A202000544E
:1038B00069656D706F20646520696D702E3A0054E3
:1038C000656D706F206469207374616D70613A007A
:1038D000436173207469736B75203A202000507225
:1038E000696E742074696D653A20200046696C61C8
:1038F0006D656E747665726272617563683A0046D2
:10390000696C616D656E74203A20200046696C61B7
:103910006D656E746F203A20200046696C616D659C
:103920006E746F20757361746F3A0046696C616DD7
:10393000656E74203A20200046696C616D656E7476
:1039400020757365643A2020005374617469737440
:10395000696B656E200053746174797374796B615F
:103960002020004573746164697374696361202069
:10397000005374617469737469636865005374619A
:1039800074697374696B6120200053746174697386
:10399000746963732020004572726F72202D20734A
:1039A0007461746963206D656D6F727920686173ED
:1039B000206265656E206F766572777269747465D2
:1039C0006E00476573636877696E6469676B6569E4
:1039D0007400507265646B6F73630056656C6F633F
:1039E000696461640056656C6F6369746100527943
:1039F00063686C6F73740053706565640020536F67
:103A0000667477617265205265736574004D6F64EA
:103A10006520202020205B6C656973655D004D6F1B
:103A200064202020202020205B63696368795D008A
:103A30004D6F646F2020205B73696C656E63696FE6
:103A40005D004D6F646F205B73696C656E7A696FA2
:103A5000736F5D004D6F64202020202020205B7458
:103A6000696368795D004D6F646520202020205BCC
:103A700073696C656E745D004D6F6465205B486FA3
:103A80006865204C656973745D004D6F64205B77D9
:103A900020777964616A6E6F73635D004D6F646F48
:103AA000205B72656E642E706C656E6F5D004D6F8D
:103AB00064652020202020205B666F7274655D00A5
:103AC0004D6F6420205B7679732E2076796B6F6E54
:103AD0005D004D6F6465205B6869676820706F7773
:103AE00065725D00456E64736368616C7465722015
:103AF000537461742E00506F6B617A206B72616E2B
:103B0000636F776B6900456E73656E6120746F70CB
:103B1000652066696E616C00537461746F2066691C
:103B20006E65636F7273610053746176206B6F6EA4
:103B3000632E207370696E2E0053686F7720656E58
:103B4000642073746F70730054656D702E20656906
:103B50006E7365747A656E0055737461776963205E
:103B600074656D706572617475726500457374611A
:103B7000626C656365722074656D702E3A00496DE4
:103B8000706F7374612074656D70657261747572A5
:103B900061004E61737461767465207465706C6F3A
:103BA00074753A005365742074656D706572617444
:103BB0007572653A0045696E7374656C6C756E67F5
:103BC000656E00557374617769656E696100436F56
:103BD0006E66696775726163696F6E00496D706FBB
:103BE0007374617A696F6E69004E61737461766592
:103BF0006E690053657474696E677300566572640C
:103C000072616874756E676665686C657200426C97
:103C1000616420706F6C61637A656E6961004572E2
:103C2000726F7220646520636F6E6578696F6E00D5
:103C30004572726F7265206361626C616767696F5C
:103C4000004368796261207A61706F6A656E69000D
:103C5000576972696E67206572726F720053656C86
:103C6000627374746573742073746172742000419C
:103C700075746F746573742073616C69646100415D
:103C800076766961206175746F746573740053652D
:103C90006C662074657374207374617274202000E4
:103CA0004269747465207072756566653A00536B7D
:103CB0006F6E74726F6C756A203A00436F6E747227
:103CC0006F6C61203A00566572696669636172655E
:103CD0003A005A6B6F6E74726F6C756A7465203A35
:103CE00000506C6561736520636865636B203A0002
:103CF00053656C62737474657374204F4B00417527
:103D0000746F74657374204F4B0053656C66207438
:103D1000657374204F4B004E6963687420616E6751
:103D2000657363686C6F7373656E004E69652070B0
:103D30006F646C61637A6F6E6F202020004E6F207D
:103D400068617920636F6E6578696F6E2020004E20
:103D50006F6E20636F6E6E6573736F004E657A6170
:103D6000706F6A656E6F20202020004E6F74206394
:103D70006F6E6E65637465640053696C6E696B0089
:103D80004D6F746F7265004D6F746F720043616C9C
:103D9000656E742E2F5465726D6973746F72005264
:103DA000697363616C642E2F5465726D6973742E30
:103DB000004865617465722F546865726D6973742B
:103DC0006F72004C75656674657274657374005427
:103DD0006573742077656E74796C61746F726100BD
:103DE000546573742064656C2076656E74696C61CB
:103DF000646F720050726F76612064656C20766526
:103E00006E74696C61746F720054657374207665AA
:103E10006E74696C61746F72750046616E207465B2
:103E200073740053656C62737474657374206D6988
:103E300073736C756E672E0053656C66746573746E
:103E4000206E69657564616E79004175746F746583
:103E500073742066616C6C61646F004175746F747B
:103E60006573742066616C6C69746F0053656C6671
:103E7000746573742073656C68616C2020005365F1
:103E80006C6674657374206661696C6564202000DB
:103E90004C696E6B6572204C7565667465723F0087
:103EA0004C6577792077656E74206E612064797334
:103EB0007A653F0056656E742E20656E206C612019
:103EC000697A673F0056656E742053582073756C8D
:103ED0006C277567656C6C6F3F004C657679207652
:103EE000656E74206E61207472797363653F004C57
:103EF00065667420686F74656E642066616E3F004D
:103F000053656C6274657374204665686C657221D4
:103F1000004175746F74657374206572726F7221DD
:103F2000004175746F74657374206E6567617469A0
:103F3000766F0053656C6674657374206572726F7A
:103F400072202100456E6465206E69636874206785
:103F50006574726F662E00546F70652066696E2EF0
:103F6000206E6F20746F632E0046696E65632E208D
:103F700066756F726920706F722E00456E6473747F
:103F80006F70206E6F742068697400456E6473638F
:103F900068616C74657200546F7065732066696E39
:103FA000616C0046696E65636F7273612028322907
:103FB00000456E6473746F707300546F7065206693
:103FC000696E616C0046696E65636F72736100456E
:103FD0006E6473746F7000566F72646572657220E0
:103FE0004C7565667465723F0050727A6F646E69D5
:103FF0002077656E742E206472756B753F00566570
:104000006E742E20616C206672656E74653F00567A
:10401000656E74206469207374616D706120616ED7
:10402000742E3F00507265646E69207469736B6F03
:1040300076792076656E743F0046726F6E742070DC
:1040400072696E742066616E3F00507275656665B8
:10405000205A20416368736520202020004B6F6E3A
:1040600074726F6C61205A2061786973202000435C
:104070006F6E74726F6C2064656C20656A65205A7F
:104080000056657269666963612061737365205AC1
:10409000004B6F6E74726F6C61205A206178697387
:1040A000202000436865636B696E67205A20617841
:1040B0006973202000507275656665205920416340
:1040C00068736520202020004B6F6E74726F6C61E6
:1040D00020592061786973202000436F6E74726FDD
:1040E0006C2064656C20656A6520590056657269AC
:1040F0006669636120617373652059004B6F6E744C
:10410000726F6C61205920617869732020004368C8
:1041100065636B696E6720592061786973202000A0
:10412000507275656665205820416368736520206C
:104130002020004B6F6E74726F6C61205820617884
:104140006973202000436F6E74726F6C2064656C1D
:1041500020656A652058005665726966696361204A
:10416000617373652058004B6F6E74726F6C6120C1
:10417000582061786973202000436865636B696E1D
:104180006720582061786973202000507275656639
:104190006520486F74656E64004B6F6E74726F6C4F
:1041A0006120686F74656E64202000436F6E7472C6
:1041B0006F6C20686F74656E642000566572696666
:1041C000696361207567656C6C6F004B6F6E74720C
:1041D0006F6C6120686F74656E64202000436865B1
:1041E000636B696E6720686F74656E642020005091
:1041F000727565666520456E64736368616C74658D
:10420000722020004B6F6E74726F6C6120656E645B
:1042100073746F707300436F6E742E20746F7065CB
:10422000732066696E616C005665726966696361C8
:104230002066696E65636F727361004B6F6E747296
:104240006F6C6120656E6473746F70730043686592
:10425000636B696E6720656E6473746F7073005072
:1042600072FE204265642020202020202020004B68
:104270006F6E74726F6C6120626564202020202054
:1042800000436F6E74726F6C2064652063616D61B2
:10429000005665726966696361206C6574746F00AD
:1042A0004B6F6E74726F6C612062656420202020F9
:1042B0002000436865636B696E6720626564202037
:1042C00020202000416C6C657320726963687469FA
:1042D00067202020200057737A7973746B6F204F0A
:1042E0004B20202020202000546F646F20626965DD
:1042F00020004E657373756E206572726F72650073
:10430000567365204F4B2020202020202020202085
:104310002000416C6C20636F7272656374202020F2
:104320002020200043616D612F43616C656E7461D4
:10433000646F72004C6574746F2F52697363616CA3
:10434000642E00426564202F204865617465720008
:1043500041786973206C656E677468004178697391
:104360000057726974696E6720746F2066696C65A6
:104370003A2000766F6C756D652E696E69742066E3
:1043800061696C6564002053697A653A2000534482
:1043900020656E746665726E7420004B6172746184
:1043A0002077796A657461005461726A657461206E
:1043B00072657469726164610053442072696D6F43
:1043C000737361004B617274612076796A6D7574E4
:1043D0006100436172642072656D6F76656400539D
:1043E00044207072696E74696E672062797465200A
:1043F000006F70656E206661696C65642C2046698B
:104400006C653A20006F70656E526F6F7420666144
:10441000696C65640053442065696E6765736574F3
:104420007A74004B6172746120776C6F7A6F6E6181
:10443000005461726A65746120696E73657274619B
:10444000646100534420696E736572697461004B46
:104450006172746120766C6F7A656E61004361727F
:104460006420696E73657274656400534420696EDC
:104470006974206661696C0046696C652073656CBF
:1044800065637465640046696C65206F70656E6570
:10449000643A20006572726F722077726974696E77
:1044A0006720746F2066696C6500534420636172F5
:1044B00064206F6B0043616E6E6F7420656E74656F
:1044C00072207375626469723A2000447275636B7E
:1044D00020776569746572676568656E00577A6EE6
:1044E000617769616E6965206472756B75005265EC
:1044F000616E7564617220696D70726573696F6E4B
:10450000005374616D706120696E2072697072650C
:104510007361004F626E6F766F76616E69207469A9
:10452000736B7500526573756D696E672070726983
:104530006E7400447275636B20666F727467657386
:1045400065747A7400577A6E6F7769656E69652055
:104550006472756B7500526573756D69656E646F15
:1045600020696D70726573696F6E00526970726553
:104570006E6469207374616D7061004F626E6F7656
:10458000656E69207469736B7500526573756D692A
:104590006E67207072696E7400466F727473657412
:1045A0007A656E004B6F6E74796E756F776163001C
:1045B0005265616E7564617220696D707265732EEB
:1045C0000052697072656E6469207374616D706108
:1045D00000506F6B7261636F766174005265737522
:1045E0006D65207072696E7400526573656E643A11
:1045F0002000506C656173652072656D6F76652073
:10460000737465656C2073686565742066726F6D80
:1046100020686561746265642E00426C61636B6F33
:104620007574206F636375727265642E20526563C2
:104630006F766572207072696E743F005265636FA9
:10464000766572696E67207072696E742020202012
:1046500000686F77746F2E707275736133642E63A8
:104660007A00686F77746F2E707275736133642E81
:10467000637A00686F77746F2E707275736133643C
:104680002E636F6D00666F72756D2E70727573613B
:1046900033642E637A00666F72756D2E7072757357
:1046A0006133642E637A00666F72756D2E70727559
:1046B000736133642E636F6D007072757361336460
:1046C0002E637A00707275736133642E637A0070A2
:1046D0007275736133642E636F6D00447275636B22
:1046E000207061757369657274004472756B207A0D
:1046F0006174727A796D616E7900496D707265735B
:10470000696F6E20656E207061757361005374610E
:104710006D706120696E20706175736100546973FA
:104720006B20706F7A6173746176656E0050726988
:104730006E742070617573656400447275636B20DC
:104740006162676562726F6368656E004472756B63
:104750002070727A657277616E7900496D7072654A
:1047600073696F6E2063616E63656C616461005391
:1047700074616D70612061626F727469746100545C
:1047800069736B20707265727573656E0050726923
:104790006E742061626F72746564005072696E7429
:1047A000657220646973636F6E6E6563746564001F
:1047B000756E64204B6E6F70662064727565636BF6
:1047C000656E004E616369736E696A2070727A79F2
:1047D0006369736B0050756C73617220656C206D3A
:1047E000616E646F006520636C696363617265204C
:1047F0006D616E6F706F6C61006120737469736BB3
:104800006E65746520746C616369746B6F00616EB2
:104810006420707265737320746865206B6E6F62BC
:1048200000447565736520566F72776165726D65BA
:104830006E004E6167727A656A206479737A6521C9
:104840000050726563616C656E7461722065787486
:104850007275736F72005072657269732E2075677E
:10486000656C6C6F210050726564656872656A746E
:104870006520747279736B7521005072656865618B
:104880007420746865206E6F7A7A6C652100566FAB
:1048900072776165726D656E0047727A616E6965E7
:1048A0000050726563616C656E7461720050726570
:1048B00072697363616C64610050726564656872EB
:1048C0006576005072656865617400506F77657237
:1048D00055700042697474652077617274656E006A
:1048E00050726F737A6520637A656B616300506FF5
:1048F00072204661766F7220457370657261720036
:10490000417370657474610050726F73696D2063D8
:10491000656B656A746500506C65617365207761CD
:104920006974004269747465206C6164656E20531B
:104930006965207A756572737420504C4120466910
:104940006C616D656E742E0050726F737A652C20E9
:104950006E616A7069657277207A616C6164756AEC
:104960002066696C616D656E7420504C412E004369
:104970006172676120656C2066696C616D656E743B
:104980006F20504C41207072696D65726F20706F9E
:1049900072206661766F722E0050657220666176B5
:1049A0006F7265207072696D612063617269636105
:1049B00072652066696C616D656E746F2064692034
:1049C000504C412E004E656A6472697665207A61AA
:1049D000766564746520504C412066696C616D6534
:1049E0006E742070726F73696D2E00506C65617308
:1049F00065206C6F616420504C412066696C616D6C
:104A0000656E742066697273742E00497374205049
:104A10004C412046696C616D656E742067656C6100
:104A200064656E3F004669616C6D656E7420504C24
:104A300041206A657374207A616C61646F77616E7E
:104A4000793F004573746120656C2066696C616D07
:104A5000656E746F20504C41206361726761646FB2
:104A60003F00496C20504C41206520737461746F85
:104A700020636172696361746F3F004A6520504C26
:104A8000412066696C616D656E74207A617665643B
:104A9000656E3F00497320504C412066696C616D22
:104AA000656E74206C6F616465643F002020506CFB
:104AB000616E6E6572427566666572427974657381
:104AC0003A2000506C6561736520706C61636520ED
:104AD000737465656C207368656574206F6E2068FB
:104AE0006561746265642E0050494E4441206572D0
:104AF000776165726D656E0047727A616E696520D7
:104B000050494E44410043616C656E74616E646F40
:104B10002050494E44410052697363616C642E20F9
:104B200050494E4441004E6168726976616E692059
:104B300050494E44410050494E44412048656174FB
:104B4000696E670054656D70657261747572207767
:104B500075726465206E69636874206B616C69624C
:104B6000726965727400436965706C6E61206B6177
:104B70006C69627261636A61206E69652062796C3A
:104B8000612070727A6570726F7761647A6F6E619E
:104B9000004C612074656D7065726174757261207E
:104BA00064652063616C6962726163696F6E206E17
:104BB0006F206861207369646F20616A7573746126
:104BC00064610054617261747572612064656C6C1B
:104BD000612074656D7065726174757261206E6FAD
:104BE0006E20616E636F72612065736567756974AD
:104BF00061005469736B61726E61206E6562796CDD
:104C000061207465706C6F746E65207A6B616C697D
:104C100062726F76616E610054656D706572617469
:104C20007572652063616C6962726174696F6E2070
:104C3000686173206E6F74206265656E2072756E98
:104C40002079657400504944204B616C69622E00E4
:104C50004B616C2E205049440043616C2E2050491A
:104C60004420202020202020202020200043616C90
:104C70002E2050494400504944206B616C2E202066
:104C80002020202020202020200050494420636143
:104C90006C2E202020202020202020202000504981
:104CA00044204B616C69622E2066657274696700EE
:104CB0004B616C2E20504944207A616B6F6E637A91
:104CC0006F6E610043616C2E205049442074657200
:104CD0006D696E6164610043616C2E20504944200F
:104CE000636F6D706C65746100504944206B616C3A
:104CF0002E20756B6F6E63656E61005049442063B2
:104D0000616C2E2066696E69736865640050494461
:104D1000204B616C696272696572756E67004B61E8
:104D20006C69627261636A61205049440043616C3E
:104D30006962726163696F6E205049440043616C1F
:104D4000696272617A696F6E65205049440050490A
:104D500044206B616C696272616365005049442054
:104D600063616C6962726174696F6E00447275632D
:104D70006B20756E74657262726563682E00507286
:104D80007A6572776163206472756B005061757328
:104D9000617220696D70726573696F6E004D657424
:104DA000746920696E20706175736100506F7A615B
:104DB000737461766974207469736B0050617573E4
:104DC00065207072696E74004C6567656E20656958
:104DD0006E20426C61747420506170696572207538
:104DE0006E7465722064696520447565736520770B
:104DF00061656872656E6420646572204B616C69E0
:104E00006272696572756E6720646572206572737F
:104E100074656E20342050756E6B74652E20576556
:104E20006E6E2064696520447565736520646173E6
:104E3000205061706965722065696E6B6C656D6D7F
:104E4000742C20447275636B657220736F666F7289
:104E50007420617573736368616C74656E00556D61
:104E600069657363206B6172746B65207061706932
:104E7000657275206E6120706F646B6C6164636530
:104E800020692074727A796D616A20706F64206481
:104E900079737A6120706F64637A617320706F6DCB
:104EA00069617275207069657277737A79636820B9
:104EB000342070756E6B746F772E204A65736C6941
:104EC000206479737A61207A616861637A79206FEE
:104ED000207061706965722C2077796C61637A202B
:104EE0006472756B61726B652E00436F6C6F6361EA
:104EF0007220756E6120686F6A6120646520706140
:104F000070656C20736F627265206C6120737570C0
:104F10006572666963696520646520696D70726594
:104F200073696F6E20647572616E7465206C6120A8
:104F300063616C6962726163696F6E206465206C85
:104F40006F73207072696D65726F73203420707595
:104F50006E746F732E205369206C6120626F7175BF
:104F6000696C6C61206D7565766520656C2070617B
:104F700070656C2C2061706167617220696D707260
:104F800065736F726120696E6D6564696174616DCE
:104F9000656E74652E00506F72726520756E2066A6
:104FA0006F676C696F20736F74746F206C277567FF
:104FB000656C6C6F20647572616E7465206C612025
:104FC00063616C696272617A696F6E65206465699C
:104FD000207072696D6920342070756E74692E209E
:104FE000496E206361736F206C277567656C6C6F09
:104FF000206D756F766120696C20666F676C696FD4
:1050000020737065676E6572652070726F6E746173
:105010006D656E7465206C61207374616D70616E76
:1050200074652E00556D697374657465206C6973C1
:105030007420706170697275206E6120706F646C8D
:105040006F7A6B752061207564727A756A74652059
:105050006A656A20706F6420747279736B6F752053
:10506000626568656D206D6572656E692070727627
:105070006E696368203420626F64752E20506F6BF8
:10508000756420747279736B61207A6163687974D6
:10509000692070617069722C207679706E65746514
:1050A000207469736B61726E752E00506C6163655C
:1050B0002061207368656574206F6620706170657B
:1050C0007220756E64657220746865206E6F7A7ADE
:1050D0006C6520647572696E672074686520636111
:1050E0006C6962726174696F6E206F6620666972A6
:1050F0007374203420706F696E74732E204966209B
:10510000746865206E6F7A7A6C6520636174636879
:105110006573207468652070617065722C20706FF3
:10512000776572206F666620746865207072696E9C
:1051300074657220696D6D6564696174656C792E42
:10514000006F6B004F6666004B65696E65204265B7
:10515000776567756E672E0053696E206D6F76698F
:105160006D69656E746F004E657373756E206D6F3B
:1051700076696D656E746F2E004E6F206D6F76656B
:105180002E004B65696E65205344204B6172746537
:10519000004272616B206B61727479205344004E3F
:1051A0006F20686179207461726A6574612053446C
:1051B000004E657373756E61205344005A61646ECE
:1051C00061205344206B61727461004E6F20534420
:1051D0002063617264004475657365004479737A75
:1051E0006100426F7175696C6C61005567656C6C2C
:1051F0006F00547279736B61004E6F7A7A6C650040
:1052000046696C2E206E696368742067656C616402
:10521000656E004272616B2066696C616D656E74CB
:10522000750046696C2E206E6F20696E74726F6413
:10523000756369646F0046696C2E206E6F6E206323
:105240006172696361746F0046696C616D656E744B
:10525000206E657A61766564656E0046696C616D85
:10526000656E74206E6F74206C6F616465640046B7
:105270006172626520756E6B6C6172004B6F6C6F52
:1052800072207A616E6965637A79737A2E00436F52
:105290006C6F72206E6F20686F6D6F67656E656FE3
:1052A00000436F6C6F7265206E6F6E207075726F49
:1052B000004261727661206E656E69206369737465
:1052C0006100436F6C6F72206E6F7420636C656158
:1052D00072004E65696E004E6965004E65004E6F46
:1052E00000426974746520616B7475616C697369DF
:1052F0006572656E2E0050726F737A65207A616BED
:105300007475616C697A6F7761630041637475616C
:105310006C697A617220706F72206661766F7200BC
:10532000507265676120616767696F726E612E00F8
:1053300050726F73696D20616B7475616C697A75F9
:105340006A74652E00506C656173652075706772B4
:105350006164652E004E657565204669726D7761E2
:1053600072652056657273696F6E20766572667518
:1053700065676261723A005779737A6C61206E6F6B
:10538000776120776572736A61206669726D7761F3
:1053900072653A004E7565766F206669726D776149
:1053A000726520646973706F6E69626C653A004E55
:1053B000756F76612076657273696F6E65206465BE
:1053C0006C206669726D7761726520646973706FB5
:1053D0006E6962696C65005679736C61206E6F76D8
:1053E00061207665727A65206669726D7761726593
:1053F0003A004E6577206669726D77617265207636
:10540000657273696F6E20617661696C61626C654B
:105410003A00426577656765205A0050727A657375
:10542000756E6163205A004D6F766572205A004D8B
:10543000756F7669205A00506F73756E6F757420A2
:105440005A004D6F7665205A004265776567652082
:10545000590050727A6573756E61632059004D6F03
:105460007665722059004D756F7669205900506F2E
:1054700073756E6F75742059004D6F7665205900F5
:1054800042657765676520580050727A6573756E5E
:1054900061632058004D6F7665722058004D756F1E
:1054A0007669205800506F73756E6F7574205800C0
:1054B0004D6F766520580045787472756972004D9D
:1054C000756F7669204573747275736F72650045E8
:1054D000787472756465720041636873626577659C
:1054E00067756E670052756368206F7369004D6F52
:1054F00076657220656A6573004D756F7669206107
:1055000073736500506F73756E6F7574206F73756C
:10551000004D6F76652061786973004D6573682072
:105520006C6976656C2E206C6574746F004D6573C4
:105530006820426564204C6576656C696E67004B37
:10554000616C696272696572756E67004B616C6946
:10555000627261636A610043616C6962726163696E
:105560006F6E0043616C696272617A696F6E65008B
:105570004B616C6962726163650043616C69627260
:105580006174696F6E0020766F6E203900207A207A
:105590003900206465203900207375203900207A95
:1055A000203900206F662039004D657373656E20C9
:1055B000646572205265666572656E7A686F6568AB
:1055C0006520646573204B616C69627269657270F5
:1055D000756E6B746573004F6B7265736C616D20D3
:1055E0007779736F6B6F7363206F646E696573692E
:1055F000656E69612070756E6B7475206B616C6986
:1056000062726163796A6E65676F004D6564697285
:10561000206C6120616C747572612064656C20700F
:10562000756E746F206465206C612063616C6962C3
:10563000726163696F6E004D697375726172652086
:105640006C27616C74657A7A61206469207269667E
:105650006572696D656E746F2064656C2070756E1F
:10566000746F2064692063616C696272617A696F2A
:105670006E65004D6572696D207265666572656E56
:10568000636E69207679736B75206B616C696272E9
:1056900061636E69686F20626F6475004D65617348
:1056A0007572696E67207265666572656E636520E6
:1056B000686569676874206F662063616C696272EF
:1056C0006174696F6E20706F696E740048617570E7
:1056D000746D656E7565004D656E7520676C6F77CE
:1056E0006E65004D656E75207072696E63697061DC
:1056F0006C004D656E75207072696E636970616CC7
:105700006500486C61766E69206E616269646B61E8
:10571000004D61696E004D32323120496E76616C08
:10572000696420657874727564657220004D323149
:105730003820496E76616C6964206578747275648E
:10574000657220004D32303020496E76616C69649C
:1057500020657874727564657220005265706F728E
:1057600074696E6720656E6473746F702073746102
:10577000747573004D3131372045727374652D5344
:10578000636869636874204B616C2E004D3131375A
:10579000204B616C2E20312E2077617273747779E3
:1057A000004D3131372043616C2E207072696D6578
:1057B0007261206361702E004D3131372043616C7E
:1057C0002E207072696D6F206C617965722E004DAC
:1057D000313137204B616C2E207072766E692076E5
:1057E0007273747679004D31313720466972737463
:1057F000206C617965722063616C2E004649524DC0
:10580000574152455F4E414D453A4D61726C696E4C
:105810002056312E302E323B20537072696E7465E3
:10582000722F6772626C206D617368757020666F8D
:10583000722067656E36204649524D574152455F8A
:1058400055524C3A68747470733A2F2F67697468B4
:1058500075622E636F6D2F707275736133642F5094
:10586000727573612D69332D506C75732F205052F2
:105870004F544F434F4C5F56455253494F4E3A3168
:105880002E30204D414348494E455F545950453ACA
:105890005072757361206933204D4B332045585445
:1058A00052554445525F434F554E543A3120555559
:1058B00049443A30303030303030302D30303030B4
:1058C0002D303030302D303030302D3030303030E1
:1058D000303030303030300A004D31303920496EB0
:1058E00076616C69642065787472756465722000F5
:1058F0004D31303520496E76616C6964206578746D
:10590000727564657220004D31303420496E7661C5
:105910006C696420657874727564657220004C6FE0
:105920007365205269656D656E736368656962654C
:10593000004B6F6C6F207061736F776500506F6CF8
:105940006561207375656C74610050756C6567677F
:105950006961206C656E74610055766F6C6E656E62
:10596000612072656D656E69636B61004C6F6F736A
:10597000652070756C6C65790046696C616D656E4B
:1059800074206C6164656E005770726F7761647A21
:105990002066696C616D656E7400496E74726F6427
:1059A000756369722066696C616D2E00436172696E
:1059B00063612066696C616D656E746F005A617613
:1059C0006573742066696C616D656E74004C6F61FF
:1059D000642066696C616D656E740046696C616D0A
:1059E000656E74206C65616474005770726F772EF9
:1059F0002066696C616D656E747500496E74726FB6
:105A000064756369656E646F2066696C616D2E00F4
:105A10004361726963616E646F2066696C616D2EAB
:105A2000005A61766164656E692066696C616D65B6
:105A30006E7475004C6F6164696E672066696C6195
:105A40006D656E74004C616465204661726265002C
:105A5000437A79737A637A2E206B6F6C6F7275005C
:105A600043616D6269616E646F20636F6C6F720079
:105A70004361726963616E646F20636F6C6F7265FE
:105A80000043697374656E69206261727679004CB7
:105A90006F6164696E6720636F6C6F720057616538
:105AA000686C652053707261636865005779626F36
:105AB00072206A657A796B610043616D6269616524
:105AC00020656C206964696F6D610053656C657A4F
:105AD000696F6E61206C696E6775610056796265E9
:105AE00072206A617A796B610053656C656374201A
:105AF0006C616E6775616765004465757473636892
:105B000000506F6C736B6900457370616E6F6C0051
:105B10004974616C69616E6F0043657374696E618D
:105B200000456E676C697368004142474542524FB9
:105B30004348454E2E2000504152414441204445A7
:105B400020454D455247454E43494100494E20545A
:105B5000494C542E004B494C4C45442E2000496E74
:105B600076616C696420657874727564657200464C
:105B7000696C616D656E742065696E6C6567656ED4
:105B8000005770726F7761647A2066696C616D6529
:105B90006E7400496E74726F647563697220666911
:105BA0006C616D656E746F00496E736572697265C4
:105BB0002066696C616D656E746F00566C6F7A74E7
:105BC000652066696C616D656E7400496E736572FF
:105BD000742066696C616D656E74005072696E74D4
:105BE0002046414E3A20004E6F7A7A6C652046413D
:105BF0004E3A00457874727564657220696E666FFE
:105C00000020766F6E203400207A203400206465F6
:105C1000203400207375203400207A203400206F57
:105C200066203400566572626573736572756E67BF
:105C300020426564204B616C69627269657270759F
:105C40006E6B7400506F7072617769616D20707255
:105C50006563797A796A6E6F73632070756E6B74A1
:105C600075206B616C6962726163796A6E65676FDA
:105C7000004D656A6F72616E646F2063616D6120B3
:105C800070756E746F2064652063616C6962726107
:105C900063696F6E0050657266657A696F6E2E205B
:105CA000696C206C6574746F2070756E746F2064FD
:105CB000692063616C696272617A2E005A6C65704A
:105CC00073756A6920707265736E6F7374206B618F
:105CD0006C69627261636E69686F20626F647500DF
:105CE000496D70726F76696E6720626564206361CA
:105CF0006C6962726174696F6E20706F696E740096
:105D00004B616C69627269657265205A004B616C07
:105D1000696272756A65205A0043616C69627261DA
:105D20006E646F205A0043616C696272616E646FC9
:105D3000205A004B616C696272756A69205A00438F
:105D4000616C6962726174696E67205A004B616CA4
:105D5000696272696572756E67204F4B004B616CAA
:105D600069627261636A61204F4B0043616C6962D2
:105D7000726163696F6E204F4B0043616C696272A0
:105D8000617A696F6E65204F4B004B616C6962727E
:105D9000616365204F4B0043616C69627261746995
:105DA0006F6E20646F6E65004B616C69627269652D
:105DB00072656E205A004B616C696272756A205A76
:105DC0000043616C6962726172205A0043616C69C0
:105DD000627261205A004B616C6962726F76617405
:105DE000205A0043616C696272617465205A0041F7
:105DF0007566776165726D656E204F4B0047727AEC
:105E0000616E6965204F4B2E0043616C656E746155
:105E10006D69656E746F2066696E616C2E005269E3
:105E20007363616C642E20636F6D706C65746F00BA
:105E30005A6168726976616E69204F4B2E00486521
:105E40006174696E6720646F6E652E0041756677B8
:105E50006165726D656E0047727A616E69652E2E9E
:105E60002E0043616C656E74616E646F2E2E2E0081
:105E700052697363616C64616D656E746F2E2E2E52
:105E8000005A6168726976616E690048656174697B
:105E90006E670046696C2E2073656E736F722020EA
:105EA0005B6F6E5D0046696C2E2073656E736F725A
:105EB000205B6F66665D002046726565204D656DEE
:105EC0006F72793A200044657220447275636B6585
:105ED00072207775726465206E6F6368206E6963E7
:105EE0006874206B616C696272696572742E2042FD
:105EF0006974746520666F6C67656E2053696520F0
:105F000064656D2048616E64627563682C204B6126
:105F1000706974656C20466972737420737465705F
:105F2000732C2041627363686E6974742043616CE2
:105F30006962726174696F6E20666C6F772E0044BF
:105F400072756B61726B61206E6965207A6F737414
:105F5000616C61206A65737A637A6520736B616C2A
:105F60006962726F77616E612E2050726F737A650D
:105F7000206B6965726F7761632073696520696E54
:105F8000737472756B636A612C20726F7A647A69BC
:105F9000616C205A61637A796E616D792C20706F23
:105FA00064726F7A647A69616C2053656C6674659B
:105FB00073742E00496D707265736F7261206E6F1D
:105FC00020657374612063616C6962726164612031
:105FD000746F64617669612E20506F7220666176FD
:105FE0006F72207573617220656C206D616E7561D2
:105FF0006C2C20656C206361706974756C6F204631
:10600000697273742073746570732C2073656C658A
:106010006363696F6E2043616C6962726174696F5A
:106020006E20666C6F772E005374616D70616E74B4
:106030006520616E636F7261206E6F6E2063616CAC
:106040006962726174612E205369207072656761A4
:10605000206469207365677569726520696C206DBD
:10606000616E75616C652C2063617069746F6C6F13
:10607000205052494D492050415353492C207365BB
:106080007A696F6E652064656C6C612063616C6910
:106090006272617A696F6E652E005469736B61720A
:1060A0006E61206E6562796C61206A65737465202B
:1060B0007A6B616C6962726F76616E612E20506FCF
:1060C00073747570756A74652070726F73696D2072
:1060D000706F646C65206D616E75616C752C206BE2
:1060E000617069746F6C61205A6163696E616D657E
:1060F0002C206F6473746176656320506F737475C0
:1061000070206B616C6962726163652E0050726908
:106110006E74657220686173206E6F7420626565AD
:106120006E2063616C696272617465642079657464
:106130002E20506C6561736520666F6C6C6F7720E4
:10614000746865206D616E75616C2C206368617088
:106150007465722046697273742073746570732C51
:106160002073656374696F6E2043616C696272614C
:1061700074696F6E20666C6F772E00447572636869
:10618000666C7573730050727A65706C797700462F
:106190006C756A6F00466C7573736F00507275741E
:1061A0006F6B00466C6F77004265776567756E6749
:1061B000206265656E64656E004B6F6E637A656E16
:1061C0006965206472756B75005465726D2E206D63
:1061D0006F76696D69656E746F7300417272657375
:1061E000746F20696E20636F72736F00446F6B6F02
:1061F0006E636F76616E6920706F687962750046B4
:10620000696E697368696E67206D6F76656D656E1E
:1062100074730020766F6E203400207A20340020C2
:106220006465203400207375203400207A20340007
:10623000206F6620340053756368656E2042656484
:10624000204B616C69627269657270756E6B740067
:10625000537A756B616D2070756E6B7475206B6110
:106260006C6962726163796A6E65676F20706F64D2
:106270006B6C61646B690042757363616E646F205F
:1062800063616D612070756E746F20646520636159
:106290006C6962726163696F6E00526963657263F3
:1062A000612064656C206C6574746F2070756E7409
:1062B0006F2064692063616C696272617A2E0048A4
:1062C0006C6564616D206B616C69627261636E699B
:1062D00020626F6420706F646C6F7A6B7900536515
:1062E00061726368696E67206265642063616C69CE
:1062F00062726174696F6E20706F696E74004974A8
:10630000657261636A6120005265697465726163D8
:10631000696F6E2000526569746572617A696F6E8B
:106320006520004974657261636520004974657277
:106330006174696F6E2000446F6E652073617669C9
:106340006E672066696C652E00446F6E6520707202
:10635000696E74696E672066696C650049737420A4
:106360004661726265207265696E3F00437A7920EA
:106370006B6F6C6F72206A65737420637A797374C3
:10638000793F00457320656C206E7565766F2063DC
:106390006F6C6F72206E697469646F3F00496C2086
:1063A000636F6C6F7265206527206E697469646F16
:1063B0003F004A652062617276612063697374618F
:1063C0003F00497320636F6C6F7220636C6561726C
:1063D0003F0046696C616D656E742D576563687327
:1063E000656C0057796D69656E69632066696C61DB
:1063F0006D656E740043616D626961722066696CDF
:10640000616D656E746F0043616D622E2066696C0C
:10641000616D656E746F0056796D656E6974206686
:10642000696C616D656E74004368616E67652066B6
:10643000696C616D656E74004C7565667465722D6E
:1064400054656D706F00507265646B6F7363207775
:10645000656E742E0056656C6F63696461642056C6
:10646000656E742E0056656C6F6369746120766585
:106470006E742E00527963686C6F73742076656E4B
:10648000742E0046616E20737065656400656E71E0
:106490007565696E67202200456B7374727564655B
:1064A00072004578747275736F72004573747275FB
:1064B000736F72650045787472756465720020456B
:1064C000787465726E616C205265736574005072E9
:1064D000696E7465722073746F7070656420647582
:1064E0006520746F206572726F72732E2046697812
:1064F00020746865206572726F7220616E64207509
:106500007365204D39393920746F20726573746159
:1065100072742E202854656D706572617475726591
:106520002069732072657365742E20536574206929
:106530007420616674657220726573746172746927
:106540006E6729004E6F204C696E65204E756D6236
:106550006572207769746820636865636B73756D15
:106560002C204C617374204C696E653A20004E6F8C
:1065700020436865636B73756D2077697468206C60
:10658000696E65206E756D6265722C204C61737446
:10659000204C696E653A200020746F6F206C6F6E1E
:1065A0006720657874727573696F6E207072657696
:1065B000656E746564004C696E65204E756D62652C
:1065C00072206973206E6F74204C617374204C6963
:1065D0006E65204E756D6265722B312C204C617397
:1065E00074204C696E653A20005072696E74657251
:1065F0002068616C7465642E206B696C6C2829209E
:1066000063616C6C6564210020636F6C6420657845
:1066100074727573696F6E2070726576656E7465DD
:106620006400636865636B73756D206D69736D617C
:106630007463682C204C617374204C696E653A2039
:10664000004645484C45523A00424C41443A0045C8
:1066500052524F52453A0043485942413A0045523E
:10666000524F523A00456E642066696C65206C6931
:106670007374006F70656E00545249474745524528
:106680004400656E6473746F7073206869743A2097
:106690000045696E656E204D6F6D656E7420626990
:1066A0007474652E00456E206573706572610053C9
:1066B0006F7370656E73696F6E652E2E2E00536C4E
:1066C0006565702E2E2E004D6F746F72656E2061A1
:1066D00075730057796C61637A79632073696C6EA6
:1066E000696B6900417061676172206D6F746F72D0
:1066F0006573004469736162696C6974206D6F74BD
:106700006F7269005679706E6F7574206D6F746F5B
:1067100072790044697361626C652073746570708E
:1067200065727300416B7475656C6C6573005479A8
:106730006C6B6F20616B7475616C6E650041637486
:1067400075616C0041747475616C6500506F757A89
:106750006520616B7475616C6E690043757272655A
:106760006E74004372617368206465742E2020206B
:106770005B6F6E5D004372617368206465742E20E8
:10678000205B6F66665D0020436F756E7420583A1B
:1067900020005765636873656C206F6B3F00577905
:1067A0006D69616E61206F6B3F0043616D6269616D
:1067B000646F20636F72726563742E3F0043616D76
:1067C000626961746F20636F72722E3F0056796D3B
:1067D000656E61206F6B3F004368616E6765642082
:1067E000636F72726563746C793F0041626B7565AB
:1067F000686C656E00577963686C6F647A696300D2
:10680000456E6672696172005261666672656464A3
:1068100061005A63686C6164697400436F6F6C64F3
:106820006F776E00204C61737420557064617465DD
:10683000643A2000576165686C656E205369652075
:106840004578747275646572005779626965727A09
:1068500020656B7374727564657200456C65676959
:1068600072206578747275736F723A0053656C6547
:106870007A696F6E61206573747275736F72653AB1
:106880000056796265727465206578747275646506
:10689000723A0043686F6F7365206578747275642F
:1068A00065723A005765636873656C206572666F40
:1068B0006C67722E210057796D69616E61206F6B74
:1068C000210043616D62696F20636F72726563744A
:1068D0006F0043616D62696F2072697573636974DB
:1068E0006F21005A6D656E612075737065736E61FE
:1068F00021004368616E6765207375636365737318
:106900002100447275636B656E20766F6E20534470
:10691000004472756B207A205344004D656E7520DB
:106920007461726A657461205344005374616D70C0
:1069300061206461205344005469736B207A2053B2
:1069400044005072696E742066726F6D205344006B
:1069500054656D702E206B616C6962726965726539
:106960006E00436965706C6E61206B616C69627268
:106970002E0043616C6962726163696F6E20746599
:106980006D702E0054617261747572612074656D52
:10699000702E005465706C6F742E206B616C696290
:1069A000726163650054656D702E2063616C69626D
:1069B000726174696F6E0043616C696272617469BF
:1069C0006E67205A004B616C696272696572656E10
:1069D00000536B616C6962726F7761630043616C35
:1069E00069627261720043616C6962726172650012
:1069F0005A6B616C6962726F7661740043616C6995
:106A000062726174650052657365742058595A202A
:106A10004B616C6962722E005265736574206B6104
:106A20006C6962722E2058595A0052657365742041
:106A300058595A206B616C6962722E0052657365F9
:106A4000742058595A2063616C6962722E004B6140
:106A50006C696272696572756E672058595A004B8D
:106A6000616C69627261636A612058595A004361BE
:106A70006C696272612058595A0043616C69627294
:106A8000612058595A004B616C69627261636520DC
:106A900058595A0043616C69627261746520585993
:106AA0005A002042726F776E206F757420526573A2
:106AB000657400426567696E2066696C65206C6963
:106AC00073740058595A2D4B616C69627269657212
:106AD000756E6720756E67656E61752E204C696EE8
:106AE0006B657220766F726465726572204B616CA3
:106AF00069627269657270756E6B74206973742057
:106B00007A75207765697420766F726E652E004BFA
:106B1000616C69627261636A612058595A206E69BA
:106B200065646F6B6C61646E612E204C65777920B3
:106B300070727A65646E692070756E6B74207A620B
:106B4000797420777973756E6965747920646F2024
:106B500070727A6F64752E0043616C696272617A3B
:106B6000696F6E2058595A20636F6D70726F6D6532
:106B7000746964612E2050756E746F2064656C6159
:106B80006E7465726F20697A7175696572646F20C1
:106B90006E6F20616C63616E7A61626C652E00437A
:106BA000616C696272617A696F6E652058595A200A
:106BB000636F6D70726F6D657373612E2050756EAB
:106BC000746F20616E746572696F72652073696E8F
:106BD000697374726F206E6F6E207261676769757A
:106BE0006E676962696C652E004B616C69627261E7
:106BF00063652058595A206E65707265736E612EF8
:106C0000204C65767920707265646E6920626F64CD
:106C1000206D6F63207670726564752E0058595A26
:106C20002063616C6962726174696F6E20636F6D5D
:106C300070726F6D697365642E204C656674206692
:106C4000726F6E742063616C6962726174696F6ED9
:106C500020706F696E74206E6F7420726561636856
:106C600061626C652E0058595A2D4B616C696272D5
:106C7000696572756E6720756E67656E61752E2029
:106C8000566F7264657265204B616C6962726965EA
:106C90007270756E6B74652073696E64207A7520EE
:106CA0007765697420766F726E652E004B616C6932
:106CB00062722E2058595A206E6965646F6B6C6140
:106CC000646E612E2050727A65646E6965207075FD
:106CD0006E6B7479206B616C6962722E205A6279D6
:106CE00074207779732E20646F2070727A6F6475C8
:106CF0002E0043616C696272617A696F6E20585927
:106D00005A20636F6D70726F6D65746964612E20B7
:106D100050756E746F2064656C616E7465726F730C
:106D2000206E6F20616C63616E7A61626C65732E98
:106D30000043616C696272617A696F6E65205859AF
:106D40005A20636F6D70726F6D657373612E205082
:106D5000756E746920616E746572696F7269206EF8
:106D60006F6E207261676769756E676962696C69C9
:106D70002E004B616C6962726163652058595A201C
:106D80006E65707265736E612E20507265646E69F7
:106D9000206B616C69627261636E6920626F6479F5
:106DA000206D6F63207670726564752E0058595A95
:106DB0002063616C6962726174696F6E20636F6DCC
:106DC00070726F6D697365642E2046726F6E7420E9
:106DD00063616C6962726174696F6E20706F696E55
:106DE0007473206E6F7420726561636861626C6594
:106DF0002E0058595A204B616C6962726965727530
:106E00006E6720696E204F72646E756E672E205813
:106E10002F592041636873656E2073696E64206525
:106E200074776173207363686965662E004B616CCB
:106E300069627261636A612058595A207072617781
:106E400069646C6F77612E204F73696520582F59E4
:106E5000206C656B6B6F20736B6F736E652E2044B7
:106E60006F62726120726F626F7461210043616CA6
:106E70006962726163696F6E2058595A20636F723C
:106E800072656374612E204C6F7320656A65732090
:106E900058202F205920657374616E206C696765D6
:106EA00072616D656E746520696E636C696E616494
:106EB0006F732E204275656E2074726162616A6F15
:106EC000210043616C696272617A696F6E20585962
:106ED0005A20636F7272657474612E2041737369F6
:106EE00020582F59206C65676765726D656E7465F3
:106EF0002073746F7274692E2042656E206661740F
:106F0000746F21004B616C6962726163652058592E
:106F10005A207620706F7261646B752E20582F593D
:106F2000206F7379206D69726E65207A6B6F73655F
:106F30006E652E20446F62726120707261636521FC
:106F40000058595A2063616C6962726174696F6E8E
:106F500020616C6C2072696768742E20582F59204C
:106F6000617865732061726520736C696768746C01
:106F70007920736B657765642E20476F6F64206A94
:106F80006F62210058595A204B616C6962726965C1
:106F900072756E6720696E204F72646E756E672E13
:106FA00020536368696566686569742077697264EF
:106FB000206175746F6D617469736368206B6F72A3
:106FC000726967696572742E004B616C69627261E7
:106FD000636A612058595A207072617769646C6FD6
:106FE00077612E20536B6F73792062656461206135
:106FF00075746F6D617479637A6E696520777972E3
:107000006F776E616E652070727A79206472756B2D
:10701000752E0043616C6962726163696F6E2058FE
:10702000595A20636F7272656374612E204C61201F
:10703000696E636C696E6163696F6E20736520634E
:107040006F72726567697261206175746F6D6174CA
:107050006963616D656E74652E0043616C6962726F
:10706000617A696F6E2058595A20636F7272657425
:1070700074612E204C6120646973746F7273696F40
:107080006E6520766572726127206175746F6D611F
:10709000746963616D656E746520636F6D70656E94
:1070A000736174612E004B616C696272616365206B
:1070B00058595A207620706F7261646B752E205A71
:1070C0006B6F73656E692062756465206175746F9E
:1070D0006D617469636B79207679726F766E616E1B
:1070E0006F20707269207469736B752E0058595A3D
:1070F0002063616C6962726174696F6E20616C6C8F
:107100002072696768742E20536B65772077696CED
:107110006C20626520636F727265637465642061C0
:1071200075746F6D61746963616C6C792E00585968
:107130005A2D4B616C696272696572756E67206663
:1071400065686C67657363686C6167656E2E204265
:1071500065642D4B616C69627269657270756E6BE6
:1071600074206E6963687420676566756E64656E09
:107170002E004B616C6962722E2058595A206E693C
:10718000657564616E612E204B616C69627261632A
:10719000796A6E792070756E6B7420706F646B6C99
:1071A00061646B69206E69657A6E616C657A696F7E
:1071B0006E792E0043616C6962726163696F6E2043
:1071C00058595A2066616C6C6164612E2050756E4E
:1071D000746F732064652063616C696272616369B6
:1071E0006F6E20656E206C612063616D61206E6F33
:1071F00020656E636F6E747261646F732E004361FD
:107200006C696272617A696F6E652058595A20669E
:10721000616C6C6974612E20496C2070756E746F9E
:107220002064692063616C696272617A696F6E655E
:107230002073756C206C6574746F206E6F6E2065A2
:107240002720737461746F2074726F7661746F2E6F
:10725000004B616C6962726163652058595A2073F2
:10726000656C68616C612E204B616C696272616350
:107270006E6920626F6420706F646C6F7A6B792026
:107280006E656E616C657A656E2E0058595A206382
:10729000616C6962726174696F6E206661696C65A8
:1072A000642E204265642063616C69627261746956
:1072B0006F6E20706F696E7420776173206E6F74CB
:1072C00020666F756E642E0058595A2D4B616C699B
:1072D0006272696572756E67206F6B2E20582F5928
:1072E0002D41636873656E2073696E642073656EEB
:1072F0006B7265636874207A7565696E616E64652A
:10730000722E20476C7565636B77756E73636821A9
:10731000004B616C69627261636A612058595A203E
:107320006F6B2E204F73696520582F592073612091
:1073300070726F73746F7061646C652E2047726138
:1073400074756C61636A65210043616C6962726186
:1073500063696F6E2058595A206F6B2E20456A65FD
:107360007320582F592070657270656E646963755B
:107370006C617265732E2046656C69636974616324
:10738000696F6E6573210043616C696272617A692D
:107390006F6E652058595A204F4B2E20476C69203C
:1073A0006173736920582F5920736F6E6F20706559
:1073B0007270656E6469636F6C6172692E20436FD1
:1073C0006D706C696D656E746921004B616C6962EA
:1073D000726163652058595A207620706F7261641B
:1073E0006B752E20582F59206F7379206A736F7533
:1073F000206B6F6C6D652E2047726174756C756AB9
:1074000069210058595A2063616C6962726174691C
:107410006F6E206F6B2E20582F5920617865732076
:107420006172652070657270656E646963756C6108
:10743000722E20436F6E67726174756C6174696F30
:107440006E73210058595A2D4B616C6962726965DF
:1074500072756E67206665686C67657363686C61DA
:1074600067656E2E20426974746520736368617568
:10747000656E2053696520696E20646173204861E0
:107480006E64627563682E004B616C696272616341
:107490006A612058595A206E6965706F7769656412
:1074A0007A696F6E612E205370726177647A6963B6
:1074B000207720696E737472756B636A692E00435E
:1074C000616C6962726163696F6E2058595A2066F7
:1074D000616C6C6164612E20436F6E73756C7461B6
:1074E0007220656C206D616E75616C20706F72200A
:1074F0006661766F722E0043616C696272617A69AF
:107500006F6E652058595A2066616C6C6974612EE3
:1075100020536920707265676120646920636F6E13
:1075200073756C7461726520696C206D616E756134
:107530006C652E004B616C696272616365205859FD
:107540005A2073656C68616C612E204E61686C65B1
:10755000646E65746520646F206D616E75616C7515
:107560002E0058595A2063616C6962726174696FA8
:107570006E206661696C65642E20506C6561736570
:1075800020636F6E73756C7420746865206D616E16
:1075900075616C2E0058595A2D4B616C6962726985
:1075A0006572756E67206665686C67657363686C85
:1075B0006167656E2E204C696E6B657220766F7206
:1075C0006465726572204B616C6962726965727084
:1075D000756E6B7420697374207A75207765697491
:1075E00020766F726E652E004B616C6962722E2080
:1075F00058595A206E69657564616E612E204C651C
:1076000077792070727A65646E692070756E6B741C
:10761000207A62797420646F2070727A6F64752E9C
:10762000205779726F776E6163206472756B617237
:107630006B652E0043616C6962726163696F6E20D5
:1076400058595A2066616C6C61642E2050756E74B6
:107650006F2064656C616E7465726F20697A7175F4
:10766000696572646F206E6F20616C63616E7A6110
:10767000626C652E0043616C696272617A696F6E3B
:10768000652058595A2066616C6C6974612E2050CF
:10769000756E746F20616E746572696F72652073A8
:1076A000696E697374726F206E6F6E2072616767A6
:1076B00069756E676962696C652E004B616C696201
:1076C000726163652058595A2073656C68616C61FA
:1076D0002E204C65767920707265646E6920626F29
:1076E00064206D6F63207670726564752E2053720E
:1076F0006F766E656A7465207469736B61726E75FE
:107700002E0058595A2063616C6962726174696F06
:107710006E206661696C65642E204C656674206617
:10772000726F6E742063616C6962726174696F6EEE
:1077300020706F696E74206E6F742072656163686B
:1077400061626C652E0058595A2D4B616C696272EA
:10775000696572756E67206665686C6765736368D6
:107760006C6167656E2E20566F7264657265204B82
:10777000616C69627269657270756E6B7465207395
:10778000696E64207A75207765697420766F726EF1
:10779000652E004B616C6962722E2058595A206E1A
:1077A00069657564616E612E2050727A65642E2061
:1077B00070756E6B7479206B616C6962722E207AC1
:1077C00062797420646F2070727A6F64752E20570E
:1077D00079726F776E6163206472756B61726B652D
:1077E0002E0043616C6962726163696F6E20585943
:1077F0005A2066616C6C61642E2050756E746F2027
:1078000064656C616E7465726F73206E6F20616C5D
:1078100063616E7A61626C65732E0043616C6962AC
:1078200072617A696F6E652058595A2066616C6C76
:107830006974612E2050756E746920616E74657272
:10784000696F7269206E6F6E207261676769756E0D
:10785000676962696C692E004B616C696272616371
:10786000652058595A2073656C68616C612E2050F0
:107870007265646E69206B616C69627261636E69C6
:1078800020626F6479206D6F632076707265647515
:107890002E2053726F766E656A7465207469736BFF
:1078A00061726E752E0058595A2063616C6962725C
:1078B0006174696F6E206661696C65642E20467222
:1078C0006F6E742063616C6962726174696F6E209F
:1078D000706F696E7473206E6F7420726561636877
:1078E00061626C652E005A2D4B616C69627269652C
:1078F00072756E67206665686C67657363686C6730
:107900002E2053656E736F72206E696368742061F8
:107910006E67657363686C6F7373656E2E20576155
:10792000727465206175662052657365742E004B14
:10793000616C69627261636A61206E696575646118
:107940006E612E2053656E736F72206F646C61637D
:107950007A6F6E79206C75622075737A6B6F647ABA
:107960002E206B6162656C2E20437A656B616D2001
:107970006E612072657365742E004E6976656C6168
:1079800063696F6E2066616C6C6164612E20536563
:107990006E736F7220646573636F6E656374616488
:1079A0006F206F206361626C65732064616E616437
:1079B0006F732E204573706572616E646F207265FF
:1079C0007365742E004C6976656C6C616D656E74C0
:1079D0006F206C6574746F2066616C6C69746F2EB7
:1079E0002053656E736F726520646973636F6E2ECA
:1079F000206F204361766F2044616E6E2E20496EA9
:107A000020617474657361206469207265736574A4
:107A10002E004B616C696272616365205A20736548
:107A20006C68616C612E2053656E736F72206A659D
:107A3000206F64706F6A656E79206E65626F20706A
:107A40007265727573656E79206B6162656C2E204C
:107A500043656B616D206E612072657365742E00E5
:107A6000426564206C6576656C696E672066616945
:107A70006C65642E2053656E736F72206469736346
:107A80006F6E6E6563746564206F72206361626CF3
:107A9000652062726F6B656E2E2057616974696E26
:107AA0006720666F722072657365742E005A2D4BC5
:107AB000616C2E206665686C67657363686C672E01
:107AC0002053656E736F72206E69636874206175F0
:107AD0007367656C6F6573742E205363686D75747E
:107AE0007A6967652044756573653F2057617274D4
:107AF0006520617566205265736574004B616C6921
:107B0000627261636A61206E69657564616E612E7F
:107B10002053656E736F72206E696520646F746B9D
:107B20006E616C2E205A616E6965637A79737A2E64
:107B3000206479737A613F20437A656B616D206EB2
:107B4000612072657365742E004E6976656C6163A1
:107B5000696F6E2066616C6C6164612E2053656E86
:107B6000736F72206E6F2066756E63696F6E612E23
:107B7000204573636F6D62726F7320656E20426F74
:107B80007175692E3F204573706572616E646F2058
:107B900072657365742E004C6976656C6C616D65F9
:107BA0006E746F206C6574746F2066616C6C6974A0
:107BB0006F2E4E6F5269737053656E736F722052E1
:107BC000657369647569207375207567656C6C6F82
:107BD0003F20496E2061747465736120646920726E
:107BE000657365742E004B616C6962726163652018
:107BF0005A2073656C68616C612E2053656E736FDB
:107C000072206E657365706E756C2E205A6E65639A
:107C1000697374656E6120747279736B613F204380
:107C2000656B616D206E612072657365742E004214
:107C30006564206C6576656C696E67206661696C49
:107C400065642E2053656E736F72206469646E7470
:107C500020747269676765722E2044656272697369
:107C6000206F6E206E6F7A7A6C653F205761697461
:107C7000696E6720666F722072657365742E005A94
:107C80002D4B616C696272696572756E67206665FD
:107C9000686C67657363686C672E2053656E736FDD
:107CA00072207A7520686F63682061757367656CF0
:107CB0006F6573742E20576172746520617566203C
:107CC00052657365742E004B616C69627261636A00
:107CD00061205A206E69657564616E612E2053655E
:107CE0006E736F7220646F746B2E207A61207779C7
:107CF000736F6B6F2E20437A656B616D206E612010
:107D000072657365742E004E6976656C6163696F88
:107D10006E2066616C6C6164612E2053656E736FBA
:107D2000722066756E63696F6E612064656D617344
:107D30006961646F2074656D7072616E6F2E20458D
:107D400073706572616E646F2072657365742E0066
:107D50004C6976656C6C616D656E746F206C6574D2
:107D6000746F2066616C6C69746F2E526973702039
:107D700073656E736F72652074726F70706F2070B0
:107D8000726573746F496E206174746573612064E9
:107D9000692072657365742E004B616C6962726153
:107DA0006365205A2073656C68616C612E20536591
:107DB0006E736F72207365706E756C207072696C73
:107DC0006973207679736F6B6F2E2043656B616DDD
:107DD000206E612072657365742E00426564206CAC
:107DE0006576656C696E67206661696C65642E20D6
:107DF00053656E736F72207472696767657265642C
:107E000020746F6F20686967682E205761697469F4
:107E10006E6720666F722072657365742E0042650E
:107E20006420617566776165726D656E0047727A70
:107E3000616E69652073746F6C696B612E2E0043EF
:107E4000616C656E74616E646F204261736500528F
:107E5000697363616C642E206C6574746F005A6181
:107E600068726976616E69206265640042656420AB
:107E700048656174696E6700426564204F4B00532A
:107E8000746F6C696B204F4B2E00426173652070DC
:107E900072657061726164610050696174746F2011
:107EA000666174746F2E00426564204F4B2E004251
:107EB000656420646F6E650052656368747320208A
:107EC00020205B756D5D005720707261776F205BBD
:107ED000756D5D00446572656368612020205B7587
:107EE0006D5D00446573747261202020205B756DA8
:107EF0005D0056707261766F205B756D5D00526932
:107F000067687420736964655B756D5D00527565A3
:107F1000636B7365747A656E0052657365740048AF
:107F2000696E74656E202020205B756D5D00446F66
:107F30002074796C7520205B756D5D0041747261F1
:107F40007320202020205B756D5D00526574726F78
:107F500020202020205B756D5D00567A61647520BD
:107F6000205B756D5D0052656172207369646520E8
:107F70005B756D5D00426564206C6576656C204BB9
:107F80006F7272656B74004B6F72656B74612070F9
:107F90006F646B6C61646B6900436F72722E206456
:107FA00065206C612063616D6100436F7272657A58
:107FB0002E206C69762E6C6574746F004B6F726541
:107FC0006B636520706F646C6F7A6B7900426564D7
:107FD000206C6576656C20636F7272656374004C0B
:107FE000696E6B7320202020205B756D5D0057202B
:107FF0006C65776F20205B756D5D00497A717569DE
:1080000065726461205B756D5D0053696E697374A0
:10801000726120205B756D5D00566C65766F202067
:108020005B756D5D004C6566742073696465205BEB
:10803000756D5D00566F726E6520202020205B7587
:108040006D5D00446F2070727A6F6475205B756D92
:108050005D004164656C616E746520205B756D5DCB
:108060000046726F6E7465202020205B756D5D0088
:10807000567072656475205B756D5D0046726F6E3B
:108080007420736964655B756D5D0053746F6C6912
:108090006B0042617365004C6574746F00426564E7
:1080A000004465722041627374616E64207A77695E
:1080B000736368656E2064657220537069747A65B5
:1080C0002064657220447565736520756E64206454
:1080D00065722042656420697374206E6F63682046
:1080E0006E696368742065696E67657374656C6C2E
:1080F000742E20426974746520666F6C67656E200B
:108100005369652064656D2048616E6462756368BB
:108110002C2046697273742073746570732C2073FD
:10812000656374696F6E204669727374206C61793F
:1081300065722063616C6962726174696F6E2E0092
:108140004F646C65676C6F7363206479737A792010
:108150006F6420706F646B6C61646B69206E69651D
:10816000206A65737420736B616C6962726F7761EA
:108170006E612E20506F73746570756A207A676F18
:10818000646E6965207A20696E737472756B636AB8
:108190006120726F7A647A69616C205A61637A79BE
:1081A0006E616D792C20706F64726F7A647A696188
:1081B0006C204B616C69627261636A6120706965F1
:1081C0007277737A656A20776172737477792E009B
:1081D00044697374616E63696120656E74726520B1
:1081E0006C612070756E7461206465206C61206222
:1081F0006F7175696C6C612079206C61207375708A
:1082000065726669636965206465206C61206361DD
:108210006D61206E6F2066696A6164612061756EB0
:108220002E20506F72206661766F722073696761CD
:1082300020656C206D616E75616C2C2063617069C6
:1082400074756C6F204669727374207374657073F3
:108250002C2073656363696F6E20466972737420A6
:108260006C617965722063616C6962726174696FB7
:108270006E2E0044697374616E7A6120747261209D
:108280006C612070756E74612064656C6C27756715
:10829000656C6C6F2065206C61207375706572660B
:1082A000696369652064656C206C6574746F206E09
:1082B0006F6E20616E636F726120696D706F737491
:1082C000612E205369207072656761206469207394
:1082D00065677569726520696C206D616E75616C8A
:1082E000652C2063617069746F6C6F2046697273CE
:1082F000742073746570732C2073657A696F6E6572
:10830000204669727374206C617965722063616CB8
:108310006962726174696F6E2E004E656E69207AB3
:108320006B616C6962726F76616E6120767A6461EE
:108330006C656E6F737420747279736B79206F64DF
:10834000207469736B6F766520706F646C6F7A6BE5
:10835000792E20506F73747570756A746520707211
:108360006F73696D20706F646C65206D616E7561EF
:108370006C752C206B617069746F6C61205A61633D
:10838000696E616D652C206F64737461766563201E
:108390004E6173746176656E69207072766E6920C5
:1083A0007672737476792E0044697374616E6365B6
:1083B000206265747765656E20746970206F662031
:1083C000746865206E6F7A7A6C6520616E642074C3
:1083D00068652062656420737572666163652068F4
:1083E0006173206E6F74206265656E207365742002
:1083F0007965742E20506C6561736520666F6C6CB6
:108400006F7720746865206D616E75616C2C2063D8
:108410006861707465722046697273742073746544
:1084200070732C2073656374696F6E204669727374
:1084300074206C617965722063616C696272617429
:10844000696F6E2E005A2065696E7374656C6C6579
:108450006E00446F7374726F6A656E6965206F7326
:1084600079205A004D6963726F7061736F20456A9D
:1084700065205A00436F6D70656E73617A696F6E27
:1084800065205A00446F6C6164656E69206F737972
:10849000205A004C6976652061646A757374205AAD
:1084A0000041646A757374696E67205A0053746181
:1084B0007274706F736974696F6E004C6C6576616D
:1084C0007220616C206F726967656E0054726F76FE
:1084D00061206F726967696E65004175746F20680D
:1084E0006F6D6500207C20417574686F723A2000C2
:1084F000416C6C650057737A7973746B6F00546FBD
:10850000646F730054757474690056736500416C30
:108510006C00416374697665204578747275646592
:10852000723A2000FF12EF12DA12C712B3129E1233
:1085300013131B1323132C1334134D134913461316
:1085400043133F133C13511359130614EC13C9136F
:10855000A8139213611353151B15DD14A31475147E
:1085600024144C162C160516D915C01591154D1846
:10857000EC1782172617D0166F16841CD91BFA1A0F
:10858000411A9D19B0188F1E4C1E111EBC1D851D51
:10859000381D8E203520DF1F901F421FDC1EC62293
:1085A0005A22F32193214221D520CB247F242A244F
:1085B000DF23902325238B264826E925A9256D2531
:1085C0001C2542272E271027FB26E626C82607292A
:1085D000AD285028FE27B3275627FC2AAD2A532A58
:1085E000FE29B8294F29082CE42BB32B8B2B692BA0
:1085F000462BAB2C962C772C5C2C422C282C462D11
:10860000372D1E2D022DEB2CBF2C682E3A2E052E59
:10861000CB2DA42D632DB6305930DF2F812F262F7F
:10862000962E16311D3169315F3150314431393167
:108630002D31CD31BB31A9319731873175311432AC
:1086400014320232F0311432DE31843270325D3253
:108650004A3239322532EB32DA32C832B732A832F6
:1086600096325633443332331F330E33FB32693381
:10867000AA33A4339D3395338C337C33D533D53330
:10868000D533D533C333AF330B340B340B340B3406
:10869000F933E7336D345D344D343D342C341C34C0
:1086A000D334C234B134A0348E347D340236C7356D
:1086B0008C3550351B35E434A3368E367936643626
:1086C0004F363A36EF36E736DB36CF36C336B83676
:1086D0001137093711370137FB36113767375937EB
:1086E0004A373837293719378F378F3784377D37EF
:1086F0008F3772379937AD371A380C38FA37EB376E
:10870000DA37C83782387038613850383D382D38FC
:10871000DE38D038BF38AF38A038933838392B39E5
:108720001A390C39FF38EC388A397D397139633997
:10873000563949399739F739EE39E539DB39D239C4
:10874000C239FD39663A543A423A303A1E3A0D3A45
:10875000D23AC03AAE3A9C3A8A3A783A393B283B08
:10876000183B063BF63AE43AA43B923B7E3B6C3B1B
:10877000583B483BF33BE93BDC3BCE3BC33BB53B83
:10878000503C413C303C1E3C0E3CFC3B8E3C8E3C05
:108790007F3C6F3C8E3C5D3CE13CD23CC63CBB3CEC
:1087A000AE3CA03C0A3D0A3DFE3C0A3D0A3DF03C81
:1087B0006B3D5C3D4F3D3D3D2B3D173D873D873D2E
:1087C000803D873D793D873DB13DB13D9F3D8D3D2C
:1087D000B13DB13D1A3E093EF43DE03DCF3DC33DC4
:1087E0007E3E6C3E5B3E4A3E383E233EEF3EDA3EE6
:1087F000C53EB43EA03E903E333F333F213F113F44
:10880000333F003F7B3F7B3F693F573F7B3F443FC8
:10881000B13FB13FA33F973FB13F8B3FCF3FCF3FEA
:10882000C53FBA3FCF3FCF3F394024400F40FE3FC6
:10883000E93FD73FA340914081406F405D404A40AF
:108840000E41FC40EC40DA40C840B54079416741F8
:108850005741454133412041DD41CB41BB41AB4113
:1088600099418B414D423B42284216420442EF411E
:10887000B242A042914281426F425F4212430043A2
:10888000F242E842D642C442434343433443244382
:108890004343434350435C43614373438643D24362
:1088A000C443B943A8439B438E43DF43F14305448C
:1088B0005D444F4443443144234415446B4478445D
:1088C00086449444AA44B544244513450145EE44E6
:1088D000DD44CB448A457B456B455645454533458C
:1088E000DC45D145C145B045A4459945E945F2452A
:1088F0001A463C4673466246734673465146734673
:10890000A7469646A746A7468546A746CF46C446ED
:10891000CF46CF46B946CF462D471D470D47FA46AD
:10892000EA46DB468D477F476F475B474C473A47F0
:108930009B470E48F947E547D547C347B0477A48B4
:1089400066485648414832482148C348B948AD486E
:10895000A14899488E48CB48174908490049EE4834
:10896000E048D348EB49C54999496F4948492349EB
:10897000944A7B4A624A434A254A0B4AAC4AC34A54
:10898000364B264B174B064BF84AE84A184CF24B2D
:10899000C34B914B664B444B8A4C764C6D4C594CB7
:1089A000504C454CFB4CE94CD74CC44CB04C9E4C05
:1089B0005C4D4E4D3D4D2D4D1E4D0D4DBC4DAC4DA8
:1089C0009D4D8C4D7E4D6C4DAB502450964FEA4ED4
:1089D0005E4EC84D415144517951795167515851BA
:1089E00079514851CB51BC51B1519F519151825154
:1089F000F951F251EB51E251DC51D6515B524852E0
:108A00003652225213520052C252B152A1528E52C9
:108A10007C526F52DE52DB52DE52DE52D752D252BD
:108A20004553305320530B53F652E152F253D75370
:108A3000AF53945377535553425437542F542754BC
:108A40001B54125479546E5466545E545254495413
:108A5000B054A5549D54955489548054CF54CF5448
:108A6000BF54B754CF54CF5411550455F954EE5454
:108A7000E554D8542D552D551B552D552D552D5597
:108A80007A557055635557554C553F55A3559E55CE
:108A9000985592558D5586559C56735637560B569C
:108AA000D755A95511570257F256E356D756CC560B
:108AB00016572D5744575B57E657CF57B857A1570E
:108AC0008C577457FC57D958F05807596C59595955
:108AD0004A593D5931591E59CD59BD59AC599A5928
:108AE00088597959345A215A105AFB59EA59DB5995
:108AF0008F5A815A705A605A505A455AE95ADC5A6C
:108B0000CB5AB95AAC5A9D5A215B195B105B085B72
:108B1000015BF95A555B555B4C5B375B555B295BD9
:108B20005E5BCB5BBB5BA85B935B815B6F5BDB5B83
:108B3000E75BF35B1E5C195C135C0D5C085C015C1D
:108B4000E05CBC5C955C715C445C245C3F5D335DC7
:108B5000265D195D0D5D005D975D8A5D7A5D6B5DDB
:108B60005D5D4D5DE35DD65DCC5DC15DB65DA85DCF
:108B70003E5E305E1E5E095EFD5DEF5D8B5E815E7A
:108B8000705E625E575E4C5E935EA55EB75E0D6181
:108B90009A602860B45F3F5FC65EA3619C61956187
:108BA0008F6186617B61FF61EC61DB61C961B961E5
:108BB000A86130622B6225621F621A621362DE6254
:108BC000BF629A627762506236622C6323631563D8
:108BD0000863FE622C6337634963C263B2639D63BB
:108BE00083636C635C63286417640764F563E36301
:108BF000D2638364746465645564466438648D64C8
:108C0000B564B564AB64A2649864B564BE64CE64B4
:108C100044656E659865B665E965086622665E66B8
:108C200057664F665E664966416665667366786636
:108C30008266BE66BE66AF66A566BE66916613674F
:108C40000467F366E466D366C7665B674C67446790
:108C50003D672E672467636775678767D867CD6749
:108C6000BD67AA679E6792671B68126808680068FC
:108C7000F567EB672468936881686C685B6849688E
:108C80003468F268E368D268C268B668A46842696A
:108C900038692B691B6911690269A569936984693F
:108CA000726962695069B769FC69F069E669DD69F2
:108CB000D169C5693C6A2A6A3C6A3C6A186A066AD4
:108CC000946A866A7A6A6E6A5F6A4E6AA26AB36A50
:108CD0001D6CE96B9F6B586B0F6BC36AAD6D726D4A
:108CE000316DF26CAC6C666C416F046FC26E6D6E70
:108CF0002D6EF26DED70A6705A701370C96F846F8F
:108D00008B725172FE71B47172712E710374CB73D8
:108D1000877349731173C87262753475F774BF74C1
:108D2000887444740277BB7675763476E8759575E9
:108D3000A67858781B78E27793774677607A127A2C
:108D4000C5797A792F79E6782F7CE67B977B497B0A
:108D5000FC7AAD7ADB7D997D507D077DC77C7F7C79
:108D60006C7E5E7E4F7E3F7E2D7E1E7EAF7EA77E1A
:108D7000997E8A7E7F7E787EFE7EF27EE37ED47E42
:108D8000C77EB87E197F197F197F197F197F0D7FE4
:108D9000667F5A7F4B7F3C7F2E7F1F7FCD7FBC7FBE
:108DA000AA7F997F877F757F258019800A80FB7F46
:108DB000EE7FDF7F7C8070806180528043803480D2
:108DC0009D809D80978092808B809D80A8831A8350
:108DD0007382D0814081A18093848484748464846C
:108DE00052844584A184DA84DA84CC84BB84DA8416
:108DF000AD84E4840E850A850485FE84F584F084C0
:108E00001285457872656D65207370616E206F669E
:108E100020746865205A2076616C75657321004363
:108E2000616C63756C6174696F6E206F6620746825
:108E300065206D616368696E6520736B657720617D
:108E40006E64206F6666736574206661696C656424
:108E50002E00203C20005741524E494E473A2046B2
:108E6000726F6E7420706F696E74206E6F742072F2
:108E70006561636861626C652E205920636F6F7253
:108E800064696E6174653A00004974657261746961
:108E90006F6E3A2000496E76616C69642062656489
:108EA00020636F7272656374696F6E206D61747296
:108EB00069782E20526573657474696E6720746FCB
:108EC000206964656E746974792E00496E76616CF0
:108ED00069642062656420636F7272656374696F90
:108EE0006E206D61747269782E20582F5920617838
:108EF000657320617265206661722066726F6D20F5
:108F00006265696E672070657270656E646963750D
:108F10006C61722E00496E76616C696420626564D2
:108F200020636F7272656374696F6E206D61747215
:108F300069782E205368696674206F7574206F6697
:108F40002072616E67652E005A65726F20706F69BE
:108F50006E7420636F7272656374696F6E3A004954
:108F60006E76616C69642062656420636F727265FD
:108F70006374696F6E206D61747269782E204C6520
:108F80006E677468206F6620746865205920766566
:108F900063746F72206F7574206F662072616E67E4
:108FA000652E005920766563746F72206C656E675C
:108FB00074683A00496E76616C6964206265642069
:108FC000636F7272656374696F6E206D617472692C
:108FD000782E204C656E677468206F662074686513
:108FE000205820766563746F72206F7574206F66E9
:108FF0002072616E67652E005820766563746F720B
:10900000206C656E6774683A00556E646566696EBB
:1090100065642062656420636F7272656374696F52
:109020006E206D61747269782E000000404100006E
:10903000000000005C430000000000005C430000F2
:109040004043000040410000404300004041000018
:1090500000000000E4420000000000005743000050
:109060000000000057430000C0420000E44200003E
:10907000C042000040410000C042000040410000EA
:1090800040430000E442000040430000574300001A
:1090900040435A00205A3A00590020593A005800DB
:1090A00020583A0024F4D43050C38E20C2A2401776
:1090B000828B7011127A910D816CD90AA861E10836
:1090C000C7586607615143061E4B5D05C145A7049D
:1090D0001A411104093D9803713931034036DB020E
:1090E00065339102D4305402802E1D02632CEE01B0
:1090F000752AC501B028A001102781018F256401C0
:109100002B244B01E0223401AC211F018D200D01E5
:10911000801FFC00841EED00971DDF00B81CD200EC
:10912000E61BC600201BBC00641AB200B219A800DE
:109130000A19A0006A189900D117910040178B00F6
:10914000B516840031167E00B31579003A15730008
:10915000C7146F0058146A00EE136600881363008A
:1091600025135E00C7125B006C12570015125400E5
:10917000C111510070114F0021114B00D610490050
:109180008D1047004610440002104200C00F4000FE
:10919000800F3E00420F3C00060F3B00CB0E380014
:1091A000930E37005C0E3500270E3400F30D3200AD
:1091B000C10D3100900D3000600D2E00320D2D00DC
:1091C000050D2C00D90C2B00AE0C2900850C2900B4
:1091D0005C0C2700350C27000E0C2600E80B240041
:1091E000C40B2400A00B23007D0B23005A0B21008D
:1091F000390B2100180B2000F80A1F00D90A1E00A5
:10920000BB0A1E009D0A1D00800A1D00630A1C0087
:10921000470A1B002C0A1B00110A1A00F7091A0042
:10922000DD091900C4091900AB09190092091700DA
:109230007B091800630917004C091600360916004F
:10924000200916000A091500F5081500E0081400A9
:10925000CC081400B8081400A408140090081300E7
:109260007D0812006B08130058081200460812000F
:109270003408110023081100120811000108110020
:10928000F0071000E0071000D0071000C007100022
:10929000B0070F00A107100091070E0083070F0011
:1092A00074070F0065070E0057070E0049070E00F0
:1092B0003B070D002E070E0020070D0013070D00C1
:1092C00006070D00F9060C00ED060D00E0060C0087
:1092D000D4060C00C8060C00BC060C00B0060C003E
:1092E000A4060B0099060C008D060B0082060B00ED
:1092F00077060B006C060B0061060A0057060B0090
:109300004C060A0042060A0038060A002E060A0029
:1093100024060A001A060A001006090007060A00B9
:10932000FD050900F4050900EB050900E205090047
:10933000D9050900D0050900C7050900BE050900C7
:10934000B5050800AD050800A50509009C05080045
:10935000940508008C050800840508007C050800B9
:10936000740508006C050700650508005D05070029
:10937000560508004E050700470507004005080090
:1093800038050700310507002A05070023050700F7
:109390001C050600160507000F0507000805060056
:1093A00002050700FB040600F5040700EE040600B2
:1093B000E8040600E2040700DB040600D50406000A
:1093C000CF040600C9040600C3040600BD0406005D
:1093D000B7040600B1040500AC040600A6040600AC
:1093E000A00405009B0406009504050090040600F7
:1093F0008A04050085040500800406007A0405003F
:1094000075040500700405006B0405006604050082
:10941000610405005C0405005704050052040500C2
:109420004D04050048040500430405003E04040003
:109430003A04050035040500300404002C0405003E
:1094400027040400230405001E0404001A04040079
:1094500016040500110404000D04040009040500AD
:109460000404040000040400FC030400F8030400E6
:10947000F4030400F0030400EC030400E803040018
:10948000E4030400E0030400DC030400D803040048
:10949000D4030400D0030400CC030400C803030079
:1094A000C503030024F404D9201BC40C5C0E9804EB
:1094B000C4095F0265077101F405F900FB04B300FC
:1094C00048048700C10369005803550003034500A1
:1094D000BE023A008402310053022A00290225000C
:1094E00004022000E4011C00C8011900AF011700AC
:1094F0009801140084011300710110006101100033
:1095000051010E0043010D0036010B002B010B0031
:1095100020010B00150109000C01090003010800DE
:10952000FB000800F3000800EB000700E400060061
:10953000DE000600D8000600D2000600CC000500C0
:10954000C7000500C2000500BD000400B90004000A
:10955000B5000400B1000400AD000400A90004003F
:10956000A5000300A20003009F0004009B0003006D
:109570009800030095000200930003009000030090
:109580008D0002008B0003008800020086000200AC
:1095900084000300810002007F0002007D000200C1
:1095A0007B000200790002007700010076000200D3
:1095B0007400020072000100710002006F000200DE
:1095C0006D0001006C0002006A00010069000200E9
:1095D00067000100660001006500010064000200F0
:1095E0006200010061000100600001005F000200F4
:1095F0005D0001005C0001005B0001005A000100F9
:1096000059000100580001005700010056000100F8
:1096100055000100540001005300000053000100F8
:109620005200010051000100500001004F000100F4
:109630004E0000004E0001004D0001004C000100F2
:109640004B0000004B0001004A00010049000100EE
:1096500048000000480001004700010046000000EB
:1096600046000100450000004500010044000100E3
:1096700043000000430001004200000042000100DE
:109680004100000041000100400001003F000000D7
:109690003F0001003E0000003E0001003D000000D0
:1096A0003D0001003C0000003C0000003C000100C7
:1096B0003B0000003B0001003A0000003A000100BE
:1096C00039000000390001003800000038000000B7
:1096D00038000100370000003700010036000000AC
:1096E00036000000360001003500000035000000A3
:1096F0003500010034000000340000003400010097
:10970000330000003300000033000100320000008D
:109710003200000032000100310000003100000082
:109720003100010030000000300000003000010076
:109730002F0000002F0000002F0000002F0001006C
:109740002E0000002E0000002E0001002D00000061
:109750002D0000002D0000002D0001002C00000055
:109760002C0000002C0000002C0001002B00000049
:109770002B0000002B0000002B0001002A0000003D
:109780002A0000002A0000002A0001002900000031
:109790002900000029000000290000002900010024
:1097A0002800000028000000280000002800000019
:1097B000280001002700000027000000270000000B
:1097C00027000000270001002600000026000000FE
:1097D00026000000260000002600010025000000F1
:1097E00025000000250000002500000025000000E5
:1097F00025000100240000002400000024000000D7
:1098000024000000240001002300000023000000C9
:1098100023000000230000002300000023000000BC
:1098200023000100220000002200000022000000AE
:1098300022000000220000002200010021000000A0
:109840002100000021000000210000002100000094
:109850002100000021000100200000002000000085
:109860002000000020000000200000002000000078
:1098700020000000200001001F0000001F00000069
:109880001F0000001F0000001F0000001F0000005C
:109890001F0001001E0000001E0000001E0000004E
:1098A0001E0000004572723A204D494E54454D50FD
:1098B000204245440054656D70657261747572652F
:1098C00020686561746564206265642073776974DB
:1098D00063686564206F66662E204D494E54454D81
:1098E0005020747269676765726564202100457253
:1098F000723A204D415854454D5020424544005441
:10990000656D7065726174757265206865617465F6
:109910006420626564207377697463686564206F8E
:1099200066662E204D415854454D5020747269672B
:1099300067657265642021004572723A204D494E78
:1099400054454D50003A2045787472756465722014
:109950007377697463686564206F66662E204D496D
:109960004E54454D50207472696767657265642076
:1099700021004572723A204D415854454D50003AED
:1099800020457874727564657220737769746368B2
:109990006564206F66662E204D415854454D502019
:1099A00074726967676572656420210020484F54AE
:1099B000454E4420544845524D414C2052554E414D
:1099C0005741590020484541544245442054484598
:1099D000524D414C2052554E415741590054484533
:1099E000524D414C2052554E415741590042454439
:1099F00020544845524D414C2052554E41574159F3
:109A00000020544845524D414C2052554E4157413B
:109A1000592028205052454845415420484F54452C
:109A20004E44290020544845524D414C2052554E39
:109A3000415741592028205052454845415420481B
:109A4000454154424544290050524548454154201F
:109A50004552524F520042454420505245484541DC
:109A600054204552524F52004572723A205052498A
:109A70004E542046414E204552524F5200455252BC
:109A80004F523A205072696E742066616E20737076
:109A9000656564206973206C6F77657220746865F2
:109AA0006E206578706563746564004572723A2053
:109AB000455854522E2046414E204552524F520096
:109AC0004552524F523A204578747275646572203F
:109AD00066616E207370656564206973206C6F77B2
:109AE0006572207468656E2065787065637465645E
:109AF00000202D20496E76616C696420657874724F
:109B000075646572206E756D626572202100504922
:109B100044204175746F74756E652066696E697353
:109B2000686564212050757420746865206C6173C9
:109B300074204B702C204B6920616E64204B642094
:109B4000636F6E7374616E74732066726F6D2061E3
:109B5000626F766520696E746F20436F6E66696709
:109B600075726174696F6E2E6800504944204175AA
:109B7000746F74756E65206661696C65642120740C
:109B8000696D656F75740020403A006F6B20543A20
:109B9000006F6B20423A00504944204175746F7445
:109BA000756E65206661696C6564212054656D7011
:109BB0006572617475726520746F6F20686967687B
:109BC00000204B643A2000204B693A2000204B7063
:109BD0003A200020436C617373696320504944202C
:109BE000002054753A2000204B753A2000206D610A
:109BF000783A2000206D696E3A200020643A2000F7
:109C000020626961733A200010137D0020157800EE
:109C100060177300C0196E00401C6900E01E6400EC
:109C200080215F0040245A00F02655009029500002
:109C3000202C4B00802E4600C0304100D0323C002A
:109C4000B034370050363200C0372D0000392800BC
:109C5000103A2300F03A1E00B03B1900503C1400AB
:109C6000D03C0F00303D0A00803D0500C03D0000A3
:109C7000F03DFBFF103EF6FF303EF1FF403EECFFB3
:109C8000503EE7FF603EE2FF703EDDFF703ED8FFD2
:109C90001000C90210012C014001220170011801BD
:109CA000B0010E01F00104015002FA00B002F00010
:109CB0003003E600D003DC009004D2007005C80039
:109CC000A006BE000008B400B009AA00D00BA00096
:109CD000600E960060118C0000158200201978003B
:109CE000C01D6E00A0226400B0275A00902C5000C6
:109CF00000314600E0343C0010383200903A280031
:109D0000603C1E00A03D1400803E0A00203F000081
:109D100070012C0190012701B0012201C0011D0139
:109D2000F00118011002130130020E016002090156
:109D300090020401C002FF000003FA004003F50096
:109D40008003F000D003EB002004E6007004E10083
:109D5000E004DC004005D700C005D2004006CD007D
:109D6000D006C8008007C3003008BE00F008B90064
:109D7000C009B400B00AAF00B00BAA00D00CA50017
:109D8000000EA000500F9B00C010960050129100D2
:109D900000148C00C0158700B0178200B0197D0038
:109DA000D01B7800001E730040206E0090226900D6
:109DB000F024640040275F0090295A00E02B5500F2
:109DC000102E500020304B0010324600E03341008E
:109DD00090353C001037370070383200A0392D0024
:109DE000B03A2800A03B2300603C1E00103D190043
:109DF000903D1400103E0F00703E0A00C03E05006A
:109E0000003F0000544D4320445249564552204FD4
:109E100056455254454D502000436F6E74696E751F
:109E200065207769746820616E6F7468657220625E
:109E30006F7764656E3F005072696E742066616E64
:109E40003A0045787472756465722066616E3A00F6
:109E500041786973206C656E677468206469666612
:109E60006572656E63653A004D6561737572656410
:109E70002061786973206C656E6774683A004D38AC
:109E800034004731205A31350047323820570053CB
:109E9000746174653A2000473736004D3435205AD6
:109EA000004D3435004738300020003E003E002091
:109EB000003E003E003E003E0020003E003E0020EE
:109EC000000053657665726520736B65773A000014
:109ED000536C6967687420736B65773A002D2D2D7C
:109EE0002D2D2D2D2D2D2D2D2D2D2D2D2D2D2D2DA2
:109EF0002D004E2F41004D656173757265642073AE
:109F00006B65773A20004E2F41006D6D000052695D
:109F10006768743A004C6566743A00592064697346
:109F200074616E63652066726F6D206D696E3A00B4
:109F30004D373031004D373032004D35303000472D
:109F400031205A3135204631353030004739310023
:109F5000473120583530205931393020453020469E
:109F60003730303000473930004D373032004D3710
:109F700030322043004D3730322055004D373032DB
:109F8000004731205A3135204631353030004739CD
:109F90003100473120583530205931393020453093
:109FA000204637303030004D383300473930004DCF
:109FB0003834004D313034205330004D38340047B0
:109FC000312058313020593138302046343030304B
:109FD000004731205A31302046313330302E303076
:109FE00030004D313430205330004D313034205367
:109FF00030004D31303700473120452D302E30377D
:10A000003530302046323130302E30303030300074
:10A01000473120583530205935352045332E3632DA
:10A02000373733004731205832303020593535200A
:10A0300045302E34393338360047312058323030ED
:10A04000205937352045332E3632373733004731E4
:10A0500020583530205937352045302E34393338A3
:10A060003600473120583530205939352045332EB8
:10A0700036323737330047312058323030205939A3
:10A08000352045302E3439333836004731205832A8
:10A09000303020593131352045332E363237373381
:10A0A0000047312058353020593131352045302E88
:10A0B0003439333836004731205835302059313360
:10A0C000352045332E36323737330047312058326A
:10A0D000303020593133352045302E363631373443
:10A0E0000047312058323030205931353520453243
:10A0F0002E3632373733004731205831303020592F
:10A100003135352045320047312058373520593117
:10A1100035352045322E3500473120463130383034
:10A12000004731205835302059313535004731202E
:10A130004634303030004D323034205331303030FE
:10A14000004731205A302E313530204637323030FA
:10A150002E30303000473120452D312E3530303013
:10A16000302046323130302E3030303030004D38F3
:10A17000330047393000473231004739322045300B
:10A180002E3000473120583130302E3020453132CA
:10A190002E352046313030302E30004731205836B1
:10A1A000302E302045392E302046313030302E30A0
:10A1B000004739322045302E3000473238004738CA
:10A1C00037004D3130392053323130004D31393084
:10A1D00020533535004D31343020533535004D3165
:10A1E00030342053323130004D3130370047393070
:10A1F000004731204531004D3832004D3833004D95
:10A2000031303620532564004D32323020532564DE
:10A21000003A200020202020202020202020202064
:10A220002020202020202000203A20002020202054
:10A23000202020202020202020202020202020201E
:10A240000020202020202020202020202020002549
:10A2500073002020002D2D3A2D2D002000200020FD
:10A26000004C002020002046002D2D2D003E55538F
:10A2700042005344002D2D002520202020200020C6
:10A2800020002020000120002020202D2D2D200046
:10A2900020205A002020000120004D36303000469A
:10A2A0004C4558202D20203233302F35300050506F
:10A2B0002020202D20203235342F313030004849E5
:10A2C0005053202D20203232302F31303000504575
:10A2D0005420202D20203234302F393000504C4172
:10A2E00020202D20203231352F353500414253209A
:10A2F000202D20203235352F313030006661726DCF
:10A3000020202D20203235302F3430004D323400C3
:10A310004D323320257300052E2E00580059005A67
:10A320000045787472756465720047393900446974
:10A330007361626C65206661726D206D6F64653F4C
:10A340000044697361626C65206661726D206D6F97
:10A350006465004661726D206E756D626572004DB8
:10A360003834005A30005A31005930005931005801
:10A370003000583100456E642073746F7073206430
:10A38000696167004D343400473238205700417509
:10A39000746F207265636F76657220637261736893
:10A3A00000436865636B2066616E73205B444953AC
:10A3B0005D00436865636B2066616E73205B454E8C
:10A3C0005D0054656D7065726174757265730058D7
:10A3D000595A2063616C2E2064657461696C730046
:10A3E0002D2D2D2D2D2D2D2D2D2D2D2D00466C613E
:10A3F000736841697220495020416464723A002DAB
:10A400002D2D2D2D2D2D2D2D2D2D2D004E6F76200A
:10A410003133203230313700446174653A20002DE9
:10A420002D2D2D2D2D2D2D2D2D2D2D00453344760B
:10A430003666756C6C0045494E595F3034610031A9
:10A440005F37356D6D5F4D4B33002D2D2D2D2D2D2F
:10A450002D2D2D2D2D2D0020332E302E31322D522D
:10A4600043322062313038004669726D776172651F
:10A470003A0025642E25642E25642E25640046614D
:10A48000696C207374617473004661726D206E751F
:10A490006D62657200007263006265746100616CD8
:10A4A00070686100646576005052555341334446EC
:10A4B0005700332E302E31322D5243320000000A25
:10A4C0000B02090C0D0E0807030401000000000038
:10A4D000000000000000000000000000000000007C
:10A4E0000000000000000000001211100000000039
:10A4F000000000000000000000000000000000005C
:10A50000000000000000000000000000000000004B
:10A5100000000001021020200808102040102040F8
:10A520008002010201080402010102040810204017
:10A530008080402010080402018004020180402035
:10A54000100804020108040201010204081020405E
:10A5500080010204081020408010080408801020A8
:10A5600040044080102040048005050505070508CB
:10A57000080808020202020A0A0808040404040186
:10A5800001010101010101030303030303030304A8
:10A590000707070C0C0C0C0C0C0C0C020202020638
:10A5A000060606060606060B0B0B0B0B0B0B0B0722
:10A5B000070A0A0A0A0A0A0505050404040808002D
:10A5C0000020002300260029002C002F003200006C
:10A5D00001000003010601090100002200250028F6
:10A5E000002B002E0031003400020100000501089C
:10A5F000010B0100002100240027002A002D00305B
:10A6000000330001010000040107010A01024E416C
:10A610004E494E495459494E46CDCCCC3D0AD723DC
:10A620003C17B7D13877CC2B329595E6241FB14F24
:10A630000A000020410000C84200401C4620BCBE69
:10A640004CCA1B0E5AAEC59D7400407A10F35A00D6
:10A65000A0724E18090010A5D4E80000E87648174B
:10A660000000E40B54020000CA9A3B000000E1F530
:10A6700005000080969800000040420F000000A0F6
:10A680008601000000102700000000E80300000021
:10A69000006400000000000A00000000000100004B
:10A6A0000000002C76D888DC674F0823DFC1DFAEBE
:10A6B00059E1B1B796E5E3E453C63AE65199769687
:10A6C000E8E6C28426EB898C9B62ED407C6FFCEF50
:10A6D000BC9C9F40F2BAA56FA5F490055A2AF75C7E
:10A6E000936B6CF9676DC11BFCE0E40D47FEF52030
:10A6F000E6B500D0ED902E030094357705008084F8
:10A700001E080000204E0A000000C80C333333330B
:10A710000F986E12831141EF8D2114893BE6551677
:10A72000CFFEE6DB18D1844B381BF77C1D901DA4AF
:10A73000BBE424203284725E228100C9F124ECA1A2
:10A74000E53D270064C5FAEBAF013101FD0195C578
:10A7500011241FBECFEFD1E2DEBFCDBF00E00CBFA2
:10A760001AE0A0E0B2E0E8E6FCEC03E00BBF02C0B8
:10A7700007900D92A036B107D9F72CE1A0E6BAE018
:10A7800001C01D92A439B207E1F717EACEE4D7EA77
:10A7900000E006C022970109FE010BBF0F94A4DC64
:10A7A000C434D10780E00807A9F70F948BD60D9425
:10A7B00022E60C940000CF92DF92EF92FF920F936B
:10A7C0001F93CF93DF938C01D42EC62FD72FD60E95
:10A7D000DC1671F1F801E080F180C990C7010F9497
:10A7E000E6E2C816F1F06C2DC7010F9416E3C7011D
:10A7F0000F94E6E28C15A9F0E2EAF7E08491882351
:10A8000041F09091C00095FFFCCF8093C600319637
:10A81000F5CF8091C00085FFFCCF8AE08093C60011
:10A8200007C0F80180819181019691838083D0CF08
:10A83000DF91CF911F910F91FF90EF90DF90CF901C
:10A840000895EF92FF920F931F93CF93DF931F9280
:10A85000CDB7DEB78C017B01460FF8018081918175
:10A8600049830F94E6E2F70181937F01F80180812B
:10A87000918101969183808349814E11EECF0F9093
:10A88000DF91CF911F910F91FF90EF900895FF926C
:10A890000F931F93CF93DF93CDB7DEB72C970FB6EF
:10A8A000F894DEBF0FBECDBF8C01F62E80E390E39F
:10A8B000A0E3B0E08D839E83AF83B8871C870B87AE
:10A8C00044E0BE016B5F7F4FCE010B9674DF40E129
:10A8D0006EEE79E1CE010B966EDF40E16EEF79E12D
:10A8E000CE010B9668DF40E16EED79E1CE010B966B
:10A8F00062DF44E066ED79E1CE010B965CDF44E077
:10A9000062ED79E1CE010B9656DF44E06AED79E124
:10A91000CE010B9650DF44E06EEB79E1CE010B9651
:10A920004ADF44E06EE07AE1CE010B9644DF44E07A
:10A9300062EC79E1CE010B963EDF44E066EC79E112
:10A94000CE010B9638DF44E06AEC79E1CE010B963C
:10A9500032DF44E06EEC79E1CE010B962CDF4CE067
:10A960006AE97BE0CE010B9626DF44E063E97BE0F9
:10A97000CE010B9620DF44E066EA72E0CE010B9632
:10A980001ADF44E062EA72E0CE010B9614DF44E085
:10A990006EE972E0CE010B960EDF44E066E972E0EC
:10A9A000CE010B9608DF44E062E972E0CE010B961F
:10A9B00002DF44E06EE872E0CE010B96FCDE80E23E
:10A9C00090E09A87898742E0BE01675F7F4FCE01A2
:10A9D0000B96F1DE41E06FE87BE0CE010B96EBDEFB
:10A9E00044E06DE172E0CE010B96E5DE44E065E106
:10A9F00072E0CE010B96DFDE44E06AE87BE0CE0138
:10AA00000B96D9DE44E066E87BE0CE010B96D3DE00
:10AA100044E061E172E0CE010B96CDDE41E066EBF1
:10AA20007BE0CE010B96C7DE44E06DE372E0CE0121
:10AA30000B96C1DE89E08F1560F444E06DE074E1AF
:10AA4000CE010B96B8DE44E069E074E1CE010B96CE
:10AA5000B2DE46E551E360E070E049835A836B83E0
:10AA60007C831C870B8744E0BE016F5F7F4FCE0164
:10AA70000B96A1DEE2E0FFE08491882341F0909103
:10AA8000C00095FFFCCF8093C6003196F5CFE2E978
:10AA9000F7E08491882341F09091C00095FFFCCFAE
:10AAA0008093C6003196F5CF8091C00085FFFCCF22
:10AAB0008AE08093C6002C960FB6F894DEBF0FBED6
:10AAC000CDBFDF91CF911F910F91FF9008951F93FC
:10AAD000CF93DF93182FC2E0DFE0FE01849188233B
:10AAE00041F09091C00095FFFCCF8093C600319655
:10AAF000F5CFE2E8F7E08491882341F09091C0001F
:10AB000095FFFCCF8093C6003196F5CF8091C000B1
:10AB100085FFFCCF8AE08093C600FE018491E2E0CD
:10AB2000FFE0882349F09091C00095FFFCCF80930F
:10AB3000C60031968491F5CF4091EE195091EF19EE
:10AB40006091F0197091F1198AE797E00E94FE6C0C
:10AB50004091F2195091F3196091F4197091F5191F
:10AB600087E797E00E94FE6C4091F6195091F71923
:10AB70006091F8197091F91984E797E00E94FE6CD2
:10AB80004091FA195091FB196091FC197091FD19CF
:10AB900081E797E00E94FE6C8091C00085FFFCCFAA
:10ABA0008AE08093C600FE018491E2E0FFE0882302
:10ABB00049F09091C00095FFFCCF8093C60031967C
:10ABC0008491F5CFE7E5F7E08491882341F09091F7
:10ABD000C00095FFFCCF8093C6003196F5CF8091E1
:10ABE000C00085FFFCCF8AE08093C600FE018491FF
:10ABF000E2E0FFE0882349F09091C00095FFFCCF90
:10AC00008093C60031968491F5CF4091FE19509102
:10AC1000FF196091001A7091011A8EE497E00E946A
:10AC2000FE6C4091021A5091031A6091041A7091BF
:10AC3000051A8BE497E00E94FE6C4091061A509131
:10AC4000071A6091081A7091091A88E497E00E9427
:10AC5000FE6C40910A1A50910B1A60910C1A709177
:10AC60000D1A85E497E00E94FE6C8091C00085FF7C
:10AC7000FCCF8AE08093C600FE018491E2E0FFE011
:10AC8000882349F09091C00095FFFCCF8093C600C7
:10AC900031968491F5CFE7E2F7E08491882341F083
:10ACA0009091C00095FFFCCF8093C6003196F5CF00
:10ACB0008091C00085FFFCCF8AE08093C600FE0132
:10ACC0008491E2E0FFE0882349F09091C00095FF75
:10ACD000FCCF8093C60031968491F5CF4091DE1968
:10ACE0005091DF196091E0197091E1198EE197E0C0
:10ACF0000E940F6D4091E2195091E3196091E4199F
:10AD00007091E5198BE197E00E940F6D4091E61973
:10AD10005091E7196091E8197091E91988E197E07D
:10AD20000E940F6D4091EA195091EB196091EC1956
:10AD30007091ED1985E197E00E940F6D8091C00040
:10AD400085FFFCCF8AE08093C600FE018491E2E09B
:10AD5000FFE0882349F09091C00095FFFCCF8093DD
:10AD6000C60031968491F5CFE0EEF6E08491882319
:10AD700041F09091C00095FFFCCF8093C6003196C2
:10AD8000F5CF8091C00085FFFCCF8AE08093C6009C
:10AD9000FE018491E2E0FFE0882349F09091C00039
:10ADA00095FFFCCF8093C60031968491F5CF4091FA
:10ADB000D6195091D7196091D8197091D91987ED8A
:10ADC00096E00E94FE6C4091D2195091D319609187
:10ADD000D4197091D51984ED96E00E94FE6C809193
:10ADE000C00085FFFCCF8AE08093C600FE018491FD
:10ADF000E2E0FFE0882349F09091C00095FFFCCF8E
:10AE00008093C60031968491F5CFE1E2F6E084911B
:10AE1000882341F09091C00095FFFCCF8093C6003D
:10AE20003196F5CF8091C00085FFFCCF8AE08093FA
:10AE3000C600FE018491E2E0FFE0882349F0909192
:10AE4000C00095FFFCCF8093C60031968491F5CF6A
:10AE50004091DA195091DB196091DC197091DD197C
:10AE600088E196E00E94FE6C4091BE195091BF1996
:10AE70006091C0197091C11985E196E00E94FE6C45
:10AE800040910E1A50910F1A6091101A7091111A78
:10AE900082E196E00E940F6D4091C2195091C31952
:10AEA0006091C4197091C5198FE096E00E94FE6C04
:10AEB0004091C6195091C7196091C8197091C9196C
:10AEC0008CE096E00E94FE6C4091CA195091CB191B
:10AED0006091CC197091CD1989E096E00E94FE6CCA
:10AEE0004091CE195091CF196091D0197091D1191C
:10AEF00086E096E00E94FE6C8091C00085FFFCCF4A
:10AF00008AE08093C600FE018491E2E0FFE088239E
:10AF100049F09091C00095FFFCCF8093C600319618
:10AF20008491F5CFE4EFF5E08491882341F090918E
:10AF3000C00095FFFCCF8093C6003196F5CF80917D
:10AF4000C00085FFFCCF8AE08093C600FE0184919B
:10AF5000E2E0FFE0882349F09091C00095FFFCCF2C
:10AF60008093C60031968491F5CF40919A0B509111
:10AF70009B0B60919C0B70919D0B8BEE95E00E945A
:10AF8000FE6C40919E0B50919F0B6091A00B7091B5
:10AF9000A10B88EE95E00E94FE6C4091A20B5091AF
:10AFA000A30B6091A40B7091A50B85EE95E00E9418
:10AFB000FE6C8091C00085FFFCCF8AE08093C600C4
:10AFC000FE018491E2E0FFE0882349F09091C00007
:10AFD00095FFFCCF8093C60031968491F5CFE7EDC5
:10AFE000F5E08491882341F09091C00095FFFCCF5B
:10AFF0008093C6003196F5CF8091C00085FFFCCFCD
:10B000008AE08093C600FE018491E2E0FFE088239D
:10B0100049F09091C00095FFFCCF8093C600319617
:10B020008491F5CF4091A6025091A7026091A802A9
:10B030007091A9028DEC95E00E94FE6C6091A202D5
:10B040007091A3028091A4029091A5020F946A5975
:10B05000AB01BC018AEC95E00E94FE6C60919E02FF
:10B0600070919F028091A0029091A1020F94765955
:10B07000AB01BC0187EC95E00E94FE6C8091C000A2
:10B0800085FFFCCF8AE08093C600FE018491E2E058
:10B09000FFE0882349F09091C00095FFFCCF80939A
:10B0A000C60031968491F5CFE1EBF5E084918823D9
:10B0B00041F09091C00095FFFCCF8093C60031967F
:10B0C000F5CF8091C00085FFFCCF8AE08093C60059
:10B0D000FE018491E2E0FFE0882349F09091C000F6
:10B0E00095FFFCCF8093C60031968491F5CF4091B7
:10B0F000960250919702609198027091990287EAA6
:10B1000095E00E94FE6C6091920270919302809192
:10B110009402909195020F946A59AB01BC0184EAA4
:10B1200095E00E94FE6C60918E0270918F0280917A
:10B130009002909191020F947659AB01BC0181EA83
:10B1400095E00E94FE6C8091C00085FFFCCF8AE0F4
:10B150008093C600FE018491E2E0FFE0882349F07D
:10B160009091C00095FFFCCF8093C60031968491EA
:10B17000F5CFEDE6F5E08491882341F09091C00091
:10B1800095FFFCCF8093C6003196F5CF8091C0002B
:10B1900085FFFCCF8AE08093C600FE018491E2E047
:10B1A000FFE0882349F09091C00095FFFCCF809389
:10B1B000C60031968491F5CF40911D0250911E0238
:10B1C00060911F027091200283E695E00E94FE6C60
:10B1D00020E030E040E752E46091150270911602E1
:10B1E00080911702909118020F9448DAAB01BC01CC
:10B1F00080E695E00E94FE6C40918A0B50918B0B8B
:10B2000060918C0B70918D0B8DE595E00E94FE6C2A
:10B210008091C00085FFFCCF8AE08093C600FE01CC
:10B220008491E2E0FFE0882349F09091C00095FF0F
:10B23000FCCF8093C60031968491F5CFE1E3F5E031
:10B240008491882341F09091C00095FFFCCF8093BA
:10B25000C6003196F5CF8091C00085FFFCCF8AE013
:10B260008093C600FE018491E2E0FFE0882349F06C
:10B270009091C00095FFFCCF8093C60031968491D9
:10B28000F5CF4091860B5091870B6091880B7091A0
:10B29000890B87E295E00E94FE6C20E030E040E7F9
:10B2A00052E4609111027091120280911302909108
:10B2B00014020F9448DAAB01BC0184E295E00E94CD
:10B2C000FE6C8091C00085FFFCCF8AE08093C600B1
:10B2D000FE018491E2E0FFE0882349F09091C000F4
:10B2E00095FFFCCF8093C60031968491F5CFEAECB0
:10B2F000F4E08491882341F09091C00095FFFCCF49
:10B300008093C6003196F5CF8091C00085FFFCCFB9
:10B310008AE08093C600FE018491E2E0FFE088238A
:10B3200049F09091C00095FFFCCF8093C600319604
:10B330008491F5CF40918F0B50E060E070E080EC9D
:10B3400094E00E940F6D8091C00085FFFCCF8AE0E1
:10B350008093C600FE018491E2E0FFE0882349F07B
:10B360009091C00095FFFCCF8093C60031968491E8
:10B37000F5CF8091B60B8823A1F1EDEAF4E084913A
:10B38000882341F09091C00095FFFCCF8093C600C8
:10B390003196F5CF8091C00085FFFCCF8AE0809385
:10B3A000C600FE018491E2E0FFE0882349F090911D
:10B3B000C00095FFFCCF8093C60031968491F5CFF5
:10B3C00040913D0250913E0260913F0270914002D7
:10B3D00083EA94E00E94FE6C8091C00085FFFCCF60
:10B3E00011C0E7E8F4E08491882341F09091C00017
:10B3F00095FFFCCF8093C6003196F5CF8091C000B9
:10B4000085FFFCCF8AE08093C6001A3008F43EC066
:10B41000FE01C491E2E0FFE0CC2349F08091C0003E
:10B4200085FFFCCFC093C6003196C491F5CFEEE600
:10B43000F4E08491882341F09091C00095FFFCCF07
:10B440008093C6003196F5CF8091C00085FFFCCF78
:10B450008AE08093C60040910D1450910E146091C3
:10B460000F147091101484E694E00E94FE6C4091D9
:10B47000091450910A1460910B1470910C148AE510
:10B4800094E0DF91CF911F910C94FE6CDF91CF91EE
:10B490001F910895AF92BF92CF92DF92EF92FF92E9
:10B4A0000F931F93CF93DF93CDB7DEB7E0970FB61F
:10B4B000F894DEBF0FBECDBF80E1EBEDF2E0DE0120
:10B4C000919601900D928A95E1F780E1EBEEF2E022
:10B4D000DE01519601900D928A95E1F780E1EBEF44
:10B4E000F2E0DE01119601900D928A95E1F76E016E
:10B4F00081E2C80ED11C8EEEE82E89E1F82E8E0175
:10B500000F5E1F4F6EEF79E1AE014F5F5F4F9EED13
:10B51000A92E99E1B92E20E030E0F60181919191B8
:10B52000A191B1916F01F70181939193A193B1938F
:10B530007F01F80181919191A191B1918F01FB015E
:10B5400081939193A193B193BF01FA01819191915C
:10B55000A191B191AF01F50181939193A193B19321
:10B560005F012F5F3F4F24303105B9F60F9443360A
:10B5700080E090E4ACE9B4E48093D6199093D719B5
:10B58000A093D819B093D9198093D2199093D31955
:10B59000A093D419B093D5191092DA191092DB192F
:10B5A0001092DC191092DD1980E29EE4A0E0B0E078
:10B5B00080930E1A90930F1AA093101AB093111A39
:10B5C0001092BE191092BF191092C0191092C11991
:10B5D00080E090E0A0E7B1E48093C2199093C31992
:10B5E000A093C419B093C5198093C6199093C71935
:10B5F000A093C819B093C9198DEC9CECACECBEE3D8
:10B600008093CA199093CB19A093CC19B093CD19FC
:10B6100080E090E0A0E2B0E48093CE199093CF193F
:10B62000A093D019B093D1191092A20B1092A30B32
:10B630001092A40B1092A50B10929E0B10929F0BD0
:10B640001092A00B1092A10B10929A0B10929B0BD0
:10B6500010929C0B10929D0B8DE39AE0A1E8B1E44F
:10B660008093A6029093A702A093A802B093A90288
:10B670006DEC7CEC84E99FE30F9464596093A20223
:10B680007093A3028093A4029093A50265E87BEED9
:10B6900080E692E40F94705960939E0270939F022B
:10B6A0008093A0029093A1020F94AA4880E090E0BA
:10B6B000A0E8BFE380939A0290939B02A0939C0220
:10B6C000B0939D0210928F0B80E090E0A0E4B0E474
:10B6D00080931D0290931E02A0931F02B09320023C
:10B6E00040E050E064E372E4409315025093160288
:10B6F000609317027093180210928A0B10928B0BB2
:10B7000010928C0B10928D0B1092860B1092870B5F
:10B710001092880B1092890B40E050E060E071E4D9
:10B72000409311025093120260931302709314021B
:10B730001092B60B80933D0290933E02A0933F027D
:10B74000B09340020E947882E2E0FFE08491882377
:10B7500041F09091C00095FFFCCF8093C6003196D8
:10B76000F5CFEEE1F4E08491882341F09091C000A0
:10B7700095FFFCCF8093C6003196F5CF8091C00035
:10B7800085FFFCCF8AE08093C600E0960FB6F89460
:10B79000DEBF0FBECDBFDF91CF911F910F91FF9004
:10B7A000EF90DF90CF90BF90AF9008951F93CF930D
:10B7B000DF93CDB7DEB72C970FB6F894DEBF0FBE80
:10B7C000CDBF162F9C878B8786E591E3A0E0B0E084
:10B7D00089839A83AB83BC8344E0BE016B5F7F4F58
:10B7E000CE010B962ED843E050E0BE016B5F7F4F39
:10B7F000CE0101960F9455E0892B09F0FFC040E17E
:10B800006EEE79E1CE010B961CD840E16EEF79E146
:10B81000CE010B9616D840E16EED79E1CE010B9684
:10B8200010D80F94433644E066ED79E1CE010B96D3
:10B8300008D844E062ED79E1CE010B9602D844E0ED
:10B840006AED79E1CE010B960E94215444E06EEB43
:10B8500079E1CE010B960E94215444E06EE07AE13A
:10B86000CE010B960E94215444E062EC79E1CE01B6
:10B870000B960E94215444E066EC79E1CE010B96D0
:10B880000E94215444E06AEC79E1CE010B960E94BB
:10B89000215444E06EEC79E1CE010B960E942154D4
:10B8A0004CE06AE97BE0CE010B960E94215444E013
:10B8B00063E97BE0CE010B960E94215444E066EAE6
:10B8C00072E0CE010B960E94215444E062EA72E0DD
:10B8D000CE010B960E94215444E06EE972E0CE0145
:10B8E0000B960E94215444E066E972E0CE010B966B
:10B8F0000E94215444E062E972E0CE010B960E945E
:10B90000215444E06EE872E0CE010B960E9421546F
:10B9100042E0BE01675F7F4FCE010B960E9421542B
:10B9200041E06FE87BE0CE010B960E94215444E099
:10B930006DE172E0CE010B960E94215444E065E176
:10B9400072E0CE010B960E94215444E06AE87BE04D
:10B95000CE010B960E94215444E066E87BE0CE01C4
:10B960000B960E94215444E061E172E0CE010B96F7
:10B970000E94215441E066EB7BE0CE010B960E94D1
:10B98000215444E06DE372E0CE010B960E942154F5
:10B990001A3070F044E06DE074E1CE010B960E9425
:10B9A000215444E069E074E1CE010B960E942154D9
:10B9B0000E9478820F94AA48E2E0FFE084918823F5
:10B9C00041F09091C00095FFFCCF8093C600319666
:10B9D000F5CFE0E4F4E08491882341F09091C00039
:10B9E00095FFFCCF8093C6003196F5CF8091C000C3
:10B9F00085FFFCCF8AE08093C60001C04BDD2C960A
:10BA00000FB6F894DEBF0FBECDBFDF91CF911F916F
:10BA10000895682F772767FD70958091F2109091B7
:10BA2000F31089509F4E0F943AE09093E910809361
:10BA3000E81021E0892B09F420E0822F08958091FD
:10BA4000E8109091E91060E070E001960D94E3DC5D
:10BA50008A3010F0895A01C0805D9091C00095FF36
:10BA6000FCCF8093C6000895CF93C82F82958F7026
:10BA7000EFDF8C2F8F70CF91EBCFCF93C82F892F13
:10BA8000F3DF8C2FCF91F0CFCF93DF93FB0120E03A
:10BA900030E0DC01ED018D918823A1F141155105C4
:10BAA00019F02417350774F58032A1F38A3051F16B
:10BAB00090ED980F9A3020F4682F6295607F08C04F
:10BAC0009FE9980F9630A8F4682F6295607F6057C1
:10BAD000CE0102967981A0EDA70FAA3018F4762F37
:10BAE0007A2B0CC0AFE9A70FA63018F47755762B48
:10BAF00005C088279927821B930B05C071932F5F80
:10BB00003F4FC7CFC901DF91CF910895E091E81071
:10BB1000F091E91081818823C9F063E673E080E643
:10BB20009AE00E94F76682E474DF882369F0F89453
:10BB300028E088E190E00FB6F894A8958093600023
:10BB40000FBE20936000FFCF0C9400000895CF93A8
:10BB5000DF936EE673E080E69AE00E94F766F89461
:10BB6000C0E0D0E060E0CE010F9416E32196C1154D
:10BB700080E1D807B9F77894DF91CF910895AF921B
:10BB8000BF92CF92DF92EF92FF920F931F93CF93CA
:10BB9000DF93CDB7DEB760970FB6F894DEBF0FBE68
:10BBA000CDBF60E873E080E69AE00E94F76681E42A
:10BBB00030DF8823A9F08091E8109091E910FC0112
:10BBC0002181283741F440E150E060E070E00296C6
:10BBD0000F944BDE03C033DF0F94E2D77B0102C02A
:10BBE000E12CF12C83E415DF882331F028DF0F945A
:10BBF000E2D7262F872F02C020E080E2FFE1FF225C
:10BC0000022F182F013020E2120710F000E010E29E
:10BC1000C8018E0D9F1D8130904220F000E010E29F
:10BC20000E191F0988E5F5DE882381F18091E8105F
:10BC30009091E91040E150E0BE016F5F7F4F0196A7
:10BC400023DF8C01009711F1FE013196CF01800FA7
:10BC5000911FD701E817F90719F021912D93FACF19
:10BC60004AE050E0B80180E69AE00E945C6764E92F
:10BC700073E080E69AE00E94F766C701FEDE8091DD
:10BC8000C00085FFFCCF8AE08093C60080E2B82E1A
:10BC90009AE0A92E0115110529F1C701EEDE809168
:10BCA000C00085FFFCCFB092C6006701F0E1CF0E67
:10BCB000D11CF7012FEFE21AF20A80819091C000A7
:10BCC00095FFFCCFB092C600CFDE0150110919F0EC
:10BCD000EC14FD0471F78091C00085FFFCCFA092A9
:10BCE000C600D8CF60960FB6F894DEBF0FBECDBFAA
:10BCF000DF91CF911F910F91FF90EF90DF90CF9048
:10BD0000BF90AF900895AF92BF92CF92DF92EF9223
:10BD1000FF920F931F93CF93DF93CDB7DEB760975A
:10BD20000FB6F894DEBF0FBECDBF66EB73E080E6C2
:10BD30009AE00E94F76681E46CDE8823A9F0809186
:10BD4000E8109091E910FC012181283741F440E18D
:10BD500050E060E070E002960F944BDE03C06FDEAF
:10BD60000F94E2D77B0102C0E12CF12C83E451DE79
:10BD7000882331F064DE0F94E2D7262F872F02C08C
:10BD800020E080E2FFE1FF22022F182F013020E2A5
:10BD9000120710F000E010E2C8018E0D9F1D8130E7
:10BDA000904220F000E010E20E191F0988E531DE14
:10BDB0008823B9F18091E8109091E91040E150E0BA
:10BDC000BE016F5F7F4F01965FDE8C01009749F1E6
:10BDD000CE0101965C01C12CD12CC016D10661F0B8
:10BDE000F50161915F01C6018E0D9F1D0F9416E351
:10BDF000FFEFCF1ADF0AF1CF4AE050E0B80180E64A
:10BE00009AE00E945C676DEC73E080E69AE0EFD701
:10BE1000C70133DE8091C00085FFFCCF8AE08093AC
:10BE2000C60020E2B22E3AE0A32E0115110531F131
:10BE3000C70123DE8091C00085FFFCCFB092C60011
:10BE4000670120E1C20ED11CC701EFEFEE1AFE0A16
:10BE50000F94E6E29091C00095FFFCCFB092C6002F
:10BE600003DE0150110919F0EC14FD0469F780910B
:10BE7000C00085FFFCCFA092C600D7CF60960FB65A
:10BE8000F894DEBF0FBECDBFDF91CF911F910F9110
:10BE9000FF90EF90DF90CF90BF90AF900895CF923A
:10BEA000DF92EF92FF92CF93DF9362EF73E080E631
:10BEB0009AE09DD780E5ADDD882309F46BC0BFDD36
:10BEC0000F94E2D76B017C018FEFC816D10411F0FB
:10BED00008F060C086E49DDD882379F0B0DD0F9422
:10BEE000E2D76115710511F460E004C0613071059D
:10BEF00021F461E08C2D0F9491D086E58ADD8823B2
:10BF0000B1F09DDD0F94E2D76115710511F460E089
:10BF100005C06130710509F03DC061E08C2DDF91F5
:10BF2000CF91FF90EF90DF90CF900D94CAD08C2DE1
:10BF30000F94FFD0C1E0D0E0892B11F4C0E0D0E035
:10BF4000E2E0F4E08191882339F09091C00095FF00
:10BF5000FCCF8093C600F6CF4AE050E0B60180E601
:10BF60009AE052D7EDEBF4E08191882339F090917B
:10BF7000C00095FFFCCF8093C600F6CF4AE050E0AA
:10BF8000BE0180E69AE0DF91CF91FF90EF90DF90C5
:10BF9000CF9041C7DF91CF91FF90EF90DF90CF908E
:10BFA00008959F92AF92BF92CF92DF92EF92FF924D
:10BFB0000F931F93CF93DF93CDB7DEB761970FB683
:10BFC000F894DEBF0FBECDBF66E074E080E69AE075
:10BFD0000ED781E41EDD8823D9F08091E81090917E
:10BFE000E910FC012181283751F440E150E060E084
:10BFF00070E002960F944BDE6B017C010CC01FDDDC
:10C000000F94E2D76B01EE24D7FCE094FE2C03C022
:10C01000C12CD12C760183E4FCDC882331F00FDDC8
:10C020000F94E2D7262F872F02C020E084E0F3E0B0
:10C03000EF22FF24022F182F013020E2120710F008
:10C0400000E010E2D701C601800F911FA11DB11DB4
:10C050000197A440B10520F0002711270C191D09F4
:10C0600085E4D7DCB82E88E5D4DC8823C9F080913C
:10C07000E8109091E91040E150E0BE016F5F7F4F02
:10C08000019602DD8C0121E0009709F420E0B11057
:10C090000AC0211125C050E2B52E6AE0A62E96C036
:10C0A000BB20C9F320E04AE050E0B80180E69AE006
:10C0B000298B02D76CE174E080E69AE098D6C6013D
:10C0C000DCDCE8E3F4E029898191882339F0909160
:10C0D000C00095FFFCCF8093C600F6CF2223A9F0C5
:10C0E0004AE050E0B80180E69AE0E6D669E474E000
:10C0F00080E69AE07CD6C601C0DC8091C00085FF56
:10C10000FCCF8AE08093C60021E0F8944AEA55E526
:10C11000BA014093FC1F5093FD1F6093FE1F709364
:10C12000FF1F222311F082E001C080E0B82AB09204
:10C13000FB1F1093F91F0093F81FC092F41FD092B9
:10C14000F51FE092F61FF092F71FCE010196AA2785
:10C1500097FDA095BA2F8093F01F9093F11FA093A5
:10C16000F21FB093F31F28E088E190E00FB6F89437
:10C17000A895809360000FBE20936000FFCF809150
:10C18000C00085FFFCCFB092C60040E1942E9C0C0D
:10C19000FFEFCF1ADF0AEF0AFF0AC6010197AA27AD
:10C1A00097FDA095BA2FABBFFC0187919091C0007D
:10C1B00095FFFCCFB092C60057DC0150110971F415
:10C1C0008091C00085FFFCCFA092C600011511052B
:10C1D00041F08E2D3DDCC60150DCD1CF9C10D8CF74
:10C1E000EFCF61960FB6F894DEBF0FBECDBFDF91E3
:10C1F000CF911F910F91FF90EF90DF90CF90BF9064
:10C20000AF909F900895F8948AEA95E5DC018093B9
:10C21000FC1F9093FD1FA093FE1FB093FF1F87E0AC
:10C220008093FB1F80E09CE09093F91F8093F81FA0
:10C2300080E094EEA3E0B0E08093F01F9093F11FB4
:10C24000A093F21FB093F31F80E094EFA3E0B0E05F
:10C250008093F41F9093F51FA093F61FB093F71FE0
:10C2600028E088E190E00FB6F894A89580936000EC
:10C270000FBE20936000FFCF08950895CF9365E728
:10C2800074E080E69AE0B3D5E091E810F091E9100F
:10C2900085818F3311F0811170C0E5E8F4E0819160
:10C2A000882339F09091C00095FFFCCF8093C600A1
:10C2B000F6CF4AE050E06091F11380E69AE0E9D5CC
:10C2C000ECE8F4E08191882339F09091C00095FF6B
:10C2D000FCCF8093C600F6CF4AE050E06091F013A7
:10C2E00080E69AE0D6D5E4E9F4E08191882339F03C
:10C2F0009091C00095FFFCCF8093C600F6CF60916F
:10C30000EE137091EF134AE050E080E69AE07CD59E
:10C31000E8E9F4E08191882339F09091C00095FF1D
:10C32000FCCF8093C600F6CF6091EC137091ED13B3
:10C330004AE050E080E69AE067D5ECE9F4E08191CC
:10C34000882339F09091C00095FFFCCF8093C60000
:10C35000F6CF4AE050E06091EB1380E69AE099D581
:10C36000E0EAF4E08191882309F455C09091C0007F
:10C3700095FFFCCF8093C600F5CF813209F053C002
:10C380000F94E321E5E9F4E08191882339F090915D
:10C39000C00095FFFCCF8093C600F6CF6091EE13EE
:10C3A0007091EF134AE050E080E69AE02DD5E8E97D
:10C3B000F4E08191882339F09091C00095FFFCCF83
:10C3C0008093C600F6CF6091EC137091ED134AE0B4
:10C3D00050E080E69AE018D5ECE9F4E081918823FA
:10C3E00039F09091C00095FFFCCF8093C600F6CF46
:10C3F0004AE050E06091EB1380E69AE04AD5E0EA2B
:10C40000F4E08191882339F09091C00095FFFCCF32
:10C410008093C600F6CF4AE050E06091EA1380E6D0
:10C420009AE0CF913CC582E5F4DA882361F107DB1D
:10C430000F94E2D7C62FE4EAF4E08191882339F023
:10C440009091C00095FFFCCF8093C600F6CF4AE0E4
:10C4500050E06C2F80E69AE01CD5ECEBF4E0819183
:10C46000882339F09091C00095FFFCCF8093C600DF
:10C47000F6CF6C2F8C2F0F946F224AE050E0BC0156
:10C4800080E69AE0C8D488E5C4DA8823E1F0D7DAF8
:10C490000F94E2D77093EF136093EE13EFEBF4E099
:10C4A0008191882339F09091C00095FFFCCF809353
:10C4B000C600F6CF6091EE137091EF134AE050E0A2
:10C4C00080E69AE0A1D489E5A4DA8823E9F0B7DA16
:10C4D0000F94E2D77093ED136093EC13EAECF4E061
:10C4E0008191882339F09091C00095FFFCCF809313
:10C4F000C600F6CF6091EC137091ED134AE050E066
:10C5000080E69AE0CF9180C4CF910895CF93DF93D6
:10C51000EC0160E08E810F94CAD081E090E00F942E
:10C520000CCF61E08E810F94CAD081E090E00F942F
:10C530000CCF60E08E810F94CAD084E690E0DF914A
:10C54000CF910D940CCFCF92DF92EF92FF920F9389
:10C550001F93CF93DF937C01C0E0D0E0C62ED12C97
:10C5600087010C0F1D1F61E0F80187810F9491D0A6
:10C57000B6010C2E02C0759567950A94E2F76170BA
:10C58000F80187810F94CAD02196C430D10541F7B4
:10C59000C701DF91CF911F910F91FF90EF90DF9036
:10C5A000CF90B4CFCF92DF92EF92FF920F931F9371
:10C5B000CF93DF937C01C0E0D0E0C62ED12C870161
:10C5C0000C0F1D1F61E0F80187810F9491D0B60117
:10C5D0000C2E02C0759567950A94E2F76170F80118
:10C5E00087810F94CAD02196C830D10541F7C70181
:10C5F000DF91CF911F910F91FF90EF90DF90CF903F
:10C6000085CF1F93CF93DF93EC01162F642F8C817E
:10C610000F94CAD08D818F3F19F060E00F94CAD07B
:10C620008F85612F84FF05C0CE01DF91CF911F91CF
:10C63000B9CF70E084E0759567958A95E1F7CE01F2
:10C6400082DF612FCE01DF91CF911F917CCF40E03F
:10C65000D8CF61E0FCDF80E496E00D940CCF62E07F
:10C66000F6DF80E496E00D940CCFCF93DF93CDB747
:10C67000DEB728970FB6F894DEBF0FBECDBF28E017
:10C68000EBE0F3E0DE01119601900D922A95E1F7BF
:10C69000FC012389421710F04FEF420FFE01319643
:10C6A000E40FF11DE40FF11D2081260F2068622F99
:10C6B00028960FB6F894DEBF0FBECDBFDF91CF91A5
:10C6C000C6CFFC016089262F2460208B6C60BFCF11
:10C6D000CF93DF93EC01423018F08F8588608F870D
:10C6E0004B8B1C8A222329F0413019F48F858460FA
:10C6F0008F8780E593EC0F940CCF60E08C810F94D2
:10C70000CAD060E08E810F94CAD08D818F3F19F01E
:10C7100060E00F94CAD06F8564FD19C063E0CE015C
:10C7200012DF84E991E10F940CCF63E0CE010BDFBF
:10C7300084E991E10F940CCF63E0CE0104DF86E938
:10C7400090E00F940CCF62E0CE01FDDE13C060627A
:10C75000CE017DDF84E991E10F940CCF6F8560629B
:10C76000CE0175DF86E990E00F940CCF6F85606293
:10C77000CE016DDF6F856062CE0169DF8CE390E0F2
:10C780000F940CCF84E0888BCE019BDF8CE390E08C
:10C790000F940CCFCE015DDF88EB9BE00F940CCFA4
:10C7A00082E0898B66E0CE0152DF8CE390E0DF917E
:10C7B000CF910D940CCF6F927F928F92AF92CF92C8
:10C7C000EF920F931F93CF93DF93CDB7DEB73C016A
:10C7D000162F842F5E854F8538899989F3018483CC
:10C7E00025830683E782C086A18682865387448795
:10C7F0003587968761E00F9491D0F30185818F3F53
:10C8000019F061E00F9491D061E0F30186810F94FB
:10C8100091D0112319F0F301178603C080E1F301D1
:10C82000878720E041E060E1C301DF91CF911F9154
:10C830000F91EF90CF90AF908F907F906F9048CFF7
:10C840008F92AF92CF92EF920F93DC0113961C92CE
:10C850001E921297E9EDF4E0ED93FC931F921F9264
:10C860001F921F928C2CAE2CC02EE22E042F2FEF85
:10C87000462F61E0A0DF0F900F900F900F900F9167
:10C88000EF90CF90AF908F900895CF93DF93EC010E
:10C89000423018F08F8588608F874B8B1C8A22234B
:10C8A00029F0413019F48F8584608F8780E593ECFF
:10C8B0000F940CCF60E08C810F94CAD060E08E8121
:10C8C0000F94CAD08D818F3F19F060E00F94CAD0C9
:10C8D0006F8564FD19C063E0CE0135DE84E991E126
:10C8E0000F940CCF63E0CE012EDE84E991E10F942A
:10C8F0000CCF63E0CE0127DE86E990E00F940CCFE9
:10C9000062E0CE0120DE13C06062CE01A0DE84E9C9
:10C9100091E10F940CCF6F856062CE0198DE86E9BD
:10C9200090E00F940CCF6F856062CE0190DE6F8532
:10C930006062CE018CDE8CE390E00F940CCF84E03B
:10C94000888BCE01BEDE8CE390E00F940CCFCE013D
:10C9500086DE80E496E00F940CCF82E0898B66E05F
:10C96000CE0175DE8CE390E00F940CCF40E068E0E0
:10C97000CE017BDE6DEA79E0CE010F9465D141E016
:10C9800068E0CE0172DE6DEA79E0CE010F9465D1E8
:10C9900042E066E0CE0169DE6BEA79E0CE01DF912C
:10C9A000CF910D9465D1CF92DF92EF92FF920F93CA
:10C9B0001F93CF93DF931F921F92CDB7DEB78C01E9
:10C9C000677088E0689FB00111246064C8014983E2
:10C9D0005A833DDE4981C42E5A81D52EE12CF12C9B
:10C9E000D6016D916D01D801ED91FC910190F0811E
:10C9F000E02DC8011995BFEFEB1AFB0AE8E0EE162F
:10CA0000F10471F70F900F90DF91CF911F910F916B
:10CA1000FF90EF90DF90CF90089541E0F2DD81E04C
:10CA200090E008951F920F920FB60F9211240BB64B
:10CA30000F922F933F934F935F936F938F939F9397
:10CA4000EF93FF938091C00084FF03C08091C600E4
:10CA500019C06091C6002091E10A3091E20AC90133
:10CA600001968F7799274091E30A5091E40A841741
:10CA7000950741F0F901EF59F54F60839093E20A71
:10CA80008093E10AFF91EF919F918F916F915F9158
:10CA90004F913F912F910F900BBE0F900FBE0F90B3
:10CAA0001F9018951F920F920FB60F9211240BB67C
:10CAB0000F922F933F934F935F936F938F939F9317
:10CAC000EF93FF938091E50A813001F58091D000CA
:10CAD00084FF03C08091D60019C06091D6002091D8
:10CAE000E10A3091E20AC90101968F7799274091B6
:10CAF000E30A5091E40A8417950741F0F901EF59D0
:10CB0000F54F60839093E20A8093E10AFF91EF91E1
:10CB10009F918F916F915F914F913F912F910F90C6
:10CB20000BBE0F900FBE0F901F901895CF92DF9203
:10CB3000EF92FF926A017B01411581EE5807610572
:10CB4000710509F463C082E08093C00060E079E081
:10CB50008DE390E0A70196010F946CDC2150310920
:10CB600041095109CA01B90122E030E040E050E03A
:10CB70000F946CDC91E03093C5002093C400809149
:10CB8000C10080618093C1008091C1008860809362
:10CB9000C1008091C10080688093C1008091E50A46
:10CBA0008130D1F5992341F082E08093D00060E09C
:10CBB00079E08DE390E006C01092D00060E874E860
:10CBC0008EE190E0A70196010F946CDC21503109B1
:10CBD00041095109CA01B90122E030E040E050E0CA
:10CBE0000F946CDC3093D5002093D4008091D10059
:10CBF00080618093D1008091D10088608093D100C2
:10CC00008091D10080688093D10006C01092C0004E
:10CC100090E020E130E0AFCFFF90EF90DF90CF9039
:10CC200008952091E30A3091E40A8091E10A9091FD
:10CC3000E20A8217930771F0F901EF59F54F8081ED
:10CC40002F5F3F4F2F7733273093E40A2093E30A77
:10CC500090E008958FEF9FEF08958091E30A9091FF
:10CC6000E40A9093E20A8093E10A08954F925F925A
:10CC70006F927F928F929F92AF92BF92CF92DF92EC
:10CC8000EF92FF920F931F93CF93DF93CDB7DEB751
:10CC9000A0970FB6F894DEBF0FBECDBF5C01411563
:10CCA000510561057105E9F420E030E040E350E012
:10CCB00060E070E0A0960FB6F894DEBF0FBECDBF67
:10CCC000DF91CF911F910F91FF90EF90DF90CF9068
:10CCD000BF90AF909F908F907F906F905F904F909C
:10CCE0005BC08E010F5F1F4FC12CD12C7601480114
:10CCF000422E512C612C712C8FEFC81AD80AE80AE9
:10CD0000F80ACB01BA01A30192010F944ADCCA01CF
:10CD1000F80161938F01A901BC014115510561051D
:10CD2000710551F7F1E0CF1AD108E108F108F401DB
:10CD3000EC0DFD1D80818A3010F440E301C047E313
:10CD4000480F552747FD5095652F752F20E030E09F
:10CD5000C50122D081E0C81AD108E108F108EFEF3F
:10CD6000CE16DE06EE06FE0611F7A0960FB6F89474
:10CD7000DEBF0FBECDBFDF91CF911F910F91FF900E
:10CD8000EF90DF90CF90BF90AF909F908F907F906B
:10CD90006F905F904F9008952115310539F480917F
:10CDA000C00085FFFCCF4093C60008952A303105AE
:10CDB00009F43FC05BCF9A01462F552747FD509598
:10CDC000652F752FE9CFCF93DF93EC0120E030E0A2
:10CDD0004DE050E060E070E0DFDF20E030E04AE06E
:10CDE00050E060E070E0CE01DF91CF91D5CFFB0144
:10CDF0002191BF01222339F03091C00035FFFCCFD3
:10CE00002093C600F4CFDFCF9A01AB01662757FD10
:10CE10006095762FC1CFCF93DF93EC019A01AB01E0
:10CE2000662757FD6095762FB7DFCE01DF91CF9152
:10CE3000CACFCF92DF92EF92FF92CF93DF93EC01B4
:10CE40006A017B0177FF0FC020E030E04DE250E047
:10CE500060E070E0A1DFF094E094D094C094C11C35
:10CE6000D11CE11CF11C2AE0B701A601CE01DF9123
:10CE7000CF91FF90EF90DF90CF90F8CE2115310544
:10CE800039F48091C00085FFFCCF4093C60008951F
:10CE9000EDCE9A01462F50E060E070E0EFCFCF93E7
:10CEA000DF93EC019A01462F50E060E070E0E6DF8E
:10CEB000CE01DF91CF9187CF9A01AB0160E070E0A6
:10CEC000DDCFCF93DF93EC019A01AB0160E070E01E
:10CED000D5DFCE01DF91CF9176CFCF93DF93EC01F9
:10CEE000CDDFCE01DF91CF916ECF8F929F92AF9227
:10CEF000BF92CF92DF92EF92FF921F93CF93DF9377
:10CF0000EC016A017B01122F20E030E0A901C7018A
:10CF1000B6010F9473D787FF0CC020E030E04DE2DC
:10CF200050E060E070E0CE0137DFF7FAF094F7F8F8
:10CF3000F094B12C60E070E080E09FE3B11641F026
:10CF400020E030E040E251E40F947AD7B394F6CF7A
:10CF50009B01AC01C701B6010F949AD66B017C010D
:10CF60000F94E7D74B015C010F9413D89B01AC01E0
:10CF7000C701B6010F9499D66B017C012AE0B50177
:10CF8000A401CE0173DE112361F0E8E1F7E08191A5
:10CF9000882339F09091C00095FFFCCF8093C600A4
:10CFA000F6CF112319F120E030E040E251E4C7014F
:10CFB000B6010F9448DA6B017C010F94E2D74B0164
:10CFC000AA2497FCA094BA2CB501A401CE0131DFAC
:10CFD000C501B4010F9415D89B01AC01C701B6017E
:10CFE0000F9499D66B017C011150DBCFDF91CF916B
:10CFF0001F91FF90EF90DF90CF90BF90AF909F90E8
:10D000008F90089572CFCF93DF93EC016EDFCE0146
:10D01000DF91CF91D8CEFC01659175918591949166
:10D020000895EF92FF920F931F93CF93DF93EC013C
:10D03000CC0FDD1FCC0FDD1FCE018252914FEBDFF5
:10D040009E012A55344F79018E010656144FF8017E
:10D0500020813181428153810F949AD6F7016083F8
:10D06000718382839383CE018A50914FD4DF9E01D6
:10D07000235D3D4F7901F801208131814281538147
:10D080000F949AD6F7016083718382839383CE01D4
:10D090008651914FC0DFCF5DDD4FF8012081318196
:10D0A000428153810F949AD6688379838A839B83C4
:10D0B000DF91CF911F910F91FF90EF900895CF9343
:10D0C000C82F40910C0250910D0260910E02709198
:10D0D0000F0240935D0B50935E0B60935F0B709358
:10D0E000600B20914F02309150023093100C20932E
:10D0F0000F0C24E630E03093500220934F020F943F
:10D10000A6CE6093580B7093590B80935A0B909353
:10D110005B0B8C2FCF910D94EC3780E00F94EC37A4
:10D1200080915D0B90915E0BA0915F0BB091600BB5
:10D1300080930C0290930D02A0930E02B0930F0205
:10D1400080910F0C9091100C9093500280934F029D
:10D150000F94A6CE6093580B7093590B80935A0B83
:10D1600090935B0B0895682F772767FD70958091EA
:10D17000F2109091F31089509F4E0F943AE09093E3
:10D18000E9108093E81021E0892B09F420E0822F38
:10D1900008958091E8109091E9104AE050E060E035
:10D1A00070E001960F944BDECB0108958091E8105A
:10D1B0009091E9104AE050E060E070E001960D9433
:10D1C0004BDE2091F2103091F310BC01C90189505F
:10D1D0009F4E0F9472E09093E9108093E81021E045
:10D1E000892B09F420E0822F08950F931F93CF938A
:10D1F000DF930091E8101091E91065E470E0C80138
:10D200000F943AE0EC01009751F460E070E0C8013F
:10D210000196DF91CF911F910F910D94E3DC18825D
:10D220008091E8109091E91060E070E001960F9411
:10D23000E3DC25E42883DF91CF911F910F910895BE
:10D240008091E8109091E91060E070E001960D94F3
:10D25000E3DC2F923F924F925F926F927F928F9278
:10D260009F92AF92BF92CF92DF92EF92FF920F9375
:10D270001F93CF93DF93CDB7DEB760970FB6F894C7
:10D28000DEBF0FBECDBF1C012A013B014801590181
:10D2900020E030E04CE052E4C301B2010F9499D693
:10D2A00025E535E547E052E40F947AD76B017C0120
:10D2B0000F9450D80F94E2D78B0177FF12C020E073
:10D2C00030E040E85FE3C701B6010F9476D9181645
:10D2D0000CF05DC0C12CD12CE0E8EE2EEFE3FE2E69
:10D2E00056C066307105DCF02AEA3AE24CE453E4B9
:10D2F000C301B2010F9499D625E535E547E052E424
:10D300000F947AD76B017C0120E030E0A9010F94E3
:10D3100073D787FF3FC0C12CD12C76013BC0882733
:10D3200077FD8095982F0F9415D825E535E547E0D2
:10D3300052E40F9448DA20E030E04CE052E40F94DD
:10D340009AD69B01AC01C301B2010F9499D625E591
:10D3500035E547E052E40F947AD76B017C0120E079
:10D3600030E0A9010F9473D787FD17C020E030E0AB
:10D3700040E85FE3C701B6010F9476D9181684F42C
:10D38000C12CD12C70E8E72E7FE3F72E09C000E016
:10D3900010E006C005E010E003C0C12CD12C7601DE
:10D3A00020E030E040EC50E4C501B4010F9499D680
:10D3B0002BEA3AEA42E052E40F947AD72B013C017F
:10D3C0000F9450D80F94E2D7788B6F8777FF12C0F5
:10D3D00020E030E040E85FE3C301B2010F9476D96A
:10D3E00018160CF05FC0412C512C60E8662E6FE3DC
:10D3F000762E58C0AF85B8891697E4F026E535E556
:10D4000049E253E4C501B4010F9499D62BEA3AEAF4
:10D4100042E052E40F947AD72B013C0120E030E047
:10D42000A9010F9473D787FD40C0E5E0F0E0F88BC9
:10D43000EF8746C0882777FD8095982F0F9415D8E1
:10D440002BEA3AEA42E052E40F9448DA20E030E076
:10D4500040EC50E40F949AD69B01AC01C501B40195
:10D460000F9499D62BEA3AEA42E052E40F947AD725
:10D470002B013C0120E030E0A9010F9473D787FD18
:10D480001CC020E030E040E85FE3C301B2010F942C
:10D4900076D91816ACF4412C512C50E8652E5FE378
:10D4A000752E0EC0188A1F860BC0412C512C3201DC
:10D4B00025E030E0388B2F8703C0412C512C3201FE
:10D4C000A701960160E070E080E89FE30F9499D691
:10D4D00069837A838B839C83C80101969E838D83A5
:10D4E000AF85B8891196BA87A987A301920160E038
:10D4F00070E080E89FE30F9499D66B877C878D87D7
:10D500009E8747E02F853889429FF001439FF00DA9
:10D510001124F887EF83E00FF11FEE0FFF1FEE0FCE
:10D52000FF1FE20DF31D2181328143815481698106
:10D530007A818B819C810F9448DA4B015C01EF81E9
:10D54000F8858D819E81E80FF91FEE0FFF1FEE0F0A
:10D55000FF1FE20DF31D2181328143815481C701F8
:10D56000B6010F9448DA9B01AC01C501B4010F94D8
:10D570009AD69B01AC016B857C858D859E850F9429
:10D5800048DA4B015C0127E0E985FA852E9FD0013E
:10D590002F9FB00D1124B887AF83FD01E00FF11F5D
:10D5A000EE0FFF1FEE0FFF1FE20DF31D21813281F1
:10D5B0004381548169817A818B819C810F9448DAFF
:10D5C00069837A838B839C83AF81B8858D819E81AB
:10D5D000A80FB91FAA0FBB1FAA0FBB1FA20DB31D17
:10D5E00011962D913D914D915C911497C701B60113
:10D5F0000F9448DA9B01AC0169817A818B819C810F
:10D600000F949AD69B01AC01C301B2010F9448DA82
:10D610009B01AC01C501B4010F949AD660960FB678
:10D62000F894DEBF0FBECDBFDF91CF911F910F9158
:10D63000FF90EF90DF90CF90BF90AF909F908F9032
:10D640007F906F905F904F903F902F9008954F92F2
:10D650005F926F927F929F92AF92BF92CF92DF9232
:10D66000EF92FF920F931F93CF93DF937C015B01A7
:10D670008A01E90190902413911014C0FC0180816B
:10D680009181A281B381FA0180839183A283B383C4
:10D69000FB0180819181A281B38188839983AA83D0
:10D6A000BB837FC091FE55C0FC0120813181428146
:10D6B00053816091141370911513809116139091FA
:10D6C00017130F9448DA2B013C01F50120813181B9
:10D6D00042815381609118137091191380911A132C
:10D6E00090911B130F9448DA9B01AC01C301B20166
:10D6F0000F949AD6F8016083718382839383F70134
:10D70000208131814281538160911C1370911D13DE
:10D7100080911E1390911F130F9448DA6B017C01C6
:10D72000F5012081318142815381609120137091F4
:10D73000211380912213909123130F9448DA9B01B7
:10D74000AC01C701B6010F949AD6688379838A83A6
:10D750009B8390FE26C02091FC123091FD124091D7
:10D76000FE125091FF12F8016081718182819381D4
:10D770000F949AD6F80160837183828393832091FA
:10D7800000133091011340910213509103136881EB
:10D7900079818A819B810F949AD6688379838A8361
:10D7A0009B83DF91CF911F910F91FF90EF90DF90BE
:10D7B000CF90BF90AF909F907F906F905F904F9071
:10D7C00008952F923F924F925F926F927F928F9225
:10D7D0009F92AF92BF92CF92DF92EF92FF920F9300
:10D7E0001F93CF93DF93CDB7DEB728970FB6F8948A
:10D7F000DEBF0FBECDBF8C011B019E012F5F3F4FCF
:10D80000AE014B5F5F4F23DF20E030E0A9016D8167
:10D810007E818F8198850F9473D787FF07C01D8203
:10D820001E821F821886FF24F39401C0F12C20E091
:10D8300030E040E451EC69817A818B819C810F94C6
:10D8400073D787FF0AC080E090E0A0E4B1EC898341
:10D850009A83AB83BC83FF24F39420E030E04AE753
:10D8600053E46D817E818F8198850F9476D9181647
:10D8700054F480E090E0AAE7B3E48D839E83AF8305
:10D88000B887FF24F39420E030E042E553E4698157
:10D890007A818B819C810F9476D918164CF480E0A4
:10D8A00090E0A2E5B3E489839A83AB83BC8303C091
:10D8B000FF2009F483C0C980DA80EB80FC808D8072
:10D8C0009E80AF80B8847090241371100BC0F80153
:10D8D00080829182A282B382F101C082D182E282EF
:10D8E000F3826AC070FE1CC02091FC123091FD12C0
:10D8F0004091FE125091FF12C501B4010F9499D6C8
:10D900004B015C01209100133091011340910213EF
:10D9100050910313C701B6010F9499D66B017C0196
:10D9200071FE4AC0209104133091051340910613F3
:10D9300050910713C501B4010F9448DA2B013C0143
:10D94000209108133091091340910A1350910B1341
:10D95000C701B6010F9448DA9B01AC01C301B201C3
:10D960000F949AD6F8016083718382839383209108
:10D970000C1330910D1340910E1350910F13C501EC
:10D98000B4010F9448DA4B015C01209110133091DF
:10D9900011134091121350911313C701B6010F9444
:10D9A00048DA9B01AC01C501B4010F949AD6F1018C
:10D9B0006083718382839383FF24F3948F2D289651
:10D9C0000FB6F894DEBF0FBECDBFDF91CF911F9190
:10D9D0000F91FF90EF90DF90CF90BF90AF909F900E
:10D9E0008F907F906F905F904F903F902F90089511
:10D9F000682F87EF9FE00D94F8E20895FC012491D1
:10DA0000222341F03091C00035FFFCCF2093C600A7
:10DA10000196F4CF22E030E080E69AE0F3CAFC0100
:10DA20002491222341F03091C00035FFFCCF209398
:10DA3000C6000196F4CF2AE030E080E69AE01ECAE4
:10DA4000CF936DED74E080E69AE0D1D9C1E0C09348
:10DA5000AA026FEF89E69FE00F94F8E2C093D70225
:10DA6000CF9108956DEE74E080E69AE0C0D91092EF
:10DA7000AA0260E089E69FE00F94F8E21092D702D4
:10DA80000895EF92FF920F931F93CF93DF931F920E
:10DA9000CDB7DEB789830F94EC708981823009F4A9
:10DAA00068C0B4F5882309F442C0813009F0F4C09D
:10DAB0009FB7F894809102018460809302019FBF18
:10DAC000EFEFF1EE24E0E150F0402040E1F700C03C
:10DAD00000009FB7F894809102018B7F8093020130
:10DAE0009FBF40E050E0BA018DEE9FE00F940AE343
:10DAF00040E050E0BA0181EF9FE00F940AE30F90FD
:10DB0000DF91CF911F910F91FF90EF900D94A7900F
:10DB1000833009F45CC0843009F0BEC00F90DF91FF
:10DB2000CF911F910F91FF90EF900D9481BC9FB703
:10DB3000F894809102018460809302019FBF2FEFCF
:10DB400081EE94E0215080409040E1F700C0000059
:10DB50009FB7F894809102018B7F809302019FBF51
:10DB60000F90DF91CF911F910F91FF90EF900D9447
:10DB700096710F94967180EF3BDF10922F1C1092DC
:10DB80002E1C6091301C84EC9FE00F94F8E26EE252
:10DB90007CE181EC9FE00F941A719FB7F89480911B
:10DBA00002018460809302019FBF8FEF91EEE4E059
:10DBB00081509040E040E1F700C000009FB7F8942A
:10DBC000809102018B7F809302019FBF65C085EB2E
:10DBD0009EE00F948A8344EA5EE062E081E00F9465
:10DBE0009F989FB7F894809102018460809302010E
:10DBF0009FBFFFEF21EE84E0F15020408040E1F72D
:10DC000000C000009FB7F894809102018B7F809341
:10DC100002019FBF1092440B1092430B4DE95EE04E
:10DC200063E083E00F949F984091430B5091440B25
:10DC300063E083E00F94F770E12CF12C09E210E02F
:10DC40006FEFC7010F9416E3C701B8010F9437DCDB
:10DC5000892BD9F48091430B9091440B01969093BA
:10DC6000440B8093430B46E95EE063E083E00F944E
:10DC70009F984091430B5091440B63E083E00F94D5
:10DC8000F77084E99EE00F948A839FEFE91AF90AFE
:10DC9000E114E0E1FE06A1F60F90DF91CF911F9114
:10DCA0000F91FF90EF90089580E1E6EAFBE0A1E795
:10DCB000BBE001900D928A95E1F708954F925F9233
:10DCC0006F927F928F929F92AF92BF92CF92DF928C
:10DCD000EF92FF92CF93DF9300D01F92CDB7DEB7C4
:10DCE0000F945F418BE43FDA882391F07EDA6B0179
:10DCF0007C0120E030E0A9010F9476D987FD08C0AF
:10DD0000C0920D14D0920E14E0920F14F0921014E1
:10DD100082E529DA882359F068DA6B017C0120E07A
:10DD200030E0A9010F9473D787FF83C006C0C12CD0
:10DD3000D12C60E8E62E6FEBF62E84E414DA88230B
:10DD400021F053DA4B015C0106C0812C912C50E884
:10DD5000A52E5FEBB52E87E506DA882321F045DA9C
:10DD60002B013C0106C0412C512C40E8642E4FEBA6
:10DD7000742E88E4F8D9882331F037DA69837A83FE
:10DD80008B839C8308C080E090E0A0E8BFEB898390
:10DD90009A83AB83BC8320E030E0A901C501B401C4
:10DDA0000F9476D987FD45C020E030E0A901C3017A
:10DDB000B2010F9476D987FD3CC020E030E0A90184
:10DDC00069817A818B819C810F9476D987FD31C0DE
:10DDD00020E030E0A901C501B4010F9473D7882376
:10DDE00091F120E030E040E05FE3C501B4010F9421
:10DDF00048DA6B017C0129813A814B815C81C30146
:10DE0000B2010F9448DA4B015C01A7019601C701EA
:10DE1000B6010F9448DA2BED3FE049E450E40F944B
:10DE200048DA9B01AC01C501B4010F947AD76B01AC
:10DE30007C0120E030E0A901C701B6010F9476D93A
:10DE400087FF04C00BC0C12CD12C7601C0920914ED
:10DE5000D0920A14E0920B14F0920C14E2E0FFE06E
:10DE60008491882341F09091C00095FFFCCF80936E
:10DE7000C6003196F5CFE2E7FAE08491882341F0BD
:10DE80009091C00095FFFCCF8093C6003196F5CFEE
:10DE900040910D1450910E1460910F147091101454
:10DEA00022E030E080E69AE0ADD88091C00085FFA6
:10DEB000FCCF8AE08093C600ECE6FAE084918823E8
:10DEC00041F09091C00095FFFCCF8093C600319641
:10DED000F5CFC0900914D0900A14E0900B14F09084
:10DEE0000C1420E030E0A901C701B6010F9473D7EC
:10DEF000882361F022E030E0B701A60180E69AE0D5
:10DF000081D88091C00085FFFCCF11C0E7E6FAE020
:10DF10008491882341F09091C00095FFFCCF8093BD
:10DF2000C6003196F5CF8091C00085FFFCCF8AE016
:10DF30008093C6000F900F900F900F90DF91CF91BC
:10DF4000FF90EF90DF90CF90BF90AF909F908F9019
:10DF50007F906F905F904F9008952F923F924F92D5
:10DF60005F926F927F928F929F92AF92BF92CF9269
:10DF7000DF92EF92FF920F931F93CF93DF931F9245
:10DF8000CDB7DEB70F94EC70E6EAFCE8459154910A
:10DF900061E080E00F949F9881E00F94EC378983D3
:10DFA000E5ECFEE0E4918E2F992781950CF4909595
:10DFB0001C0184E00F94A45CAEEABBE01D921D92AC
:10DFC0001D921C921397EAEAFBE020813181428185
:10DFD0005381A6EABBE06D917D918D919C91E2EB1E
:10DFE000CE2EEBE0DE2EE12CF12C87010F947E3457
:10DFF0005BDE8AED9EE00FD82DEC3CEC4CE85FE355
:10E000000F9448DA4B015C01B101882777FD8095B8
:10E01000982F0F9415D89B01AC01C501B4010F9442
:10E0200048DAE9E7FBE020813181428153810F9496
:10E030009AD62B013C01A9E7BBE06D937D938D93AC
:10E040009C931397E9E5F2E060817181828193816D
:10E0500060930C0270930D0280930E0290930F0256
:10E0600020E030E040E752E40F947AD74B015C01A6
:10E07000A5E7BBE02D913D914D915C91E1E7FBE07F
:10E080006081718182819381A2E9BBE0BF93AF93EC
:10E09000FDE7CF2EFBE0DF2E830172010F94D02726
:10E0A00082E00F94195A0F945F410F94245D80E031
:10E0B0000F94EC37AEEABBE01D921D921D921C92AC
:10E0C0001397EAEAFBE02081318142815381A6EA7D
:10E0D000BBE06D917D918D919C91A2EBCA2EABE03E
:10E0E000DA2EE12CF12C87010F947E34DDDD8AE0FD
:10E0F000829DB001839D700D1124882777FD809546
:10E10000982F0F9415D8E9E7FBE0208131814281F7
:10E1100053810F949AD62B013C01A9E7BBE06D9384
:10E120007D938D939C93139720E030E040E05FE374
:10E13000E9E5F2E060817181828193810F9448DA90
:10E1400060930C0270930D0280930E0290930F0265
:10E1500020E030E040E752E40F947AD74B015C01B5
:10E16000A5E7BBE02D913D914D915C91E1E7FBE08E
:10E170006081718182819381A2E9BBE0BF93AF93FB
:10E18000BDE7CB2EBBE0DB2E830172010F94D027BD
:10E190000F945F4189810F94EC3780E090E0A4E513
:10E1A000B3E4EEEAFBE080839183A283B383AAEA1F
:10E1B000BBE02D913D914D915C91E6EAFBE06081E1
:10E1C00071818281938112EBC12E1BE0D12EE12C53
:10E1D000F12C04E513E40F947E3481E00F900F904E
:10E1E0000F900F900F90DF91CF911F910F91FF90A3
:10E1F000EF90DF90CF90BF90AF909F908F907F90E7
:10E200006F905F904F903F902F9008952F923F9284
:10E210004F925F926F927F928F929F92AF92BF9236
:10E22000CF92DF92EF92FF920F931F93CF93DF93E2
:10E23000CDB7DEB729970FB6F894DEBF0FBECDBFBE
:10E240003C0181E00F94EC378F8382E06816710403
:10E2500008F081C2F301ED53F14FE491D301AA0F0D
:10E26000BB1FAA0FBB1FBA83A983AF5ABD4FBE8382
:10E27000AD838D919D910D90BC91A02D80930C024A
:10E2800090930D02A0930E02B0930F0281E0062C32
:10E2900001C0880F0A94EAF70F94A45CE981FA811F
:10E2A000EA55F44FF987E8871082118212821382AF
:10E2B000E090AE0BF090AF0B0091B00B1091B10B52
:10E2C0002091AA0B3091AB0B4091AC0B5091AD0B50
:10E2D0006091A60B7091A70B8091A80B9091A90B50
:10E2E000E2EBCE2EEBE0DE2E0F947E34E981FA8154
:10E2F000EF58F44F2F0180E090E0A0E4B0E4808379
:10E300009183A283B38320E030E040E752E4609140
:10E310000C0270910D0280910E0290910F020F94E9
:10E320007AD74B015C01E090790BF0907A0B009169
:10E330007B0B10917C0B2091750B3091760B4091EB
:10E34000770B5091780B6091710B7091720B8091EB
:10E35000730B9091740BF2E92F2EFBE03F2E3F924E
:10E360002F92ADE7CA2EABE0DA2E0F94D0270F9490
:10E370005F410F94D43780E00F94EC37A885B985BE
:10E380001D921D921D921C921397E090AE0BF0907F
:10E39000AF0B0091B00B1091B10B2091AA0B3091F3
:10E3A000AB0B4091AC0B5091AD0B6091A60B7091F3
:10E3B000A70B8091A80B9091A90BB2EBCB2EBBE0E1
:10E3C000DB2E0F947E3480E090E0A0E8BFEBF201FA
:10E3D00080839183A283B38320E030E040E752E45E
:10E3E00060910C0270910D0280910E0290910F02CB
:10E3F0000F947AD74B015C01E090790BF0907A0B87
:10E4000000917B0B10917C0B2091750B3091760B5A
:10E410004091770B5091780B6091710B7091720B5A
:10E420008091730B9091740B3F922F92EDE7CE2E5B
:10E43000EBE0DE2E0F94D0270F945F4181E00F9424
:10E44000EC3789819A818E52914F0E940B682DEC96
:10E450003CEC4CE85FEB0F9448DAD2016D937D936E
:10E460008D939C93139720E030E040E752E4609155
:10E470000C0270910D0280910E0290910F020F9488
:10E480007AD74B015C01E090790BF0907A0B009108
:10E490007B0B10917C0B2091750B3091760B40918A
:10E4A000770B5091780B6091710B7091720B80918A
:10E4B000730B9091740B3F922F920F94D0270F946F
:10E4C0005F410F94D43780E00F94EC37E885F985ED
:10E4D0001082118212821382E090AE0BF090AF0B8B
:10E4E0000091B00B1091B10B2091AA0B3091AB0BA6
:10E4F0004091AC0B5091AD0B6091A60B7091A70BA6
:10E500008091A80B9091A90BF2EBCF2EFBE0DF2EB0
:10E510000F947E3480E090E0A0E2B1E4F2018083C9
:10E520009183A283B38320E030E040E752E460911E
:10E530000C0270910D0280910E0290910F020F94C7
:10E540007AD74B015C01E090790BF0907A0B009147
:10E550007B0B10917C0B2091750B3091760B4091C9
:10E56000770B5091780B6091710B7091720B8091C9
:10E57000730B9091740B3F922F92ADE7CA2EABE0D4
:10E58000DA2E0F94D0270F945F410F94D43781E097
:10E590000F94EC3780E090E0A0E7B1ECF2018083CB
:10E5A0009183A283B38320E030E040E05FE3AD815C
:10E5B000BE816D917D918D919C910F9448DA60930D
:10E5C0000C0270930D0280930E0290930F0220E0D4
:10E5D00030E040E752E40F947AD74B015C01E090C1
:10E5E000790BF0907A0B00917B0B10917C0B2091B2
:10E5F000750B3091760B4091770B5091780B6091B1
:10E60000710B7091720B8091730B9091740B3F9210
:10E610002F920F94D0270F945F41C3010E9411687D
:10E62000F301E956F44F81E080830F94245D0F9449
:10E63000D43780E00F94EC372AE037ED43E25FE314
:10E64000E885F98560817181828193810F9499D6E3
:10E65000A885B9856D937D938D939C931397E090D6
:10E66000AE0BF090AF0B0091B00B1091B10B20915D
:10E67000AA0B3091AB0B4091AC0B5091AD0B60915C
:10E68000A60B7091A70B8091A80B9091A90BB2EBF0
:10E69000CB2EBBE0DB2E0F947E342AE037ED43E235
:10E6A0005FE3E885F98560817181828193810F94B0
:10E6B0009AD6A885B9856D937D938D939C93139776
:10E6C000F20160837183828393832AE939E949E9FE
:10E6D0005EE360910C0270910D0280910E029091A8
:10E6E0000F020F9448DA20E030E040E752E40F9444
:10E6F0007AD74B015C01E090790BF0907A0B009196
:10E700007B0B10917C0B2091750B3091760B409117
:10E71000770B5091780B6091710B7091720B809117
:10E72000730B9091740B3F922F92EDE7CE2EEBE09E
:10E73000DE2E0F94D0270F945F4110920C0210929E
:10E740000D0210920E0210920F020FB6F894DEBF67
:10E750000FBECDBF62C192E06916710409F05DC1C0
:10E76000E5ECFEE074901092AE0B1092AF0B10929D
:10E77000B00B1092B10B2091AA0B3091AB0B4091D2
:10E78000AC0B5091AD0B6091A60B7091A70B8091D3
:10E79000A80B9091A90BF2EBCF2EFBE0DF2EE12C22
:10E7A000F12C87010F947E348AED9EE00E940B6865
:10E7B0004B015C01672D772767FD7095872F972F99
:10E7C0000F9415D82B013C0120E030E040EC5FE3D2
:10E7D000C501B4010F9448DAA30192010F9448DAFD
:10E7E00069837A838B839C836093790B70937A0B14
:10E7F00080937B0B90937C0B6091590270915A022D
:10E8000080915B0290915C0260930C0270930D0208
:10E8100080930E0290930F0220E030E040E752E434
:10E820000F947AD74B015C012091750B3091760BD8
:10E830004091770B5091780B6091710B7091720B36
:10E840008091730B9091740BA2E92A2EABE03A2EC3
:10E850003F922F92BDE7CB2EBBE0DB2EE980FA8002
:10E860000B811C810F94D0270F945F411092AE0B47
:10E870001092AF0B1092B00B1092B10B2091AA0B1B
:10E880003091AB0B4091AC0B5091AD0B6091A60B4E
:10E890007091A70B8091A80B9091A90B12EBC12E40
:10E8A0001BE0D12EE12CF12C87010F947E348EECED
:10E8B0009EE00E940B689058A30192010F9448DAE1
:10E8C00069837A838B839C836093790B70937A0B33
:10E8D00080937B0B90937C0B20E030E040E752E488
:10E8E00060910C0270910D0280910E0290910F02C6
:10E8F0000F947AD74B015C012091750B3091760B08
:10E900004091770B5091780B6091710B7091720B65
:10E910008091730B9091740B3F922F920DE7C02E54
:10E920000BE0D02EE980FA800B811C810F94D02758
:10E930000F945F418EEC9EE00E940B689B01AC013E
:10E940000F949AD6A30192010F9448DA2B013C014F
:10E950006093790B70937A0B80937B0B90937C0B75
:10E9600020E030E040E05FE36091590270915A028C
:10E9700080915B0290915C020F9448DA60930C02E4
:10E9800070930D0280930E0290930F0220E030E00E
:10E9900040E752E40F947AD74B015C012091750B4C
:10E9A0003091760B4091770B5091780B6091710B01
:10E9B0007091720B8091730B9091740B3F922F9218
:10E9C000830172010F94D0270F945F4182E090E0A1
:10E9D0000E9411688091AE0B9091AF0BA091B00B8B
:10E9E000B091B10B8093790B90937A0BA0937B0B32
:10E9F000B0937C0B10920C0210920D0210920E023A
:10EA000010920F020F94D43781E08093990B0F90EE
:10EA10000F900F900F900F900F908F8129960FB647
:10EA2000F894DEBF0FBECDBFDF91CF911F910F9144
:10EA3000FF90EF90DF90CF90BF90AF909F908F901E
:10EA40007F906F905F904F903F902F900D94EC3798
:10EA5000CF92DF92EF92FF920F931F9325D980E020
:10EA600090E0D4DB81E090E0D1DBE090AE0BF09061
:10EA7000AF0B0091B00B1091B10B2091AA0B30910C
:10EA8000AB0B4091AC0B5091AD0B6091A60B70910C
:10EA9000A70B8091A80B9091A90BF2EBCF2EFBE076
:10EAA000DF2E0F947E341F910F91FF90EF90DF9037
:10EAB000CF900D94D4370F94A6CE6093580B7093DB
:10EAC000590B80935A0B90935B0B089520E030E034
:10EAD000A90168EB71E084E50F94F4D269E170E07C
:10EAE00080E090E00F94D5CE84E50F9418D664E1D1
:10EAF00070E080E090E00D94D5CE7F928F929F924F
:10EB0000AF92BF92CF92DF92EF92FF920F931F933B
:10EB1000CF93DF9300D01F92CDB7DEB71092261BA4
:10EB20001092251B1092241B1092231B0F94EC7043
:10EB30008BE99DE00F948A838E010F5F1F4F7E014A
:10EB400025E0E20EF11C80E69AE00E9411668F3FFC
:10EB5000EFEF9E07C1F3F80181938F01EE15FF05DA
:10EB600091F789809A80AB80BC808091C00085FF3E
:10EB7000FCCF8BE28093C600C12CD12C7601ABE296
:10EB80007A2E8091DA0B882309F450C002E01BE052
:10EB9000C814D904EA04FB04A1F080E69AE00E94BC
:10EBA00011668F3FFFEF9F07C1F32FEFC21AD20A02
:10EBB000E20AF20AF80181938F01FBE002341F0799
:10EBC00039F762E07BE089E19CE00E94F5DC80910E
:10EBD000C00085FFFCCF7092C6000F94BD52C814D0
:10EBE000D904EA04FB0469F671DF60E089E19CE086
:10EBF0000E9428DE1092DA0BE6EDFBE885919491F5
:10EC0000FC012491222341F03091C00035FFFCCF5C
:10EC10002093C6000196F4CF8091C00085FFFCCF01
:10EC20008AE08093C60080E090E000C00F900F90D3
:10EC30000F900F90DF91CF911F910F91FF90EF9068
:10EC4000DF90CF90BF90AF909F908F907F9008956E
:10EC50002F923F924F925F926F927F928F929F92EC
:10EC6000AF92BF92CF92DF92EF92FF920F931F93DA
:10EC7000CF93DF931F921F92CDB7DEB7382E81114D
:10EC800012C01092241B1092231B1092261B10926C
:10EC9000251B1092281B1092271B10922A1B1092E2
:10ECA000291B0F94417180E00F949BB485E293E19E
:10ECB0000F946B1C0E94D2FD0F94BC1B1092970BFB
:10ECC0001092980B1092990B81E00E945F68E0917E
:10ECD000DB0BF0E0EE0FFF1FEA51F24785919491B4
:10ECE000BE016F5F7F4F0F94DAB4B2DE36D988234E
:10ECF00009F465C1E0DE31103AC0E6EFF6E885912F
:10ED0000949140E060E00F9493B6882331F0EEEEEA
:10ED1000F8E8859194910F9477BEE091DB0BF0E0D9
:10ED2000EE0FFF1FE853F647859194910F9477BE3D
:10ED3000E091DB0BF0E0EE0FFF1FE254F44785910A
:10ED40009491BE016F5F7F4F0F94DAB441E050E0C1
:10ED500062E080E00F94F770E091DB0BF0E0EE0FE3
:10ED6000FF1FEE54F447859194910F948A8380E0BD
:10ED700090E0A0EAB0E48093AE0B9093AF0BA09329
:10ED8000B00BB093B10B20E030E040E252E4609170
:10ED9000590270915A0280915B0290915C020F942B
:10EDA0007AD74B015C012091AA0B3091AB0B4091BB
:10EDB000AC0B5091AD0B6091A60B7091A70B80919D
:10EDC000A80B9091A90BE2E9FBE0FF93EF93E2EB34
:10EDD000CE2EEBE0DE2EE12CF12C00EA10E40F94B5
:10EDE000D0270F945F4186E50E94B3680F900F9083
:10EDF000882361F0E091E810F091E9108181893079
:10EE000039F08F7D41F00E94C96803C01A8205C0A5
:10EE100081E08A8302C0A1E0AA833320B1F00E947E
:10EE20008D680E9427FE0F9443000F9417158823C6
:10EE300009F4C1C087EF9FE00F94E6E2803F09F03C
:10EE4000BAC081E00E94F86CB6C08FEF0E94F86CE7
:10EE500060E070E088EF9FE00F9412E31982BE013A
:10EE60006F5F7F4F8A810F94E8113C010E948D688B
:10EE7000212C312C10EA412E10E4512E2092AE0BA1
:10EE80003092AF0B4092B00B5092B10B20E030E0CB
:10EE900040E252E46091590270915A0280915B0203
:10EEA00090915C020F947AD74B015C012091AA0BE0
:10EEB0003091AB0B4091AC0B5091AD0B6091A60B18
:10EEC0007091A70B8091A80B9091A90BA2E9BBE0D0
:10EED000BF93AF9302EBC02E0BE0D02E82017101E5
:10EEE0000F94D0270F945F410F900F9077FC47C08D
:10EEF000198285E293E10F946B1C0E9499FD81E0D9
:10EF00000E945F68A5DDAE014F5F5F4F6A8181E0BF
:10EF10000F943D173C010E948D682092AE0B3092F9
:10EF2000AF0B4092B00B5092B10B20E030E040E2CA
:10EF300052E46091590270915A0280915B02909163
:10EF40005C020F947AD74B015C012091AA0B30919F
:10EF5000AB0B4091AC0B5091AD0B6091A60B709137
:10EF6000A70B8091A80B9091A90BA2E9BBE0BF93DE
:10EF7000AF930F94D0270F945F410F900F9069814A
:10EF8000C3010F94D5BE77FC16C086EE0E94F86CC4
:10EF90008FE59FE00F94E6E2813059F0E091DB0BC2
:10EFA000F0E0EE0FFF1FE453F247859194910F9428
:10EFB00077BE11E001C010E00F94245D01C010E0A5
:10EFC00081E00F949BB4812F0F900F90DF91CF9130
:10EFD0001F910F91FF90EF90DF90CF90BF90AF9077
:10EFE0009F908F907F906F905F904F903F902F9069
:10EFF00008958F929F92AF92BF92CF92DF92EF923D
:10F00000FF920F931F93CF93DF93159881E0809326
:10F01000CF0B82E090E09093CD0B8093CC0BE091EE
:10F02000DB0BF0E0EE0FFF1FEC51F547859194915B
:10F030000F94057220E030E04CE852E46091B20B8E
:10F040007091B30B8091B40B9091B50B0F949AD63D
:10F050006093B20B7093B30B8093B40B9093B50B8A
:10F06000E090AE0BF090AF0B0091B00B1091B10B94
:10F070002091AA0B3091AB0B4091AC0B5091AD0B92
:10F080006091A60B7091A70B8091A80B9091A90B92
:10F09000C2E9DBE0DF93CF93812C912CE0ECAE2E24
:10F0A000E0E4BE2EF2EBCF2EFBE0DF2E0F94D02754
:10F0B00020E030E048EC51E46091B20B7091B30B6A
:10F0C0008091B40B9091B50B0F949AD66093B20BCC
:10F0D0007093B30B8093B40B9093B50BE090AE0B91
:10F0E000F090AF0B0091B00B1091B10B2091AA0BD7
:10F0F0003091AB0B4091AC0B5091AD0B6091A60BD6
:10F100007091A70B8091A80B9091A90BDF93CF93DF
:10F11000812C912CA0E8AA2EAFE3BA2E0F94D02711
:10F120000F945F410F900F900F900F908091301CC3
:10F13000882331F181E00F949BB482E00F94D4B125
:10F14000E091DB0BF0E0EE0FFF1FEC5DFA478591DD
:10F1500094910F9405721092CE0B1092CF0B1092D7
:10F16000CD0B1092CC0BDF91CF911F910F91FF909F
:10F17000EF90DF90CF90BF90AF909F908F900895C9
:10F180008091CE0B8823B1F2E091DB0BF0E0EE0F23
:10F19000FF1FE652F4478591949141E060E00F949F
:10F1A00093B691E0811101C090E0C2E9DBE09111DA
:10F1B000C1CF81E00F949BB482E00F94D4B120E0E2
:10F1C00030E048EC51E46091B20B7091B30B809148
:10F1D000B40B9091B50B0F949AD66093B20B7093C9
:10F1E000B30B8093B40B9093B50BE090AE0BF09003
:10F1F000AF0B0091B00B1091B10B2091AA0B309185
:10F20000AB0B4091AC0B5091AD0B6091A60B709184
:10F21000A70B8091A80B9091A90BDF93CF93812C22
:10F22000912CE0E8AE2EEFE3BE2EF2EBCF2EFBE00A
:10F23000DF2E0F94D0270F945F41E091DB0BF0E0BD
:10F24000EE0FFF1FE652F4478591949141E060E094
:10F250000F9493B60F900F9081116CCFAACF0F949B
:10F26000A6CE6093580B7093590B80935A0B9093D2
:10F270005B0BE091F210F091F310EC50FF4E8081A7
:10F280008130B9F4E4EDF9E885919491FC01249181
:10F29000222341F03091C00035FFFCCF2093C600FF
:10F2A0000196F4CF8091C00085FFFCCF8AE0809367
:10F2B000C600089580E69AE00E942D66ECEEF8E81C
:10F2C00085919491FC012491222341F03091C0005A
:10F2D00035FFFCCF2093C6000196F4CF4091D810A3
:10F2E0005091D9106091DA107091DB104F5F5F4F31
:10F2F0006F4F7F4F2AE030E080E69AE00E94CC66B4
:10F300008091C00085FFFCCF8AE08093C600A7CF24
:10F310008F929F92AF92BF92CF92DF92EF92FF9225
:10F320000F931F93CF93DF93B4ECEB2EB6E0FB2E3D
:10F3300006EA1BE0C1E7DBE081E1C82E8CE0D82EB5
:10F34000F70181917F010E94B368882319F10E941F
:10F3500020694B015C01F6018081811103C060913D
:10F360005C0B01C061E070E080E090E00F9415D884
:10F37000F80120813181428153810F9448DA9B0149
:10F38000AC01C501B4010F949AD6688379838A834E
:10F390009B8309C0F80180819181A281B381888318
:10F3A0009983AA83BB830C5F1F4F2496FFEFCF1A6C
:10F3B000DF0A88ECE81686E0F80611F686E40E947B
:10F3C000B3688823D9F00E9420696B017C016093A7
:10F3D000610B7093620B8093630B9093640B20E03E
:10F3E00030E0A9010F9476D9181644F4C0920C02AB
:10F3F000D0920D02E0920E02F0920F02DF91CF91B7
:10F400001F910F91FF90EF90DF90CF90BF90AF9042
:10F410009F908F9008957CDF89E40E94B3688823D1
:10F4200059F00E9420696093650B7093660B80937E
:10F43000670B9093680B08C01092650B1092660BD7
:10F440001092670B1092680B8AE40E94B3688823BD
:10F4500059F00E9420696093690B70936A0B809346
:10F460006B0B90936C0B08951092690B10926A0BC2
:10F4700010926B0B10926C0B0895CF92DF92EF926B
:10F48000FF92CF93DF93EC01BC016C5F7F4F0E9432
:10F49000E16B20E030E0A901609135027091360205
:10F4A00080913702909138020F949AD66B017C01BB
:10F4B0009B01AC01688579858A859B850F9473D7FC
:10F4C00087FF04C0C886D986EA86FB86C0902902D9
:10F4D000D0902A02E0902B02F0902C02A701960116
:10F4E000688579858A859B850F9476D9181624F4CA
:10F4F000C886D986EA86FB86DF91CF91FF90EF9090
:10F50000DF90CF9008952F923F924F925F926F922B
:10F510007F928F929F92AF92BF92CF92DF92EF92A3
:10F52000FF920F931F93CF93DF93CDB7DEB7AB97C7
:10F530000FB6F894DEBF0FBECDBF9F878E87798B45
:10F54000688B5B8B4A8B3D8B2C8B1F8B0E8BED82DC
:10F55000DC018D909D90AD90BC904090A60B50909A
:10F56000A70B6090A80B7090A90BDB018D919D916A
:10F570000D90BC91A02D88879987AA87BB87C090E2
:10F58000AA0BD090AB0BE090AC0BF090AD0B2091A0
:10F59000AE0B3091AF0B4091B00B5091B10BEA899B
:10F5A000FB8960817181828193810F9499D6688FE4
:10F5B000798F8A8F9B8F80912513811173C0AE89BB
:10F5C000BF898D909D90AD90BC90EA89FB89E080C9
:10F5D000F18002811381A889B9892D913D914D91C6
:10F5E0005C91EE85FF856081718182819381FE014E
:10F5F0003596FF93EF93CC88DD880F94D027EE8566
:10F60000FF8580819181A281B3818093A60B909325
:10F61000A70BA093A80BB093A90BE889F989808167
:10F620009181A281B3818093AA0B9093AB0BA0939D
:10F63000AC0BB093AD0BEA89FB8980819181A281EB
:10F64000B3818093AE0B9093AF0BA093B00BB093AC
:10F65000B10BEC89FD8980819181A281B381809376
:10F66000B20B9093B30BA093B40BB093B50B0F9068
:10F670000F90AB960FB6F894DEBF0FBECDBFDF91F3
:10F68000CF911F910F91FF90EF90DF90CF90BF909F
:10F69000AF909F908F907F906F905F904F903F9032
:10F6A0002F900895A3019201C501B4010F9499D63A
:10F6B0002B013C0120E030E0A9010F9476D95301E1
:10F6C0004201181624F0B7FAB094B7F8B094A70125
:10F6D0009601688579858A859B850F9499D6688778
:10F6E00079878A879B8720E030E0A9010F9476D93B
:10F6F000288539854A855B8518160CF05058C50158
:10F70000B4010F949AD66B017C0120E030E0A9018E
:10F710000F9476D918160CF052CF20E030E040EF6D
:10F7200051E4C701B6010F947AD70F9460D70F94B4
:10F73000E2D77D876C87623071050CF440CF209151
:10F74000B20B3091B30B4091B40B5091B50BAC8917
:10F75000BD896D917D918D919C910F9499D66C8FFF
:10F760007D8F8E8F9F8F22242394312C8C859D85B5
:10F77000AA2797FDA095BA2F88A799A7AAA7BBA7E4
:10F78000DE011596BF83AE83B101882777FD809592
:10F79000982F0F9415D86B017C0168A579A58AA5CF
:10F7A0009BA50F9415D89B01AC01C701B6010F941E
:10F7B0007AD76B017C01EE89FF8980809180A280DD
:10F7C000B3802C8D3D8D4E8D5F8D0F9448DA9B015B
:10F7D000AC016091B20B7091B30B8091B40B90911E
:10F7E000B50B0F949AD669837A838B839C83288D7B
:10F7F000398D4A8D5B8DC701B6010F9448DA20918F
:10F80000AE0B3091AF0B4091B00B5091B10B0F94F8
:10F810009AD668A379A38AA39BA3288539854A85AC
:10F820005B85C701B6010F9448DA2091AA0B30918D
:10F83000AB0B4091AC0B5091AD0B0F949AD66CA3CF
:10F840007DA38EA39FA3A3019201C701B6010F94CC
:10F8500048DA2091A60B3091A70B4091A80B50914C
:10F86000A90B0F949AD6FF81FF932E812F93DE016F
:10F8700011966D01E8A0F9A00AA11BA12CA13DA140
:10F880004EA15FA10F94D027BFEF2B1A3B0A0F9018
:10F890000F90EC85FD852E163F0609F075CF8FCEB3
:10F8A0004F925F926F927F928F929F92AF92BF9290
:10F8B000CF92DF92EF92FF920F931F93CF93DF933C
:10F8C000CDB7DEB728970FB6F894DEBF0FBECDBF19
:10F8D00081E79BE0D2DD0F94A6CE6093580B709326
:10F8E000590B80935A0B90935B0B8091710B909105
:10F8F000720BA091730BB091740B8D839E83AF83B9
:10F90000B8879C01AD016091A60B7091A70B809107
:10F91000A80B9091A90B0F9473D7811197C04090B9
:10F92000750B5090760B6090770B7090780BA3015D
:10F9300092016091AA0B7091AB0B8091AC0B9091EE
:10F94000AD0B0F9473D7811181C020E030E040E708
:10F9500052E460910C0270910D0280910E02909120
:10F960000F020F947AD74B015C01E090790BF09075
:10F970007A0B00917B0B10917C0B82E99BE09F93AB
:10F980008F932DE7C22E2BE0D22EA30192016D8121
:10F990007E818F8198850F94D0270F900F90809152
:10F9A000710B9091720BA091730BB091740B8093BB
:10F9B000A60B9093A70BA093A80BB093A90B8091D3
:10F9C000750B9091760BA091770BB091780B80938B
:10F9D000AA0B9093AB0BA093AC0BB093AD0B8091A3
:10F9E000790B90917A0BA0917B0BB0917C0B80935B
:10F9F000AE0B9093AF0BA093B00BB093B10B809173
:10FA00007D0B90917E0BA0917F0BB091800B80932A
:10FA1000B20B9093B30BA093B40BB093B50B289695
:10FA20000FB6F894DEBF0FBECDBFDF91CF911F910F
:10FA30000F91FF90EF90DF90CF90BF90AF909F908D
:10FA40008F907F906F905F904F900895E090920B11
:10FA500060914F0270915002882777FD8095982F12
:10FA60000F9415D820910C0230910D0240910E0296
:10FA700050910F020F9448DA2EE333EC4EE259E333
:10FA80000F9448DA69837A838B839C838E010F5F9E
:10FA90001F4F2DE73BE049E75BE065E77BE081E74F
:10FAA0009BE031DD7CCF4F925F926F927F928F927D
:10FAB0009F92AF92BF92CF92DF92EF92FF920F93FD
:10FAC0001F93CF93C62FE091920BF0E0882309F4A7
:10FAD000D9C0DF01A257B44F8C918111AFC1809181
:10FAE000A60B9091A70BA091A80BB091A90B8093A6
:10FAF000710B9093720BA093730BB093740B809166
:10FB0000AA0B9091AB0BA091AC0BB091AD0B809375
:10FB1000750B9093760BA093770BB093780B809135
:10FB2000AE0B9091AF0BA091B00BB091B10B809345
:10FB3000790B90937A0BA0937B0BB0937C0BC090C6
:10FB4000B20BD090B30BE090B40BF090B50BC09219
:10FB50007D0BD0927E0BE0927F0BF092800BEE0F2C
:10FB6000FF1FEE0FFF1FE75CFD4F208131814281B7
:10FB70005381662349F06091190270911A028091B5
:10FB80001B0290911C0208C060911D0270911E0220
:10FB900080911F02909120020F947AD79B01AC01B3
:10FBA000C701B6010F949AD66093B20B7093B30B52
:10FBB0008093B40B9093B50B82EB9BE00F941D36B2
:10FBC00080900C0290900D02A0900E02B0900F0257
:10FBD00020E030E040E752E4609115027091160297
:10FBE00080911702909118020F9448DA60930C02EA
:10FBF00070930D0280930E0290930F02E091920B8E
:10FC0000F0E0E257F44F81E080834ADE20918A0BD6
:10FC100030918B0B40918C0B50918D0B6091AE0B02
:10FC20007091AF0B8091B00B9091B10B0F9499D65E
:10FC30007B018C016093AE0B7093AF0B8093B00B84
:10FC40009093B10B2091AA0B3091AB0B4091AC0B70
:10FC50005091AD0B6091A60B7091A70B8091A80BF2
:10FC60009091A90BE2EBCE2EEBE0DE2E0F947E34CA
:10FC700017DE80920C0290920D02A0920E02B092BA
:10FC80000F02DCC0E257F44F8081882309F4D6C00C
:10FC90008090A60B9090A70BA090A80BB090A90BFA
:10FCA0008092710B9092720BA092730BB092740BB6
:10FCB0004090AA0B5090AB0B6090AC0B7090AD0BCA
:10FCC0004092750B5092760B6092770B7092780B86
:10FCD0006091AE0B7091AF0B8091B00B9091B10B16
:10FCE0006093790B70937A0B80937B0B90937C0BD2
:10FCF0000091B20B1091B30B2091B40B3091B50B66
:10FD000000937D0B10937E0B20937F0B3093800B21
:10FD100020918A0B30918B0B40918C0B50918D0B65
:10FD20000F949AD67B018C016093AE0B7093AF0B4E
:10FD30008093B00B9093B10B32EBC32E3BE0D32EEC
:10FD4000A3019201C501B4010F947E341091920B6E
:10FD5000CC2389F02091820B3091830B4091840B4E
:10FD60005091850B6091190270911A0280911B02CB
:10FD700090911C0210C02091860B3091870B40910E
:10FD8000880B5091890B60911D0270911E02809129
:10FD90001F02909120020F949AD624E0129FF00146
:10FDA0001124E75CFD4F20813181428153810F9402
:10FDB0007AD79B01AC016091B20B7091B30B80912B
:10FDC000B40B9091B50B0F9499D66093B20B7093CE
:10FDD000B30B8093B40B9093B50B82EB9BE00F9425
:10FDE0001D36C0900C02D0900D02E0900E02F090F3
:10FDF0000F0220E030E040E752E460911102709180
:10FE0000120280911302909114020F9448DA6093C9
:10FE10000C0270930D0280930E0290930F02E091FA
:10FE2000920BF0E0E257F44F10823ADDC0920C02E0
:10FE3000D0920D02E0920E02F0920F02CF911F912C
:10FE40000F91FF90EF90DF90CF90BF90AF909F9079
:10FE50008F907F906F905F904F900895AF92BF9278
:10FE6000CF92DF92EF92FF920F931F93CF93DF9386
:10FE7000D82F2091690B30916A0B40916B0B5091F8
:10FE80006C0B6091650B7091660B8091670B909184
:10FE9000680B0F9483D9C62F172F082FF92E609166
:10FEA0004F0270915002882777FD8095982F0F940C
:10FEB00015D820910C0230910D0240910E02509104
:10FEC0000F020F9448DA20E030E040E752E40F944C
:10FED0007AD720E030E048EC52E40F947AD72091B2
:10FEE000920B2F93DF93FF920F931F93CF935B019E
:10FEF0006C01B2E0EB2E01E020E045E65BE061E75B
:10FF00007BE086EA9BE00F94501E8091710B9091EC
:10FF1000720BA091730BB091740B8093A60B90930E
:10FF2000A70BA093A80BB093A90B8091750B909190
:10FF3000760BA091770BB091780B8093AA0B9093DE
:10FF4000AB0BA093AC0BB093AD0B8091790B909160
:10FF50007A0BA0917B0BB0917C0B8093AE0B9093AE
:10FF6000AF0BA093B00BB093B10B80917D0B909130
:10FF70007E0BA0917F0BB091800B8093B20B90937E
:10FF8000B30BA093B40BB093B50B0F94A6CE6093B4
:10FF9000580B7093590B80935A0B90935B0B0F90F7
:10FFA0000F900F900F900F900F90DF91CF911F91B6
:10FFB0000F91FF90EF90DF90CF90BF90AF9008959A
:10FFC000CF93DF931F92CDB7DEB78C01E0E6FAE066
:10FFD0008491882341F09091C00095FFFCCF8093DD
:10FFE000C6003196F5CF70E04AE050E080E69AE036
:10FFF0000E940B67F8940F94574B179A1092970B27
:020000021000EC
:10000000169A1092980B149AE8E0FFE084918823E6
:1000100041F09091C00095FFFCCF8093C6003196CF
:10002000F5CFE8E1FCE885919491FC01249122232D
:1000300041F03091C00035FFFCCF2093C6000196FF
:10004000F4CF8091C00085FFFCCF8AE08093C6008A
:1000500001151105E1F0F8018491F801882349F0B8
:100060009091C00095FFFCCF8093C600319684919B
:10007000F5CF8091C00085FFFCCF8AE08093C60059
:10008000BE016F5F7F4FC8010F94DAB40BC0E091DF
:10009000DB0BF0E0EE0FFF1FEC5EF44785919491CF
:1000A0000F943072789406E010E00150110951F07D
:1000B00068EC70E080E090E00F94D5CE80E00F9483
:1000C000D4B1F3CFF894FFCFCF92DF92EF92FF92AB
:1000D0000F931F93CF93C82F8091EE109091EF1044
:1000E000039714F40E9482E60F94A6CE0091540B5D
:1000F0001091550B2091560B3091570BC090580B17
:10010000D090590BE0905A0BF0905B0B6C197D0965
:100110008E099F09061717072807390740F4012B96
:10012000022B032B21F064E08CEF98E049DF409133
:1001300008025091090260910A0270910B02452B4E
:10014000462B472B19F10F94A6CE0091580B109116
:10015000590B20915A0B30915B0B601B710B820B7A
:10016000930B009108021091090220910A0230912C
:100170000B02061717072807390740F4909112144D
:1001800080911114981302C0CC2349F0CF911F9194
:100190000F91FF90EF90DF90CF900D94FE25179A6E
:1001A0001092970B169A1092980B149AEFCF0F9407
:1001B000574B8091460B811142C081E08093460BE2
:1001C0008091D8109091D910A091DA10B091DB10E5
:1001D0008093D4109093D510A093D610B093D710DD
:1001E000E8E0FFE08491882341F09091C00095FF02
:1001F000FCCF8093C6003196F5CFEEE0FCE8859108
:100200009491FC012491222341F03091C00035FFEC
:10021000FCCF2093C6000196F4CF8091C00085FFEB
:10022000FCCF8AE08093C600E091DB0BF0E0EE0F9C
:10023000FF1FE851F947859194910D940572089537
:100240008091460B0895CF93DF93EC018091920B40
:100250008093470B84E50E94B368811102C080E05F
:1002600084C00E9420690F94E7D76093470B6623F0
:10027000B1F3E2E0FFE08491882341F09091C00067
:1002800095FFFCCF8093C6003196F5CFCD36D105D2
:1002900009F435C064F4C836D105B1F0C936D105CA
:1002A00009F052C0E8ECFAE8A591B49124C0CA3D27
:1002B000D10509F432C0CD3DD10509F045C0E0EBD0
:1002C000FAE8A591B4913DC0EAECFAE885919491E1
:1002D000FC012491222309F437C03091C00035FF7E
:1002E000FCCF2093C6000196F3CF9091C00095FFFC
:1002F000FCCF8093C6008D918111F7CF25C0E6EC2D
:10030000FAE8A591B4918D918823F1F09091C00005
:1003100095FFFCCF8093C600F6CFE2EBFAE8A591FB
:10032000B4918D91882381F09091C00095FFFCCF0E
:100330008093C600F6CF9091C00095FFFCCF8093CC
:10034000C6008D918111F7CF6091470B70E04AE0B4
:1003500050E080E69AE00E9404678091C00085FF2B
:10036000FCCF8AE08093C60081E0DF91CF910895B1
:100370004F925F926F927F928F929F92AF92BF92B5
:10038000CF92DF92EF92FF92CF93DF9300D01F9234
:10039000CDB7DEB72B013C0129833A834B835C83C5
:1003A0008DEE9FE00F94E6E28F3F01F58EEE9FE029
:1003B0000F94E6E28F3FD1F48FEE9FE00F94E6E2D8
:1003C0008F3FA1F480EF9FE00F94E6E28F3F71F43E
:1003D00040E050E0BA018DEE9FE00F940AE340E068
:1003E00050E0BA0181EF9FE00F940AE381EF9FE0B4
:1003F0000F94EEE24B015C018DEE9FE00F94EEE274
:100400006B017C0169817A818B819C812CE330E0D6
:1004100040E050E00F944ADCC20ED31EE41EF51EED
:10042000B701A6018DEE9FE00F940AE3C301B2016C
:1004300028EE33E040E050E00F944ADCBA01A90115
:10044000480D591D6A1D7B1D81EF9FE00F940AE343
:100450001092D40B1092D50B1092D60B1092D70B92
:100460000F900F900F900F90DF91CF91FF90EF9032
:10047000DF90CF90BF90AF909F908F907F906F90C4
:100480005F904F900895CF92DF92EF92FF9220916C
:10049000B60B2223F1F020E030E040E05FE30F9460
:1004A00048DA6B017C0120E030E0A9010F9473D79A
:1004B000882379F0A7019601C701B6010F9448DAA5
:1004C0002BED3FE049E450E40F9448DA9B01AC0186
:1004D00004C020E030E040E85FE360E070E080E8E6
:1004E0009FE30F947AD7FF90EF90DF90CF9008951D
:1004F00060913D0270913E0280913F0290914002D6
:10050000C2DF6093390270933A0280933B0290936A
:100510003C020895CF93DF93EC010F94BD5281E02C
:10052000D3DD80E00F94D4B1209799F0C233D10588
:1005300040F062E370E080E090E00F94D5CEE29767
:10054000ECCFBE0180E090E00F94D5CEC0E0D0E0CB
:10055000E4CFDF91CF9108952F923F924F925F9217
:100560006F927F928F929F92AF92BF92CF92DF92C3
:10057000EF92FF921F93CF93DF934B015C01CC244A
:10058000CA94DC2C760165E5262E6AE0362E78EEDC
:10059000472E73E0572E612C712C1AE08091810B4D
:1005A000811126C12FEFC216D206E206F20651F0E3
:1005B000F7FC1EC10F94A6CE6C197D09683B7B40E9
:1005C00008F016C10F94A6CE681979098A099B090B
:1005D000693E73408105910508F47FC08091301C0D
:1005E000811177C0EDE5FAE08491882341F0909184
:1005F000C00095FFFCCF8093C6003196F5CFE09107
:10060000470B24E0E29FF0011124E35EF44E4081A9
:1006100051816281738121E030E080E69AE00E949E
:100620000268E9E5FAE08491882341F09091C000E6
:1006300095FFFCCF8093C6003196F5CF6091470BB4
:1006400070E04AE050E080E69AE00E940467F10121
:100650008491E5E5FAE0882349F09091C00095FF88
:10066000FCCF8093C60031968491F5CFF7FE03C08E
:10067000EBEBF9E025C00F94A6CE4B015C01C7015E
:10068000B6016854744F8F4F9F4F681979098A09D2
:100690009B09A30192010F944ADCBA01A9012AE047
:1006A00030E080E69AE00E94CC668091C00085FF31
:1006B000FCCF0DC09091C00095FFFCCF8093C60089
:1006C00081918111F7CF8091C00085FFFCCF1093FD
:1006D000C6000F94A6CE4B015C010F94BD5280E082
:1006E000F3DC80E00F94D4B1FFEFCF16DF06EF0606
:1006F000FF0609F046C08091450BE091470BF0E002
:10070000EF01CC0FDD1FCC0FDD1FC35ED44EEE0F0B
:10071000FF1FEB5DF44E8823D1F080819181BC01F5
:10072000882777FD8095982F0F9415D820E030E02A
:1007300040E85FE30F9499D69B01AC016881798111
:100740008A819B810F9476D987FF4DC027CF808106
:100750009181BC01882777FD8095982F0F9415D83B
:1007600020E030E040E85FE30F949AD69B01AC01B3
:10077000688179818A819B810F9473D718169CF5C3
:100780000DCFF7FC0BCFE091470BF0E0EF01CC0F62
:10079000DD1FCC0FDD1FC35ED44EEE0FFF1FEB5DE0
:1007A000F44E80819181BC01882777FD8095982F38
:1007B0000F9415D89B01AC01688179818A819B8156
:1007C0000F9499D60F94E2D797FF07C09095809524
:1007D000709561957F4F8F4F9F4F663071058105F2
:1007E00091050CF4DBCE0F94A6CE6B017C01D6CE26
:1007F000DF91CF911F91FF90EF90DF90CF90BF904E
:10080000AF909F908F907F906F905F904F903F90B0
:100810002F900895CF93DF931F921F92CDB7DEB72D
:10082000BE016F5F7F4F88EF9FE00F942B7189812E
:100830009A818156904F803A9F4020F11A82198206
:10084000ECE2FAE08491882341F09091C00095FF9A
:10085000FCCF8093C6003196F5CF8091C00085FF14
:10086000FCCF8AE08093C600BE016F5F7F4F88EFA8
:100870009FE00F941A718FEE99E00F9477BE81E09C
:100880000F949BB40F900F90DF91CF9108952F920A
:100890003F924F925F926F927F928F929F92AF9210
:1008A000BF92CF92DF92EF92FF920F931F93CF935D
:1008B000DF93CDB7DEB7CA58D2400FB6F894DEBF8B
:1008C0000FBECDBFC958DD4F688379838A839B8370
:1008D000C757D240FE01E75FFD4F88E2DF011D925E
:1008E0008A95E9F7E850F24080E991E0DF019C0148
:1008F0001D9221503040E1F7C75ADD4F198218820E
:10090000C955D240CE01875A9D4F5C014E019FE6EA
:10091000891A9EEF990ADE01AF51BE4F3D0190EB5F
:10092000C92E9FE0D92E23E2E22EF12C00E010E048
:10093000C359DD4F8882CD56D240CD58DD4F9882C5
:10094000C357D240B701882777FD8095982F0F9421
:1009500015D8D3016D937D938D939D933D01F50142
:10096000619171915F01882777FD8095982F0F9491
:1009700015D8D4016D937D938D939D934D010F5F99
:100980001F4F0630110559F0B501C6010F942B71A8
:10099000B5E0EB0EF11CE2E0CE0ED11CD3CFCF516F
:1009A000DE4F288139814A815B81C15ED140C958BF
:1009B000DD4F688179818A819B81C757D2400F942E
:1009C00073D787FD2BC3FE01EF51FE4F7F016E01F0
:1009D000FFE2CF1AFEEFDF0A3E012BEB621A2DEF8A
:1009E000720AC359DD4F0881CD56D240CD58DD4F34
:1009F0001881C357D24085E090E0CF58DD4F9983EE
:100A00008883C157D240CF58DD4FA881B981C157E3
:100A1000D2401197CF58DD4FB983A883C157D24038
:100A2000F7012089318942895389648975898689CA
:100A300097890F9499D64B015C01D80150962D915E
:100A40003D914D915C91539754966D917D918D910F
:100A50009C9157970F9499D6A50194010F947AD73A
:100A6000F60192938293729362936F01D301BE92C7
:100A7000AE929E928E923D0104501109B4E0EB1AA1
:100A8000F108CF58DD4FE881F981C157D240EF2BF3
:100A900009F0B9CF6E01FFECCF1AFDEFDF0A3E017E
:100AA00027E4621A2EEF720A2E013DE3430E511C19
:100AB000CE0101967C0101E010E0D6018D909D9061
:100AC000AD90BC90139714962D913D914D915C91F2
:100AD0001797C501B4010F949AD69B01AC010F94EE
:100AE0009AD6F70164A775A786A797A701301105C5
:100AF00041F080A691A6A2A6B3A684829582A68282
:100B0000B7820F5F1F4FD30114962D913D914D91E8
:100B10005C91179718966D917D918D919C911B9783
:100B20000F9499D620E030E040EC50E40F9448DA7E
:100B3000F2016083718382839383F4E0CF0ED11C32
:100B40002CE2E20EF11C34E0630E711C88E2480EC8
:100B5000511C0530110509F0B0CF8E010B5A1F4F03
:100B60006E0191E5C90ED11C22242394312C2C0E48
:100B70003D1EA8ED2A0E311CF801B8972081318165
:100B800042815381F80160817181828193810F9448
:100B90007AD74B015C01E12CF12C3601F8E26F1A97
:100BA000710826014E0C5F1CF301EE0DFF1D248120
:100BB000358146815781C501B4010F9448DA9B0104
:100BC000AC01D20114966D917D918D919C911797F6
:100BD0000F9499D6F2016483758386839783F4E03A
:100BE000EF0EF11C24E1E216F104D9F6045D1F4F6B
:100BF00038E2C30ED11C0215130509F0BDCF1E014A
:100C000085EB280E311C6E0191EBC90ED11C3E0103
:100C1000A7EE6A1AADEF7A0A14E0E12EF12C270153
:100C200000E010E0812C912CA12CB12CF601E00FFA
:100C3000F11FD301A00FB11F2D913D914D915C91FA
:100C400060817181828193810F9448DA9B01AC01AC
:100C5000B401C5010F949AD64B015C01BFEF4B1A4A
:100C60005B0A0C5F1F4FE5E04E165104F9F69B013D
:100C7000AC01D1016D917D918D919C910F9499D68C
:100C8000F60120813181428153810F947AD7D301BB
:100C90006D937D938D939C931397B1E0EB1AF108BC
:100CA000E8E22E1A3108FCE2CF1AD10824E0621AD9
:100CB0007108E114F10409F0B2CFCB50DE4F888106
:100CC0009981AA81BB81C55FD140C957DD4F888317
:100CD0009983AA83BB83C758D2408E01075F1D4FFB
:100CE000DE01AF5CBD4FC558DD4FB983A883CB573C
:100CF000D240C359DD4F2880CD56D240CD58DD4F6C
:100D00003880C357D240FE01EF51FE4FC358DD4F2C
:100D1000F983E883CD57D240C358DD4FA881B9810C
:100D2000CD57D240CD90DD90ED90FD90C358DD4F72
:100D3000B983A883CD57D240C958DD4F2881398166
:100D40004A815B81C757D240C701B6010F9473D760
:100D50001816B4F0C358DD4FE881F981CD57D24061
:100D60002081318142815381C958DD4F6881798169
:100D70008A819B81C757D2400F9473D71816FCF411
:100D8000CF58DD4F28813981C157D24024303105F9
:100D900009F01FC1C957DD4F288139814A815B8124
:100DA000C758D240C958DD4F688179818A819B81BB
:100DB000C757D2400F9476D918160CF00AC1D80143
:100DC00014968D919D910D90BC91A02DC158DD4F31
:100DD00088839983AA83BB83CF57D240F801408090
:100DE000518062807380C558DD4FA881B981CB578F
:100DF000D2408D919D910D90BC91A02DC359DD4F96
:100E000088839983AA83BB83CD56D240D1018D912B
:100E10009D910D90BC91A02DCD57DD4F8883998376
:100E2000AA83BB83C358D240A7019601C958DD4F9E
:100E3000688179818A819B81C757D2400F9499D666
:100E4000CD58DD4F688379838A839B83C357D24013
:100E500020E030E040E450E40F94ABDA6B017C0119
:100E6000A3019201C158DD4F688179818A819B81FC
:100E7000CF57D2400F9499D64B015C0120E030E06F
:100E800040EC50E4C359DD4F688179818A819B81B0
:100E9000CD56D2400F9448DA9B01AC01C501B40194
:100EA0000F947AD7A70196010F9448DA6B017C0161
:100EB00020E030E040E05FE3C301B2010F9448DA84
:100EC0004B015C01CD58DD4F288139814A815B811E
:100ED000C357D240CA01B9010F9448DA9B01AC0153
:100EE000C501B4010F9448DA9B01AC01C701B601FA
:100EF0000F949AD66B017C01CD57DD4F2881398143
:100F00004A815B81C358D240F10164817581868139
:100F100097810F9499D6C359DD4F288139814A8131
:100F20005B81CD56D2400F947AD74B015C01C359F7
:100F3000DD4F288139814A815B81CD56D240CA017B
:100F4000B9010F949AD6A30192010F9448DA2B01AC
:100F50003C01C359DD4F288139814A815B81CD56DF
:100F6000D240C158DD4F688179818A819B81CF57FA
:100F7000D2400F9448DA9B01AC01C301B2010F9437
:100F80009AD620E030E040EC50E40F947AD79B01F1
:100F9000AC01C501B4010F9499D6CD58DD4F28811D
:100FA00039814A815B81C357D2400F9448DA9B0153
:100FB000AC01C701B6010F949AD6CD57DD4F2881F9
:100FC00039814A815B81C358D2400F949AD64B0134
:100FD0005C01CF58DD4F28813981C157D2402F5F46
:100FE0003F4FCF58DD4F39832883C157D2400C5F24
:100FF0001F4FC558DD4F88819981CB57D240049649
:10100000C558DD4F99838883CB57D24094E0290E91
:10101000311C2530310509F07FCE04C0812C912C84
:10102000A12CB12CB401C501C657DD4F0FB6F89401
:10103000DEBF0FBECDBFDF91CF911F910F91FF900B
:10104000EF90DF90CF90BF90AF909F908F907F9068
:101050006F905F904F903F902F90089580910C0C6F
:101060008823C9F086EA9FE00F94E6E2882399F08E
:101070006091171B7091181B8091191B90911A1B7E
:1010800006DC2091F6193091F7194091F81950912A
:10109000F9190D947AD760E070E0CB0108954F9272
:1010A0005F926F927F928F929F92AF92BF92CF92F8
:1010B000DF92EF92FF920F931F93CF93DF93CDB701
:1010C000DEB728970FB6F894DEBF0FBECDBF0F94E2
:1010D0005F4180914F02909150029093100C809349
:1010E0000F0CE091920BF0E0EE0FFF1FEB5DF44E62
:1010F00060817181882777FD8095982F0F9415D88E
:101100006093000C7093010C8093020C9093030C7D
:101110008091900B9091910B9093FF0B8093FE0B1D
:101120000F94A6CE6093E60B7093E70B8093E80BC9
:101130009093E90B8091A60B9091A70BA091A80B1F
:10114000B091A90B89839A83AB83BC838093EE0B08
:101150009093EF0BA093F00BB093F10B4090AA0B80
:101160005090AB0B6090AC0B7090AD0B4092F20BBB
:101170005092F30B6092F40B7092F50B8091AE0BD2
:101180009091AF0BA091B00BB091B10B8D839E836A
:10119000AF83B8878093F60B9093F70BA093F80B6F
:1011A000B093F90B6091B20B7091B30B8091B40BBB
:1011B0009091B50B6093FA0B7093FB0B8093FC0B33
:1011C0009093FD0B20E030E040E85FE30F9499D668
:1011D0006093B20B7093B30B8093B40B9093B50BE9
:1011E00082E99BE09F938F93812C912CB8ECAB2EDE
:1011F000B3E4BB2E12EBC12E1BE0D12EED80FE809E
:101200000F811885A301920169817A818B819C816C
:101210000F94D02720E030E040EA51E46091AE0B1B
:101220007091AF0B8091B00B9091B10B0F949AD647
:101230002B013C010F900F9020E030E042E553E499
:101240000F9476D918164CF04092AE0B5092AF0B1B
:101250006092B00B7092B10B0CC080E090E0A2E500
:10126000B3E48093AE0B9093AF0BA093B00BB0930D
:10127000B10BE090AE0BF090AF0B0091B00B109162
:10128000B10B2091AA0B3091AB0B4091AC0B50915C
:10129000AD0B6091A60B7091A70B8091A80B90915C
:1012A000A90BA2E96A2EABE07A2E7F926F92812C75
:1012B000912CB0E7AB2EB1E4BB2EE2EBCE2EEBE0EF
:1012C000DE2E0F94D0271092261B1092251B109211
:1012D000281B1092271B10922A1B1092291B80E0BA
:1012E00090E0A8E4B2E48093A60B9093A70BA093A0
:1012F000A80BB093A90B80E090E0AEE3B3E4809339
:10130000AA0B9093AB0BA093AC0BB093AD0BE090FA
:10131000AE0BF090AF0B0091B00B1091B10B7F9220
:101320006F92812C912CF8E4AF2EF2E4BF2E9C0139
:10133000AD01C501B4010F94D0271092910B10920A
:10134000900B0F900F900F900F9028960FB6F89477
:10135000DEBF0FBECDBFDF91CF911F910F91FF90E8
:10136000EF90DF90CF90BF90AF909F908F907F9045
:101370006F905F904F900D945F41E091920B84E0ED
:10138000E89FF0011124E35EF44E408151816281B7
:101390007381ECEEF9E08491882341F09091C000D4
:1013A00095FFFCCF8093C6003196F5CF22E030E068
:1013B00080E69AE00E940268E8EEF9E084918823D2
:1013C00041F09091C00095FFFCCF8093C60031960C
:1013D000F5CF6091920B70E04AE050E080E69AE031
:1013E0000E940467E4EEF9E08491882341F0909133
:1013F000C00095FFFCCF8093C6003196F5CF409199
:101400000B1B50910C1B60910D1B70910E1B21E06A
:1014100030E080E69AE00E9402688091C00085FF7B
:10142000FCCF8AE08093C6000895CF93DF93CDB7B9
:10143000DEB72A970FB6F894DEBF0FBECDBF0F946C
:10144000A6CE6F83788789879A87179A1092970B11
:10145000169A1092980BEFEDF9E08491882341F0F1
:101460009091C00095FFFCCF8093C6003196F5CFD8
:101470008091C00085FFFCCF8AE08093C60083E4A2
:101480000F94C0601C014090D0105090D11060901B
:10149000D2107090D3100F94AB36481A590A6108D5
:1014A00071080E94B9EB481A590A6108710877FE61
:1014B00003C0412C512C32019091121480911114CF
:1014C000981799F0E091111427E5E29FF00111249B
:1014D000ED5EFB4E20E030E040E752E462A173A1F4
:1014E00084A195A10F9448DA08C060910C02709114
:1014F0000D0280910E0290910F020F94E2D77E832D
:101500006D830F9455260E9460E410921B0C789412
:1015100020E030E040E85FE36091B20B7091B30BE4
:101520008091B40B9091B50B0F9499D669837A830F
:101530008B839C83E090AE0BF090AF0B0091B00BCF
:101540001091B10B2091AA0B3091AB0B4091AC0BD9
:101550005091AD0B6091A60B7091A70B8091A80BD9
:101560009091A90BA2E9BBE0BF93AF93812C912C82
:10157000E8ECAE2EE3E4BE2EDE0111966D010F9471
:10158000D02720E030E040E85FE36091B20B70913B
:10159000B30B8091B40B9091B50B0F9499D66983DE
:1015A0007A838B839C832FE832EC45EF5FE3609175
:1015B000AE0B7091AF0B8091B00B9091B10B0F946B
:1015C0009AD66B017C0167E074E062197309F4E05C
:1015D00076956795FA95E1F780E090E00F9413D83F
:1015E0002091F6193091F7194091F8195091F91995
:1015F0000F947AD79B01AC01C701B6010F949AD61C
:101600007B018C012091AA0B3091AB0B4091AC0B6C
:101610005091AD0B6091A60B7091A70B8091A80B18
:101620009091A90BA2E9BBE0BF93AF93812C912CC1
:10163000A0E2AA2EA2E4BA2EDE0111966D010F944B
:10164000D027B301A20181E99FE00F940AE30F9034
:101650000F900F900F9005E71FE0F12CB3E0EB2EF9
:1016600080912513882341F18F2D6E2D0F9416DC68
:10167000B5E18B02F001112423E09202E00DF11D8F
:101680001124EE0FFF1FEE0FFF1FEB5DFC4E20E05D
:1016900030E04AE754E461817281838194810F9440
:1016A00048DA20E030E040E05FE30F949AD60F94F0
:1016B00050D80F94E2D702C060E070E0C8010F94E8
:1016C00012E3F3940E5F1F4F89E0F812C9CFB10106
:1016D00083E79FE00F9412E34091A60B5091A70B74
:1016E0006091A80B7091A90B8DE99FE00F940AE31C
:1016F0004091AA0B5091AB0B6091AC0B7091AD0B6C
:1017000081EA9FE00F940AE34091AE0B5091AF0B3A
:101710006091B00B7091B10B8DE89FE00F940AE3DC
:10172000BE016B5F7F4F89E89FE00F941A71E091D3
:10173000920BF0E0EE0FFF1FEB5DF44E60818CE842
:101740009FE00F94F8E26091231B8BE89FE00F94D9
:10175000F8E26091900B88E89FE00F94F8E261E076
:1017600085EA9FE00F94F8E20F945F41EAEDF9E01B
:101770008491882341F09091C00095FFFCCF809325
:10178000C6003196F5CF83E40F94C0604AE050E084
:10179000BC0180E69AE00E94616784E69FE00F94B6
:1017A000E6E261E0680F84E69FE00F94F8E2EFEC78
:1017B000F9E08491882341F09091C00095FFFCCF1F
:1017C0008093C6003196F5CF8091C00085FFFCCF95
:1017D0008AE08093C6000F94A6CEAB01BC018F8136
:1017E0009885A985BA85481B590B6A0B7B0B2AE0A3
:1017F00030E080E69AE00E946D67F894FFCF6F9822
:101800007798EAE6F0E080818F7B80838081806832
:101810008083EF9A08951F920F920FB60F921124B2
:101820000BB60F920F931F932F933F934F935F939A
:101830006F937F938F939F93AF93BF93EF93FF9398
:101840008091900B9091910B8B3491050CF441C0D9
:1018500080916A0086FF0BC00F94A6CE6093E20BC6
:101860007093E30B8093E40B9093E50B2CC00F94E3
:10187000A6CE0091E20B1091E30B2091E40B309186
:10188000E50B601B710B820B930B2091900B309139
:10189000910B253631052CF003E010E020E030E01C
:1018A00004C004E010E020E030E060177107820718
:1018B000930748F08091BD0B9091BE0B02969093D8
:1018C000BE0B8093BD0B80916A0090E489278093C2
:1018D0006A00FF91EF91BF91AF919F918F917F919E
:1018E0006F915F914F913F912F911F910F910F90A9
:1018F0000BBE0F900FBE0F901F9018956C987498A8
:10190000EAE6F0E080818160808380818D7F808342
:10191000EC9A08951F920F920FB60F9211240BB6F6
:101920000F922F933F934F935F936F937F938F9378
:101930009F93AF93BF93EF93FF93EC98EAECF9E09A
:101940008491882341F09091C00095FFFCCF809353
:10195000C6003196F5CF8091C00085FFFCCF8AE0AC
:101960008093C60080911B0C81115FDDFF91EF9188
:10197000BF91AF919F918F917F916F915F914F91A7
:101980003F912F910F900BBE0F900FBE0F901F90A5
:101990001895BF92CF92DF92EF92FF920F931F9311
:1019A000CF93DF93CDB7DEB7E1970FB6F894DEBFE4
:1019B0000FBECDBF88E89FE00F94E6E2B82EBE01CF
:1019C000605D7F4F89E89FE00F942B71E3E7F8E0BB
:1019D0008491882341F09091C00095FFFCCF8093C3
:1019E000C6003196F5CF68A979A94AE050E080E6B3
:1019F0009AE00E940B678E01015E1F4F85E9E82E79
:101A00008FE0F82ED02EC12EC7010F94E6E2F80128
:101A100081938F01FFEFEF1AFF0A8DE9E8168FE03F
:101A2000F80691F71FA2ED2DFC2D8191882339F046
:101A30009091C00095FFFCCF8093C600F6CF6EE674
:101A400078E08D2D9C2D0F9495DFCF92DF9287E665
:101A500098E09F938F938E010F5F1F4F1F930F93FB
:101A60000F94BAE00F900F900F900F900F900F907F
:101A70007E0195E0E90EF11CF7018081882349F091
:101A8000992787FD90950F9484DFF70181937F015B
:101A9000F3CF60E0C8010E94D6E481E99FE00F9493
:101AA000EEE2F62EE72ED82EC92EECE4F8E0849173
:101AB000882341F09091C00095FFFCCF8093C60031
:101AC0003196F5CF2AE030E04F2D5E2D6D2D7C2D27
:101AD00080E69AE00E946D6761E088E498E00E94E9
:101AE000D6E463E478E0C8010F94A0DF8DE99FE0BD
:101AF0000F94EEE26CA77DA78EA79FA7CE018C96D0
:101B00000F947976BC01C8010F942FE060E478E06F
:101B1000C8010F9495DF81EA9FE00F94EEE26CA775
:101B20007DA78EA79FA7CE018C960F947976BC01D6
:101B3000C8010F942FE069E378E0C8010F9495DFA6
:101B400060E0C8010E94D6E464E378E0C8010F9425
:101B5000A0DF8DE89FE00F94EEE26CA77DA78EA733
:101B60009FA7CE018C960F947976BC01C8010F9483
:101B70002FE060E0C8010E94D6E461E089E298E0CD
:101B80000E94D6E489A98F9388A98F9382E298E076
:101B90009F938F931F930F930F94BAE060E0C80157
:101BA0000E94D6E46BE178E0C8010F94A0DF8B2D92
:101BB00090E09DA78CA7CE018C960F944E79BC0126
:101BC000C8010F942FE060E0C8010E94D6E4CF92D4
:101BD000DF92EF92FF9282E198E09F938F931F93A1
:101BE0000F930F94BAE060E0C8010E94D6E461E070
:101BF0008EE098E00E94D6E40FB6F894DEBF0FBEE8
:101C0000CDBFE1960FB6F894DEBF0FBECDBFDF911A
